:020000040800F2
:1000000000200010412A0308B192020899690008F3
:10001000AD920208A9920208A59202080000000011
:10002000000000000000000000000000A192020893
:100030009D92020800000000999202089D7E00082F
:10004000A92A0308A92A0308A92A0308A92A030838
:10005000A92A0308A92A030889200008B521000855
:10006000792100083D210008012100081135000810
:1000700001350008F1340008E1340008D1340008EB
:10008000BD340008A9340008A92A0308A92A0308D6
:100090008D960208A92A0308A92A0308C52000088A
:1000A0000570000865700008A92A0308757000082B
:1000B000557000084570000835700008A92A03082B
:1000C000A92A0308A92A0308A92A0308A92A0308B8
:1000D000A92A030821800008A57F0008297F0008BD
:1000E0004F200008A92A030889920208A92A0308B8
:1000F00015700008A92A030825700008A92A03081A
:10010000000000000000000000000000A92A030811
:10011000A92A0308A92A030819B40108FDB3010894
:1001200095340008813400086D3400085934000803
:1001300045340008A92A0308000000000000000060
:10014000A92A0308A92A0308A92A03080000000015
:10015000000000000000000000000000000000009F
:100160000000000000000000A92A0308A92A0308D3
:10017000A92A0308000000000000000000000000A1
:0801800000000000A92A030899
:100188000A4B30B503F1140493F900205D78072A6F
:10019800C8BF143A811804330D7313F8025C8554F0
:1001A80013F8012C0A76A342EED130BD045403089B
:1001B80003682DE9F041DF691FB13B46BDE8F04116
:1001C8001847002A164611DD04460D460E4400E085
:1001D80023689B68204698470028F9D0236815F8BB
:1001E800011B1B6820469847AE42F1D1BDE8F0815B
:1001F80000232322027043708370C3707047152355
:1002080003701623C370172383712D2343702E2385
:1002180003712F23C37170472DE9F041846814B12D
:100228002568A4882C8541F08001446840F2E935AE
:1002380001E0002D5AD02689013D16F0020FADB21B
:10024800F7D0217304F10C0640F2E93101E00029EE
:100258005DD02589013915F0010F89B2F7D03178C1
:100268004468A1894FF0000C4FF47A714FF6FF767D
:100278004FF0FF0E634502D130E0B1421ED0258910
:10028800013915F0020589B2F7D084F80CE004F1C1
:100298000C084FF47A7102E0B9B2B1420ED0258948
:1002A80015F0010501F1FF37F6D098F80050EDB2CE
:1002B8000AB1157001320CF1010CDBE71C4B9C42B2
:1002C80004D0A3F578439C4208D10125194B03EBD0
:1002D80005156B8901339BB26B816B89836813B1F8
:1002E8001A689B8893610120BDE8F08110498C420F
:1002F80004D0A1F578418C42B3D101250D4901EB19
:1003080005156989013189B269816989A9E7084DAB
:10031800AC4203D008498C42A2D10121054C04EB20
:1003280001114C890134A4B24C814989446898E789
:1003380000300140F86F00200038004030B4836876
:1003480013B11C689B882385436840F2E93401E0B7
:10035800002C37D01D89013C15F0020FA4B2F7D04C
:10036800197303F10C0540F2E93101E000294BD083
:100378001C89013914F0010F89B2F7D02B78436832
:1003880040F2E93101E000292DD01C89013914F02F
:10039800020F89B2F7D01A7303F10C0440F2E93264
:1003A80001E0002A41D01989013A11F0010F92B2F7
:1003B800F7D02378836813B11A689B88936101206A
:1003C80030BC704721498B4204D0A1F578418B425B
:1003D800D6D101241E4901EB04146189013189B287
:1003E80061816189CCE7194A934204D0A2F5784229
:1003F8009342DFD10121164B03EB01114B890133E5
:100408009BB24B814B89D5E7104CA34203D01149CD
:100418008B42B4D101210E4B03EB01114B890133FF
:100428009BB24B814B894368AAE708498B4203D0AA
:10043800084A9342BED10122054B03EB02125389AD
:1004480001339BB253815389B4E700BF00300140A8
:10045800F86F002000380040002870B51EDB09281E
:10046800044620DD012303EB83035B00B0FBF3F2BA
:10047800092AF8D87BB10E4EB4FBF3F00928CCBF9B
:1004880057223022A6FB03E5024403FB1044EB0885
:1004980001F8012BF0D100230B7070BD2D230B70D8
:1004A80040420131DBE7303001F8010BF3E700BFD0
:1004B800CDCCCCCC884230B44FF001042ED301FB14
:1004C80004F4B0FBF4F58D42F9D284B1AAB901E085
:1004D800B0FBF4F5092DCCBF572230222A4404FB87
:1004E800150003F8012BB4FBF1F4002CF0D1002225
:1004F8001A7030BC7047B0FBF4F5092DCCBF372219
:1005080030222A4404FB150003F8012BB4FBF1F454
:10051800002CF0D100221A7030BC70470546002A22
:10052800EBD1D7E703685A1C0260197070472DE9B0
:10053800F047089C2578002B804689460CBF4FF071
:10054800200A4FF0300A661C35B3002A29DD3346ED
:1005580001E0024698B113F8011B501E0029F8D19A
:10056800971E60B13D46013D51464046C8476B1C49
:10057800002BF8DC257827EAE770013055B1041B19
:1005880029464046C847301916F8015B002DF7D1B7
:10059800BDE8F087BDE8F087002A04DC2846BDE8FE
:1005A800F0870020EBE7571EDCE783684268D0ED50
:1005B800037A00EB83010133934281ED040A8360DF
:1005C80004BF0023836000EB830393ED047A036880
:1005D80070EE277A9A42C0ED037A77EEC77AC0EDBB
:1005E800037A0CDA013307EE103AF8EEC76AB7EE71
:1005F800007A87EEA60A036030EE070A704707EE16
:10060800102AB8EEC77A87EE870A704790ED057A08
:1006180090ED004AD0ED066AD0ED014AD0ED047A9B
:1006280090ED035AD0ED025AA4EE007AB0EE406A7B
:10063800B0EE470AB0EE667AA6EE247A67EEC07A84
:10064800A0EE457AE6EE257A80ED057AC0ED067AC9
:100658007047D0ED057A90ED013AD0ED003AD0ED33
:10066800064A90ED024A90ED077A90ED035A90ED14
:10067800086AD0ED045AC0ED067AF0EE406A27EE1B
:10068800830AC0ED056AA3EEA60A80ED087AA4EEF7
:10069800240AA5EE470AA5EEC60A80ED070A7047A8
:1006A800D0ED007A90ED017A30EE670AE7EE007A35
:1006B800B0EE670AC0ED007A704770470A4491426D
:1006C80014D030B40139551E41F2210211F8014FFE
:1006D800082380EA042004044CBF82EA400040005A
:1006E800013B80B2F7D18D42F0D130BC70472DE983
:1006F800F04FDFF820B2DFF820E2BBF80020DEF888
:100708000060BBF90430BBF90250BBF90A80C2EBA8
:10071800261404FB04F424135200C2EBE60203FB84
:1007280004F305FB02F29B1303EBE223B3F5FA365D
:100738004FEAE37589B045F1FF373246A6FB064517
:10074800CDE9024502FB07F205EB4202CDE9046759
:10075800029EBBF90840039208FB02FC4FEAE879C5
:1007680006FB09CC3A46A8FB0689049ECBF818304C
:10077800E51704FB02F206FB0522A4FB0667E14429
:1007880017444FEA182242EA096200924FEA2922E6
:1007980001923D03DDE90078340345EA16553F1917
:1007A800BBF80660069048EB05083C1C48F5004578
:1007B80003EB8302A4FB068906FB0599803213121A
:1007C8004FEA69064FEAE977079356EA07038A462C
:1007D80000F09280DDE90489BBF90E20DEF80440C0
:1007E800BBF910004946C4F5801ED317DDE9024560
:1007F80002FB01F108FB0311A2FB08230B444FEA9B
:1008080043492B46C11700FB03F304FB0133A0FB4C
:100818000401BBF90C401944E30001937346DC174B
:100828000023009349EAD2394FEA4248DDE9002320
:1008380010EB080041EB0901E50712184FEACE74E6
:100848004B4145EA5E05A41A65EB0305221945EB01
:10085800050312196B4199019001801841EA9261D0
:1008680059418B00820043EA9073101943EB05014C
:100878008B00820043EA90731046001919463246ED
:100888003B46694131F004FFBBF916204C13450B78
:1008980045EAC14502FB04F6D31705FB0366A2FB34
:1008A80005233344BBF9146002FB04F405FB03443D
:1008B80006FB01FEA2FB0523F717234400FB07EE06
:1008C800540EA6FB0067774444EAC3144FEAD6489F
:1008D80000194FEA636548EA473869414FEAE74932
:1008E80018EB0008BBF9124049EB01094FEA18263A
:1008F80046EA096620013618069B0BB1360A1E60C7
:10090800BAF1000F02D0079BCAF8003009B0BDE861
:10091800F08F00BF88890020E023002070477047CF
:100928004FF480538382704750F8043C012280F8CA
:100938004520103803B11847704770B5044682B097
:100948000830656A06236A463B21A847A8B19DF886
:1009580004009DF800609DF801109DF802509DF874
:1009680003209DF8053041EA062143EA002342EAC4
:100978000522E18222836383012002B070BD70B436
:100988000468037B2268022101FA03F31A4213D098
:1009980042690A49582000FB02124FF6FE76506859
:1009A8005289C5680068296831402960C168D24306
:1009B80092B20A40C260636070BC70476C7C0020D1
:1009C80030B4094B1C7864B1084B002503EBC40410
:1009D8001A6899885562D06808330143A342D160E8
:1009E800F6D130BC704700BF2C7F0020307F00203C
:1009F80010B40268047B11680223A340194209D08D
:100A08000649406800240C7001684FF6FE742140C6
:100A1800016053605DF8044B704700BF953F0020AC
:100A2800F0B4334C00EB800004EB80046468002CC5
:100A38005BD0304E49004FF42040CDB2B060A16980
:100A4800090444D460682C4F45F08071384041F463
:100A5800903101434FF420406160B06003E0411ED3
:100A6800002838D00846A1698F07F8D54FF42040F0
:100A7800A262B06002E0421E68B31046A269110685
:100A8800F9D562681C4945F0007545F480350A407F
:100A980015434FF420406560B06002E0421ED0B1BB
:100AA8001046A2699207F9D5A362A3694FF42040C2
:100AB8009B06B06005D4431E68B11846A3699B061F
:100AC800F9D52023B060E3610120F0BC7047411ED6
:100AD80008B10846B3E7094A138801339BB24FF0BF
:100AE800FF31B1601380F0BC70472046F0BC7047FE
:100AF800D06F0020E0230020009800FC4C2A002042
:100B0800134600200A4668218AE730B50446C06CBF
:100B180061710368A26823F00103036087B0A379B9
:100B2800009213F004023DD04FF4805213F00203F8
:100B3800019244D102934FF480630022039311F091
:100B48000103059237D1049308238D07694648BFEE
:100B5800049324F04DFA6079E36CA17900F0020265
:100B6800002A15BF4FF440324FF480324FF400345E
:100B7800002410F0010F586808BF2246CC074CBF6C
:100B8800024320EA02025A609A6809074CBF42F001
:100B9800080222F008029A601A6842F001021A60FC
:100BA80007B030BD13F0020301920BD04FF400558B
:100BB80013460295C1E7042304930C23C5E74FF4B9
:100BC8000053B7E70293B8E710B50446C06CA160BC
:100BD800036823F001030360A37986B013F00402CD
:100BE800009141D04FF4805213F00203019244D196
:100BF80002934FF4806362790393D1074FF00003A7
:100C08000493059345BF0423049308230C236946E2
:100C1800920748BF049324F0EBF96079E36CA1795B
:100C280000F00202002A15BF4FF440324FF4803220
:100C38004FF40034002410F0010F586808BF224612
:100C4800CC074CBF024320EA02025A609A6809079F
:100C58004CBF42F0080222F008029A601A6842F07B
:100C680001021A6006B010BD13F00203019207D00A
:100C78004FF4005113460291BDE74FF40053B7E714
:100C88000293B8E700230122036043600370837076
:100C98000271837170472DE9F341056906460F46D5
:100CA8007DBBD0F80080C8F30A0323B30023D6F82D
:100CB800008001932AF090FB042819D1214C236964
:100CC80043F001032361BBB2A8F800302AF084FB8B
:100CD80004282ED108F102030193019B3F0C1F80C9
:100CE8002AF07AFB2369042823F00103236125D025
:100CF8006FF0010505E02AF06FFB042805D04FF0DE
:100D0800FF35284602B0BDE8F0810E4C236943F058
:100D180002032361C4F81480236943F0400323616C
:100D28002AF05AFB2369042823F002032361BDD06B
:100D3800E5E7236923F001032361D9E73368043326
:100D48003360DEE700200240F8B504460D468E18F1
:100D58000027B54201D12069F8BDE368591CE1605C
:100D6800234415F8012B1A720429F2D1A1682046F0
:100D7800FFF791FFE7602061EBE72AF0FDBD70B552
:100D880082B00446694614302AF0A2FDB0B19DF83D
:100D980005009DF801609DF802109DF803509DF82C
:100DA80004209DF8063041EA062143EA002342EA7E
:100DB8000522A187E287A4F84030012002B070BD67
:100DC80010B490E80600047B40690223A3404B60FE
:100DD80013685DF8044B4FF6FE710B40136007F083
:100DE80059B903685B6A03B11847704703681B6AFF
:100DF80003B11847704703682DE9F041DF691FB157
:100E08003B46BDE8F0411847002A164611DD044666
:100E18000D460E4400E023689B682046984700284A
:100E2800F9D0236815F8011B1B6820469847AE4285
:100E3800F1D1BDE8F0810368DB68184703689B6857
:100E4800184703685B68184703681B681847014B15
:100E58001868F9E7C4920020054B53F8203033B1E5
:100E68001A689B88918A0B4218BF1B0493617047CC
:100E7800B072002003682DE9F04F03F13845644E45
:100E8800AD0A0124755D05F01F066D09022D04FAEF
:100E980006F400F0A280032D00F0A480012D52D0AA
:100EA8008088B0FA80F4C4F11F04A4B2E50803EB0B
:100EB800850504F007042E6AA4000F27A74026EA38
:100EC80007062E622E6A01F0030702FA04F47A1E5E
:100ED8003443012AC1F3810CC1F300182C62C1F319
:100EE800411135D9C60700F19780850700F1A38025
:100EF800440700F1B180020700F1BF80C60600F187
:100F0800CD80850600F1DB80440600F1E980020609
:100F180000F1F780C60500F10581850500F1138110
:100F2800440500F12181020500F12F81C60400F17A
:100F38003D81850400F14B81440400F1598102048C
:100F480055D4BDE8F08F334D6E6934436C61A7E723
:100F5800002422464FF0010E4FF0030904E001324D
:100F6800102A04F10204ECD00EFA02F636EA000563
:100F7800F5D1D3F808A009FA04F5ED430AEA050A01
:100F8800C3F808A0D3F808B00CFA04FA4AEA0B0A26
:100F9800C3F808A0B3F804A01FFA8AFA2AEA0606DA
:100FA8009E80B3F804A008FA02F646EA0A06B6B22A
:100FB8009E801E682E401E60D3F800A007FA04F633
:100FC80046EA0A061E60D3F80CA001FA04F605EA00
:100FD8000A0A46EA0A05DD60C1E70E4DAE693443E8
:100FE800AC615DE70B4DEE693443EC6158E71A6874
:100FF80022F040421A601A6842EA87771F60DA686E
:1010080022F0404242EA8171D960BDE8F08F00BF0A
:10101800487A0308001002401A6822F003021A6096
:101028001A683A431A60DA6822F003020A4385070D
:10103800DA607FF55DAF1A6822F00C021A601A6850
:1010480042EA87021A60DA6822F00C0242EA810258
:101058004407DA607FF54FAF1A6822F030021A6051
:101068001A6842EA07121A60DA6822F0300242EA85
:101078000112DA6002077FF541AF1A6822F0C00258
:101088001A601A6842EA87121A60DA6822F0C00207
:1010980042EA8112C606DA607FF533AF1A6822F495
:1010A80040721A601A6842EA07221A60DA6822F463
:1010B800407242EA01228506DA607FF525AF1A6898
:1010C80022F440621A601A6842EA87221A60DA68D3
:1010D80022F4406242EA81224406DA607FF517AFC3
:1010E8001A6822F440521A601A6842EA07321A60F3
:1010F800DA6822F4405242EA0132DA6002067FF5E9
:1011080009AF1A6822F440421A601A6842EA873224
:101118001A60DA6822F4404242EA8132C605DA608F
:101128007FF5FBAE1A6822F440321A601A6842EA68
:1011380007421A60DA6822F4403242EA0142850521
:10114800DA607FF5EDAE1A6822F440221A601A6858
:1011580042EA87421A60DA6822F4402242EA81426F
:101168004405DA607FF5DFAE1A6822F440121A608F
:101178001A6842EA07521A60DA6822F4401242EA10
:101188000152DA6002057FF5D1AE1A6822F44002F6
:101198001A601A6842EA87521A60DA6822F4400232
:1011A80042EA8152C604DA607FF5C3AE1A6822F0BB
:1011B80040721A601A6842EA07621A60DA6822F016
:1011C800407242EA01628504DA607FF5B5AE1A68BA
:1011D80022F040621A601A6842EA87621A60DA6886
:1011E80022F0406242EA81624404DA607FF5A7AEE9
:1011F8001A6822F040521A601A6842EA07721A60A6
:10120800DA6822F0405242EA0172DA6097E603682F
:1012180003F138422DE9F04F920A584DAA5C02F0CA
:101228001F0552090124022A04FA05F400F08C80F3
:10123800032A00F08E80012A3CD001F003077A1EB1
:10124800012AC1F3810CC1F300188088C1F3411150
:1012580035D9C60700F19680850700F1A2804407BA
:1012680000F1B080020700F1BE80C60600F1CC8014
:10127800850600F1DA80440600F1E880020600F1F4
:10128800F680C60500F10481850500F11281440548
:1012980000F12081020500F12E81C60400F13C8195
:1012A800850400F14A81440400F15881020455D4B0
:1012B800BDE8F08F324A55692C435461BDE70024DC
:1012C80022464FF0010E4FF0030904E00132102AC4
:1012D80004F10204ECD00EFA02F636EA0005F5D164
:1012E800D3F808A009FA04F5ED430AEA050AC3F899
:1012F80008A0D3F808B00CFA04FA4AEA0B0AC3F8B3
:1013080008A0B3F804A01FFA8AFA2AEA06069E8003
:10131800B3F804A008FA02F646EA0A06B6B29E80B6
:101328001E682E401E60D3F800A007FA04F646EAAD
:101338000A061E60D3F80CA001FA04F605EA0A0AA8
:1013480046EA0A05DD60C1E70D4A95692C439461B8
:1013580073E70B4AD5692C43D4616EE71A6822F00B
:1013680040421A601A6842EA87771F60DA6822F0FA
:10137800404242EA8171D960BDE8F08F487A03089B
:10138800001002401A6822F003021A601A683A43F1
:101398001A60DA6822F003020A438507DA607FF5EB
:1013A8005EAF1A6822F00C021A601A6842EA8702D5
:1013B8001A60DA6822F00C0242EA81024407DA6015
:1013C8007FF550AF1A6822F030021A601A6842EAB4
:1013D80007121A60DA6822F0300242EA0112DA6073
:1013E80002077FF542AF1A6822F0C0021A601A6835
:1013F80042EA87121A60DA6822F0C00242EA8112D1
:10140800C606DA607FF534AF1A6822F440721A60B3
:101418001A6842EA07221A60DA6822F4407242EA3D
:1014280001228506DA607FF526AF1A6822F4406249
:101438001A601A6842EA87221A60DA6822F440625F
:1014480042EA81224406DA607FF518AF1A6822F46E
:1014580040521A601A6842EA07321A60DA6822F4BF
:10146800405242EA0132DA6002067FF50AAF1A6892
:1014780022F440421A601A6842EA87321A60DA682F
:1014880022F4404242EA8132C605DA607FF5FCAEBA
:101498001A6822F440321A601A6842EA07421A604F
:1014A800DA6822F4403242EA01428505DA607FF5C3
:1014B800EEAE1A6822F440221A601A6842EA87429D
:1014C8001A60DA6822F4402242EA81424405DA606E
:1014D8007FF5E0AE1A6822F440121A601A6842EAF0
:1014E80007521A60DA6822F4401242EA0152DA60BE
:1014F80002057FF5D2AE1A6822F440021A601A6813
:1015080042EA87521A60DA6822F4400242EA8152BB
:10151800C604DA607FF5C4AE1A6822F040721A6019
:101528001A6842EA07621A60DA6822F0407242EAF0
:1015380001628504DA607FF5B6AE1A6822F040626F
:101548001A601A6842EA87621A60DA6822F0406212
:1015580042EA81624404DA607FF5A8AE1A6822F094
:1015680040521A601A6842EA07721A60DA6822F072
:10157800405242EA0172DA6098E610B50409013C6B
:10158800052C17D80C4B33F8142000F00F0042FA42
:1015980000F313F001030DD0012303FA00F0013822
:1015A800104031F0C5F8054A054B125D104403EBB5
:1015B800C00010BD002010BD0C7D0308187D030875
:1015C800547A00202DE9F04F4A484B4B4B4C4FF0D2
:1015D80090414FF0010A4FF002094FF004084FF014
:1015E800080C4FF0100E20274026802530F8022BDB
:1015F80012F0010F03D01960A3F804A0083312F009
:10160800020F03D01960A3F80490083312F0040FF6
:1016180003D01960A3F80480083312F0080F03D030
:101628001960A3F804C0083312F0100F03D0196032
:10163800A3F804E0083312F0200F02D019609F804D
:10164800083312F0400F02D019609E80083312F060
:10165800800F02D019609D80083312F4807F05D076
:101668004FF4807B1960A3F804B0083312F4007FAC
:1016780005D04FF4007B1960A3F804B0083312F4C6
:10168800806F05D04FF4806B1960A3F804B008335D
:1016980012F4006F05D04FF4006B1960A3F804B082
:1016A800083312F4805F05D04FF4805B1960A3F80B
:1016B80004B0083312F4005F05D04FF4005B1960E2
:1016C800A3F804B0083312F4804F05D04FF4804BD0
:1016D8001960A3F804B00833D20B04D04FF40042C9
:1016E80019609A80083301F58061A1427FF47EAFCA
:1016F800BDE8F08F0C7D0308547A002000180048DC
:10170800002867D003682DE9F04F03F138445C4E98
:10171800A40A0125345D04F01F066409022C05FAA9
:1017280006F558D0032C00F0A580012C58D08088ED
:10173800B0FA80F4C4F11F04A4B2E50803EB8505F0
:1017480004F007042E6AA4000F27A74026EA07061C
:101758002E622E6A01F00307A2407C1E3243012C40
:10176800C1F3810CC1F300182A62C1F341113CD9BD
:10177800C60700F18980850700F19580440700F1CC
:10178800A380020700F1B180C60600F1BF8085067C
:1017980000F1CD80440600F1DB80020600F1E9800B
:1017A800C60500F1F780850500F10581440500F1C3
:1017B8001381020500F12181C60400F12F818504FF
:1017C80000F13D81440400F14B81020400F159818C
:1017D800BDE8F08F70472B4CA6693543A561A6E795
:1017E800284C666935436561A1E7002422464FF01D
:1017F800010E4FF0030904E00132102A04F102043B
:10180800E6D00EFA02F636EA0005F5D1D3F808A0BC
:1018180009FA04F5ED430AEA050AC3F808A0D3F863
:1018280008B00CFA04FA4AEA0B0AC3F808A0B3F89D
:1018380004A01FFA8AFA2AEA06069E80B3F804A0D2
:1018480008FA02F646EA0A06B6B29E801E682E40DC
:101858001E60D3F800A007FA04F646EA0A061E60DE
:10186800D3F80CA001FA04F605EA0A0A46EA0A05C2
:10187800DD60C1E7034CE6693543E56157E700BF22
:10188800487A0308001002401A6822F003021A601E
:101898001A683A431A60DA6822F003020A43850795
:1018A800DA607FF56BAF1A6822F00C021A601A68CA
:1018B80042EA87021A60DA6822F00C0242EA8102E0
:1018C8004407DA607FF55DAF1A6822F030021A60CB
:1018D8001A6842EA07121A60DA6822F0300242EA0D
:1018E8000112DA6002077FF54FAF1A6822F0C002D2
:1018F8001A601A6842EA87121A60DA6822F0C0028F
:1019080042EA8112C606DA607FF541AF1A6822F40E
:1019180040721A601A6842EA07221A60DA6822F4EA
:10192800407242EA01228506DA607FF533AF1A6811
:1019380022F440621A601A6842EA87221A60DA685A
:1019480022F4406242EA81224406DA607FF525AF3C
:101958001A6822F440521A601A6842EA07321A607A
:10196800DA6822F4405242EA0132DA6002067FF570
:1019780017AF1A6822F440421A601A6842EA87329E
:101988001A60DA6822F4404242EA8132C605DA6017
:101998007FF509AF1A6822F440321A601A6842EAE1
:1019A80007421A60DA6822F4403242EA01428505A9
:1019B800DA607FF5FBAE1A6822F440221A601A68D2
:1019C80042EA87421A60DA6822F4402242EA8142F7
:1019D8004405DA607FF5EDAE1A6822F440121A6009
:1019E8001A6842EA07521A60DA6822F4401242EA98
:1019F8000152DA6002057FF5DFAE1A6822F4400270
:101A08001A601A6842EA87521A60DA6822F44002B9
:101A180042EA8152C604DA607FF5D1AE1A6822F034
:101A280040721A601A6842EA07621A60DA6822F09D
:101A3800407242EA01628504DA607FF5C3AE1A6833
:101A480022F040621A601A6842EA87621A60DA680D
:101A580022F0406242EA81624404DA607FF5B5AE62
:101A68001A6822F040521A601A6842EA07721A602D
:101A7800DA6822F0405242EA0172DA6002047FF525
:101A8800A7AE1A6822F040421A601A6842EA8777BD
:101A98001F60DA6822F0404242EA8171D960BDE8ED
:101AA800F08F002852D0036803F138422DE9F04F37
:101AB800920A514DAA5C02F01F0552090124022A1C
:101AC80004FA05F443D0032A00F09080012A43D099
:101AD80001F003077A1E012AC1F3810CC1F3001833
:101AE8008088C1F341113CD9C60700F18980850778
:101AF80000F19580440700F1A380020700F1B1804E
:101B0800C60600F1BF80850600F1CD80440600F1CD
:101B1800DB80020600F1E980C60500F1F780850543
:101B280000F10581440500F11381020500F12181CE
:101B3800C60400F12F81850400F13D81440400F1C1
:101B48004B81020400F15981BDE8F08F70472B4AA0
:101B580095692C439461BBE7284A55692C43546125
:101B6800B6E7002422464FF0010E4FF0030904E0C7
:101B78000132102A04F10204E6D00EFA02F636EA1F
:101B88000005F5D1D3F808A009FA04F5ED430AEAEF
:101B9800050AC3F808A0D3F808B00CFA04FA4AEA10
:101BA8000B0AC3F808A0B3F804A01FFA8AFA2AEAB5
:101BB80006069E80B3F804A008FA02F646EA0A066A
:101BC800B6B29E801E682E401E60D3F800A007FAA9
:101BD80004F646EA0A061E60D3F80CA001FA04F6D9
:101BE80005EA0A0A46EA0A05DD60C1E7034AD5693B
:101BF8002C43D4616CE700BF487A03080010024008
:101C08001A6822F003021A601A683A431A60DA68FE
:101C180022F003020A438507DA607FF56BAF1A6882
:101C280022F00C021A601A6842EA87021A60DA681F
:101C380022F00C0242EA81024407DA607FF55DAFC8
:101C48001A6822F030021A601A6842EA07121A600B
:101C5800DA6822F0300242EA0112DA6002077FF500
:101C68004FAF1A6822F0C0021A601A6842EA871257
:101C78001A60DA6822F0C00242EA8112C606DA6007
:101C88007FF541AF1A6822F440721A601A6842EA76
:101C980007221A60DA6822F4407242EA01228506B5
:101CA800DA607FF533AF1A6822F440621A601A6866
:101CB80042EA87221A60DA6822F4406242EA812204
:101CC8004406DA607FF525AF1A6822F440521A609C
:101CD8001A6842EA07321A60DA6822F4405242EA85
:101CE8000132DA6002067FF517AF1A6822F4404223
:101CF8001A601A6842EA87321A60DA6822F44042A7
:101D080042EA8132C605DA607FF509AF1A6822F423
:101D180040321A601A6842EA07421A60DA6822F406
:101D2800403242EA01428505DA607FF5FBAE1A6867
:101D380022F440221A601A6842EA87421A60DA6876
:101D480022F4402242EA81424405DA607FF5EDAE92
:101D58001A6822F440121A601A6842EA07521A6096
:101D6800DA6822F4401242EA0152DA6002057FF58D
:101D7800DFAE1A6822F440021A601A6842EA8752F3
:101D88001A60DA6822F4400242EA8152C604DA6034
:101D98007FF5D1AE1A6822F040721A601A6842EADA
:101DA80007621A60DA6822F0407242EA016285042A
:101DB800DA607FF5C3AE1A6822F040621A601A68CA
:101DC80042EA87621A60DA6822F0406242EA816277
:101DD8004404DA607FF5B5AE1A6822F040521A6002
:101DE8001A6842EA07721A60DA6822F0405242EA38
:101DF8000172DA6002047FF5A7AE1A6822F0404249
:101E08001A601A6842EA87771F60DA6822F040424F
:101E180042EA8171D960BDE8F08FF0B5044690F8C8
:101E2800590083B0002840F0A480684E377B002F0B
:101E380040D004F11405A06925F080F894F85220E8
:101E48001A212846FEF77AFA012005F02BFFA0692F
:101E580025F062F828460623E56D6A464321A8471F
:101E6800D8B19DF802609DF803309DF800509DF8A8
:101E780001109DF804009DF8052043EA06231BB2D3
:101E8800E3875BB241EA052142EA00220133A187D8
:101E9800A4F8402006D003B0F0BDB4F93E305BB2E0
:101EA8000133F8D194F93C300133F4D1062005F020
:101EB8009BFAF0E704F11405A06925F03FF88022A9
:101EC8006B212846FEF73AFA962005F045FF0322D3
:101ED80068212846FEF732FA962005F03DFF0322D6
:101EE8006B212846FEF72AFA0F2005F0DBFE1022A8
:101EF8006A212846FEF722FA0F2005F0D3FE3A465B
:101F08006C212846FEF71AFA0F2005F0CBFE94F84C
:101F1800542019212846FEF711FA0F2005F0C2FEB9
:101F280018221B212846FEF709FA0F2005F0BAFEF1
:101F380010221C212846FEF701FA0F2005F0B2FEF8
:101F4800102237212846FEF7F9F90F2005F0AAFEDE
:101F5800012238212846FEF7F1F90F2005F0A2FEEC
:101F6800A06924F0D9FF012005F09CFE01233373FA
:101F780061E7FFF702FB0546D8B1202300218371F2
:101F8800C171FFF78EFD2146114B41F8103F2846DD
:101F980029F03EFCAB88B3FA83F3C3F11F035A1C44
:101FA8003FF443AF01229A400A490B6813430B6080
:101FB8003BE70146FFF775FD2146054B41F8103F09
:101FC800284629F025FC0122EEE700BFE023002087
:101FD800310900080004014010B1036882881A859D
:101FE800704710B1036882889A61704738B1002938
:101FF8008388026814BF002110218B4093617047C9
:1020080010B40A4B0A4A1C7801238340234052F833
:10201800200029B9B3FA83F149095DF8044BE5E7D3
:10202800191C18BF01215DF8044BDFE7AC720020D2
:10203800B072002030B1036882881B8A1A4214BF2C
:102048000120002070472DE9F0410B4E3468736978
:102058001C400FD0DFF824800127B4FA84F3C3F1C1
:102068001F0307FA03F558F8230003689847AC43A1
:102078007561F2D1BDE8F081000401409C81002027
:102088002DE9F0410B4E346873691C400FD0DFF81E
:1020980028800127B4FA84F3C3F11F0307FA03F574
:1020A80058F8230003689847AC437561F2D1BDE83E
:1020B800F08100BF000401409C8100202DE9F0411F
:1020C8000B4E346873691C400FD0DFF82880012755
:1020D800B4FA84F3C3F11F0307FA03F558F8230091
:1020E80003689847AC437561F2D1BDE8F08100BF41
:1020F800000401409C8100202DE9F0410B4E34681A
:1021080073691C400FD0DFF828800127B4FA84F3E4
:10211800C3F11F0307FA03F558F82300036898472B
:10212800AC437561F2D1BDE8F08100BF0004014005
:102138009C8100202DE9F0410B4E346873691C40E6
:102148000FD0DFF828800127B4FA84F3C3F11F0306
:1021580007FA03F558F8230003689847AC437561FC
:10216800F2D1BDE8F08100BF000401409C8100204D
:102178002DE9F0410B4E346873691C400FD0DFF82D
:1021880028800127B4FA84F3C3F11F0307FA03F583
:1021980058F8230003689847AC437561F2D1BDE84D
:1021A800F08100BF000401409C8100202DE9F0412E
:1021B8000B4E346873691C400FD0DFF82880012764
:1021C800B4FA84F3C3F11F0307FA03F558F82300A0
:1021D80003689847AC437561F2D1BDE8F08100BF50
:1021E800000401409C810020084A094808B5936909
:1021F80043F0010393610021402233F04AF8054B74
:102208004FF0FF321A60C3F8032008BD00100240E7
:102218009C810020DC8100202DE9F041044618460D
:102228000D46164698462FF069FD2768E672284441
:10223800A07229467D69434632462046AC46BDE831
:10224800F0416047036810B504461B689847236847
:1022580020469B689847A37B0133A37310BD10B534
:10226800036804469B689847FF230122637322731F
:1022780010BD08B52120FFF780F90C4B186018B184
:10228800112200238271C3712021FFF70AFC20204C
:10229800FFF773F9064B186018B1112200238271F9
:1022A800C3712021BDE80840FFF7FBBBD83A0020E6
:1022B800DC3A002008B5FFF760F940B12C228271A2
:1022C8000022C2712021BDE80840FFF7EABB08BD23
:1022D800F8B505015A4C5B4B625961199A4204EBF7
:1022E800050704BF01230B730646387A24F0C0F9AA
:1022F8003B7A03F01F015B090122022B02FA01F26B
:1023080078D0032B71D0012B67D063190136187967
:10231800FFF733F9F6B2074610B11223C67183717D
:1023280063195879FFF729F910B11323C67183711E
:1023380063199879FFF721F910B11423C6718371D5
:1023480066190E21F2793846FFF7DAF97079FFF746
:1023580014F9F2790E21FFF7D3F9B079FFF70DF9E7
:10236800F2790E21FFF7CCF96359374A934251D0DD
:10237800344A934259D0354A934240D02C44227B68
:10238800002A2FD1012002249A8822F480521204B4
:10239800120C9A80998889B241F4805199801A88E0
:1023A80002F4415242F44572024322431A809A8849
:1023B80022F470621204120C42F4E0629A809A8B42
:1023C80022F400621204120C07219A8319821A88D7
:1023D80092B242F040021A80F8BD1D4B996A0A4336
:1023E8009A6292E700200446CEE7194B19690A431E
:1023F8001A618AE7164BD9680A43DA6085E702F55D
:10240800EA32116941F400411161116921F4004176
:102418001161B3E702F56042D16841F48051D1609F
:10242800D16821F48051D160A8E702F5EC32116936
:1024380041F480411161116921F4804111619DE7E6
:10244800F86F00200038004000300140003C004098
:1024580000100240427A02B9704710B5044603687A
:10246800406804F10A0198470023637210BD437A5B
:102478005A1C0344D2B242729972037A934200D82A
:1024880002B9704710B504460368406804F10A01B0
:1024980098470023637210BD30B40B4D002305F13B
:1024A800140101E0272B0BD011F8132082424FEAC8
:1024B800430403F10103F5D12C44607D30BC70471F
:1024C800002030BC704700BF0454030870B544882E
:1024D80006460D46C4F30B0422460021284632F076
:1024E800D8FE3369094A934209D3094A934206D26E
:1024F800224628461946BDE8704030F0B3BB23B1E8
:1025080021462846BDE87040184770BD78C30308C7
:102518006DC40308064B07498B4202D300231846B3
:1025280070471A88C2F30B029042F8D01433F3E7CD
:10253800C8BE030878C30308024A136823EA0000E8
:1025480010607047D43C0020F8B5174D2B78A32BAA
:1025580028D16B78BE2B25D1022229464FF6FF7071
:10256800FEF7ACF8114FAC1C22884AB1A618BE423F
:1025780018D2052A16D92146FEF7A0F83446F3E703
:1025880021460222FEF79AF80222A118FEF796F8D1
:102598000634074B641B1C8041F60F53C31A58427C
:1025A8005841F8BD0020F8BD00F0030800000408F9
:1025B8004E2A00202DE9F04FDFF848914C4F8BB0A0
:1025C8000326A7EB09071822002104A832F061FEB0
:1025D800484BCDF8109005971A69120604D5464A5B
:1025E8005A6002F188325A6001228DF82420342280
:1025F800DA60424B424C1B88ADF800300222694633
:1026080004A8FEF7A1FB022269464FF6FF70FEF709
:1026180055F8DFF8F4A080464FF0000B544536D348
:102628000AAC002524F8245D0222214604A8FEF7FE
:102638008BFB022221464046FEF740F840BAC043D1
:10264800ADF80800022202A904A8FEF77DFB07984E
:1026580060B106ABC0F104022946184432F019FEF5
:10266800069904A8FEF717FB079508909DF82430F3
:10267800089A23B11F490B6943F080030B61013E9F
:102688002DD0002A9FD1FFF75FFF50B32CE065885B
:102698008DF80DB0C5F30B05AB1DADF808302388D8
:1026A800C3F30B02ADF80A201B0B062202A904A8EB
:1026B8008DF80C30FEF748FB062202A94046FDF7CC
:1026C800FDFF616880462A4604A8FEF73DFB616865
:1026D80040462A46FDF7F2FF143480469EE7002A5A
:1026E800D1D0052004F080FE0BB0BDE8F08F00BF0C
:1026F80000000408002002402301674566540308CF
:10270800C8BE030800F0030878C303080378202B29
:10271800024600F10100F9D0092BF7D02D2B2CD05F
:102728002B2B03BF5378B7EE000A0246B7EE000A18
:10273800A3F13001C8B209289FED467A10D8F2EE0D
:10274800046A07EE901AF8EEE77A12F8013FE7EE0E
:10275800267AA3F13001C8B20928B0EE677AF0D919
:102768002E2B4CD003F0DF03452B0BD0F7EE007A6D
:1027780067EE276A20EE260A70475378BFEE000AF4
:102788000246D5E710B451782D2959D02B290ABF14
:102798009178501C901C0024A1F13003092B53D8C8
:1027A800002303EB830301EB430310F8011FA1F19E
:1027B8003002092AA3F13003F3D9B3F59A7F28BF71
:1027C8004FF49A73072B42D9DFED236A1A46F7EEC6
:1027D800007A083A072A67EEA67AFAD803F00703C0
:1027E8002BB1F2EE046A013B67EEA67AFBD124B363
:1027F800C7EE276A5DF8044B20EE260A7047537827
:10280800A3F13001C8B2092802F10102AAD8F2EEF8
:10281800046AF0EE665A07EE901AF8EEE77A12F8B4
:10282800013F87EEA66AA3F13001C8B2092866EE17
:10283800A56A37EE067AEED994E767EE276AD9E7F4
:10284800901C91780124A7E7F7EE007ACFE7F7EE1E
:10285800007AC5E70000000020BCBE4CB5EEC00AF7
:10286800DFED317AF1EE10FACCBF30EE270A30EE08
:10287800670ADFED2E7A20EE270A30B5FDEEC07A22
:1028880087B017EE904A054684EAE470002303A94E
:10289800A0EBE47001930093029323F003F9002C5A
:1028A800ACBF20232D2303A88DF800302FF026FA83
:1028B800012803A924D002282DD0032805BF3023DE
:1028C800684668468DF8013032F009FD68462FF0F9
:1028D80015FA0338C4B222466946284632F05DFD2F
:1028E80000232B5528462FF009FA2E22431C2A5480
:1028F8000DEB0401E81832F00FFD284607B030BD93
:10290800302368468DF801308DF802308DF8033099
:1029180032F0E5FCDAE7302368468DF801308DF8AF
:10292800023032F0DCFCD1E76F12033A00007A443F
:102938002DE9F041064615460846B6FBF2F43CB9C7
:1029480005FB1464124B1B5D00F8013BBDE8F081E8
:10295800B4FBF2F767B90E4B05FB174705FB146488
:10296800DA5D00F8012B1B5D00F8013BBDE8F08142
:10297800B7FBF2F8B8F1000F02D04046FFF7D8FFD6
:1029880005FB1878024B13F8082000F8012BE3E741
:102998006C81030830B402681146531C036011F8B7
:1029A800024B0160D31C517803609378151D0560B4
:1029B8001B0443EA0123D078234343EA006030BC78
:1029C80070470368591C1A46016012F8021B02601E
:1029D800587841EA0020704703685A1C026018784A
:1029E800704738B504460068154630F03BF9226850
:1029F8002A44226038BD036810B40A0A5C1C0460CB
:102A08001A7003685A1C026019705DF8044B70470D
:102A180003685A1C026010B4197003680A0A5C1C27
:102A280004601A7003680A0C5C1C04601A7003685E
:102A3800090E5A1C026019705DF8044B7047036850
:102A48005A1C026019700368090A5A1C026019703E
:102A580070472DE9F047002488B080460F461E468F
:102A6800A14605AD531C0393117839B3252933D1F9
:102A7800931CCDF810900393507830284ED04FF027
:102A8800000AA0F13003DBB2092B42D96C2819D017
:102A9800642800F0938024D825281CD063D95828AE
:102AA80076D063281BD131784046B847039A531C27
:102AB80003931178043601340029D7D1204608B091
:102AC800BDE8F087039B5A1C03921B78642B7CD0CB
:102AD8002AD8252B54D1252140460134B847039ADA
:102AE800C0E7732833D044D975284FD106F1040EB6
:102AF80030682B4600220A217646FDF7DBFC049A53
:102B08000095534639464046FDF711FD039A0444A3
:102B1800A8E704AA03A929F0AFFBB7E7D31C0393DE
:102B280090784FF0010AACE7732B10D05BD9752B66
:102B38003AD0782B96D1A3F15802B2FA82F23068D3
:102B480052092B4610210436FDF7B4FCD7E7336849
:102B5800049A0093394600234046FDF7E8FC043602
:102B68000444039A7EE70028B9D1204608B0BDE89E
:102B7800F0876E28B3D1039A336804361C6071E776
:102B88002AD9582BD7D0632B8DD06BE77828A6D1BC
:102B9800A0F15802B2FA82F2306852092B4610218D
:102BA800FDF788FC0436AAE706F1040E30682B46C8
:102BB80000220A217646FDF77DFCA0E7331D306828
:102BC80029461E46FDF748FC99E7331D306829461B
:102BD8001E46FDF741FC92E7002B7FF443AF2046E9
:102BE80008B0BDE8F0876E2BC6D03BE70EB400B541
:102BF80084B005AB019053F8042B0649039301A850
:102C0800FFF727FF019B00221A7004B05DF804EB60
:102C180003B070472D0500080FB430B583B006AB7C
:102C28000B490C4853F8042B096800680193FFF717
:102C380010FF094C0546206803685B69984700281F
:102C4800F9D0284603B0BDE8304004B0704700BF53
:102C5800CC3A0020D03A0020C4920020DFED2B7A35
:102C6800B4EEE70AF1EE10FA4ADDDFED296A9FEDCE
:102C7800297A01E0B0EE670AB4EEC70AF1EE10FA5D
:102C880070EE667AF6DC9FED247AF4EEC77AF1EE00
:102C980010FA38D5DFED1E6A9FED207A01E0F0EEDC
:102CA800407AF4EEC77AF1EE10FA37EEA60AF6D4B7
:102CB800DFED1B7AB4EEE70AF1EE10FA14DDDFED72
:102CC800137A37EEC00A60EE006A9FED166A9FED30
:102CD800167ADFED167AA6EE867A20EE266AE6EEFA
:102CE800877AA6EE270A7047DFED117AB4EEE70A75
:102CF800F1EE10FA44BFDFED087A37EEC00AE2E7DA
:102D0800F0EE407ABFE7B0EE670AD1E7DB0F494043
:102D1800DB0FC940E4CB1641DB0F49C0E4CB16C139
:102D2800DB0FC93F92E741B99730083C15A82ABE86
:102D3800DB0FC9BF80EAE073A3EBE0738B4205DBCE
:102D4800002801DD401A704702D170470020704703
:102D58000844704709B909E0194690FBF1F301FBF3
:102D680013030846002BF7D1084670470146FBE7D6
:102D780010B507EE901A2DED028BB8EE678ADFEDDD
:102D8800217A28EE008A044628EE278AB0EE480AFF
:102D980030F0BEF9F0EE408AB0EE480A30F01AF989
:102DA800F7EE007A9FED187AF0EE675AE8EE875A48
:102DB8000023A361B0EE676AC7EEA56A6361236268
:102DC800E361A8EEC76ABDEC028B77EEC07AB6EE77
:102DD800007AF8EE005A27EE877A20EE250A27EEC9
:102DE800267A26EE266A67EEA67A20EE260A84ED73
:102DF800046AC4ED017A84ED007A84ED027A84EDE8
:102E0800030A10BD27D4D236F304353F10B44C0959
:102E1800012250F8243001F01F0102FA01F10B439E
:102E280040F824305DF8044B70474B0901F01F014E
:102E380050F82320012303FA01F1114214BF184668
:102E4800002070472DE9F84FDFF8B490DFF8B48020
:102E5800DFF8B4A0274E0123042089F8003024F0BD
:102E680081F8D8F80000FFF7B7F8052023F0A4FF91
:102E7800002023F0A1FF062023F09EFF002023F06E
:102E88009BFF9AF80040042044F0010423F094FFCB
:102E9800204623F091FF33888BB1174D174F00243C
:102EA80015F804B0072023F087FF584623F084FF65
:102EB8002A5D33883A550134A4B2A342F0D80720DA
:102EC80023F07AFFFF2023F077FF9AF800400420D0
:102ED80023F072FF204623F06FFFD8F80000FFF7B9
:102EE80080F8022024F03EF8002389F80030BDE87D
:102EF800F88F00BF721900201C41002050430020A9
:102F08003B43002034860020414300202DE9F04156
:102F18004A4E042024F026F83068FFF75DF8484B45
:102F28001B78012B7BD062D3022B0AD1DFF83081CA
:102F3800082388F800300D254FF4C373414F3B80B8
:102F480010E0DFF81C813F4F98F8003003F0400391
:102F5800002B14BF4FF4F0734FF4C3733B8014BFBE
:102F680010250D25002404F11000C0B223F024FF21
:102F78000134012023F020FFA3B2AB42F3D398F829
:102F88000040314D002023F017FF204623F014FFA6
:102F98002E4B1C78022023F00FFF204623F00CFF55
:102FA8002B4B1C78032023F007FF204623F004FF57
:102FB800284B1C780420044323F0FEFE204623F00F
:102FC800FBFE3068FFF70DF8022023F0CBFF3A88AC
:102FD8002148002132F05DF92B7833B11F4B1B7863
:102FE80033B300232B70BDE8F081BDE8F081A02049
:102FF80023F0E2FE002023F0DFFE00F00603022BA0
:10300800DFF85C8007D000F00500012803D14823D1
:1030180088F8003008E0082388F800308BE7DFF8EC
:103028004080482388F8003010254FF4F07385E776
:10303800FFF708FF00232B70BDE8F08134860020DD
:103048003886002072190020000000203F860020EA
:103058004086002041430020504300203B4300208D
:1030680074190020B0F1FF3F0AD0022810B403DC25
:103078005DF8044BFDF7D4BC00205DF8044B7047A5
:1030880000207047F0B55B4B5B4A97B019689142D6
:1030980000AF00F0A3805949594A00234FF470004B
:1030A800C1F888003B607B60136843F48033136089
:1030B80003E03B68B3F5A04F09D0136803F400336D
:1030C8007B603B6801333B607B68002BF1D04C4B45
:1030D8001B6813F4003318BF01237B607B68012B46
:1030E80052D0464C464B474AE260474A596A1160FB
:1030F8005A6A42F080725A625A6942F4FC025A6172
:103108000025032207F10801012341F6FF764FF05D
:103118009040FD60BE603A73BB7321F0C5FF4FF667
:10312800FF7307F108013948BB6021F0BDFF07F1C3
:1031380008013748374E21F0B7FF07F10801364834
:1031480021F0B2FF07F10801344821F0ADFF07F183
:103158000801334821F0A8FF07F1080021F05AFDC3
:10316800BB683049304AA1FB031330499B0CF0205F
:103178004FF0070E5C370B60566084F823009560AB
:10318800C2F800E0BD46F0BD294A1D4B122111606E
:103198005A685A605A685A605A6842F480625A609B
:1031A8005A6822F47C125A605A6842F4E8125A604B
:1031B8001A6842F080721A601A689201FCD5596840
:1031C8000F4A21F003015960596841F00201596022
:1031D800536803F00C03082BFAD182E700221A6027
:1031E80062B6144B1B6883F30888134B1B68984717
:1031F800FEE700BFFC9F0020EFBEADDE00ED00E063
:10320800001002400005FA05805000200004004824
:10321800000800483F190100000C00480010004851
:103228000014004883DE1B4310E000E0E872002031
:103238000020024000D8FF1F04D8FF1F70B50F4CB4
:103248000F4DC0EBC00004EB800468692669304369
:10325800686182B09209667BA1600025012101A8FE
:1032680063618DF804608DF805208DF806508DF89F
:10327800071021F0EBFB02B070BD00BF202000203A
:1032880000100240074BC0EBC00030B403EB8000D5
:10329800054C056963692B4363610176427630BC4E
:1032A800704700BF20200020001002402DE9F04F99
:1032B8005E4C54F8204083B0002C71D0666D98465F
:1032C80091465B4B7268E264A160236004F15A0185
:1032D8004FF4807304F5AD726161A261E36023610C
:1032E8000746307E23F0C4F9F068A8B1514B00219D
:1032F8005A68904203F11C0300F0928001310C29B6
:10330800F6D100207A1CD2B20C21FFF7BBFFE36C88
:10331800F26822632433A364B068D8B1454B002116
:103328005A68904203F11C0378D001310C29F7D177
:1033380000257A1CD2B20B212846FFF7A3FF2346AB
:10334800F27E3D492846FFF779FFE36CB268626375
:103358002833636494F85900FEF70FF9054694F88A
:103368005800FEF70AF918F0080F824696F819B0C7
:103378001AD0CDB118F0110F4FF00B0307F1010768
:1033880014BF4E213E21EF715A46AB712846FEF715
:10339800B7F918F0010F45D0236B5BB3636B4BB3E0
:1033A800204603B0BDE8F08F18F0010F0CBF4FF0B6
:1033B8002E084FF04E0819F0020F09D045B10B2224
:1033C8007B1CAA71EB7128465A464146FEF798F9CC
:1033D80019F0010FE0D0BAF1000FDDD001370C234E
:1033E8008AF807705A4641468AF806305046FEF772
:1033F80087F9D1E7337FB27E8DF804209B0900213D
:10340800012201A88DF805308DF806108DF80720E7
:1034180021F01CFB204603B0BDE8F08FCDB288E751
:10342800C8B26FE72846FEF7D7FDB5E7E03A0020B7
:103438006854030820200020C90D00080348D0F86C
:103448003C3113B100F59A701847704720200020CE
:103458000348D0F8203113B100F58C701847704735
:10346800202000200348D0F804310BB1FC30184765
:10347800704700BF202000200348D0F8E8300BB187
:10348800E0301847704700BF202000200348D0F8DC
:10349800CC300BB1C4301847704700BF2020002043
:1034A8000348D0F8B0300BB1A8301847704700BFB8
:1034B800202000200348D0F894300BB18C301847F6
:1034C800704700BF202000200248836F0BB1703086
:1034D80018477047202000200248C36D0BB15430B4
:1034E80018477047202000200248036C0BB1383081
:1034F80018477047202000200248436A0BB11C304F
:1035080018477047202000200248836803B11847F5
:10351800704700BF20200020F0B53E4C059D00EB11
:10352800800004EB80046468002C71D03A4E490096
:103538004FF42040CFB2B060A169090454D4606848
:10354800DFF8E0E047F4903100EA0E0001434FF461
:1035580020406160B06003E0411E002848D0084662
:10356800A1698907F8D54FF42040A262B06003E052
:10357800421E00283CD01046A2695206F8D5274AB8
:103588006168DFF8A0E0B06042EA0342174301EA4D
:103598000E0217436760C3B1013BDBB201332B4412
:1035A800A0694FF4204210F0040002F1FF3207D165
:1035B800511C26D0A06910F0040002F1FF32F7D0A8
:1035C800626A05F8012B9D42EAD14FF42040B060B1
:1035D80002E0431E60B11846A3699B06F9D5202373
:1035E800B060E3610120F0BD411E08B10846A3E7C1
:1035F8000B4A138801339BB24FF0FF311380B1603F
:10360800F0BD0749B2600B8801339BB20B80F0BD57
:103618002046F0BDD06F0020E023002000240002E7
:103628004C2A0020009800FC70B50578012D82B066
:103638001E460DD0022D02D0002002B070BD1346E8
:1036480041F08001324602B0BDE87040FCF7E4BDAD
:10365800044690F90400431CEED00228ECDC134623
:103668000A4661790096FFF757FF02B070BD70B542
:1036780082B06B460622F721FFF7D6FF9DF801209E
:103688009DF804309DF800609DF803509DF80240B5
:103698009DF80500074912011B0142EA063243EA78
:1036A800053342EA141243EA10134A600B6002B071
:1036B80070BD00BFE0230020F0B585B002AB044622
:1036C8000093032206231E210020FFF725FF002870
:1036D8003CD09DF808509DF809109DF80A709DF897
:1036E8000B209DF80C609DF80D3041EA052142EA57
:1036F800072243EA062309B212B21BB2144D06EEA2
:10370800901A07EE102A07EE903AF8EEE66A95ED61
:10371800015AD5ED035A95ED026AB8EEC77AF8EE6C
:10372800E77A66EE856A27EE257A67EE867AFDEEF9
:10373800E66ABDEEC77AFDEEE77A16EE901A17EE46
:10374800102A17EE903A2180A280638005B0F0BD60
:10375800000000202DE9F043322083B004F0FCFA89
:103768000022104611231E21FFF77CFC6023012252
:103778001E210020FFF776FC642004F0EDFA68466D
:10378800FFF79AFF0024DFF85481254626460A27CA
:10379800012302221E210020FFF764FC322004F0DE
:1037A800DBFA6846FFF788FFBDF902E0BDF90410AF
:1037B800BDF900208E457346A8BF0B469342A8BFAB
:1037C800134643454FF0010075440C44164479DB19
:1037D800FDF742FB013FDBD14FF001090022104603
:1037E80012231E21FFF73EFCDFF8F0800A27012391
:1037F80002221E210020FFF735FC322004F0ACFA2B
:103808006846FFF759FFBDF902E0BDF90410BDF99C
:1038180000208E457346A8BF0B469342A8BF1346A7
:1038280043454FF00100A5EB0E05A4EB0104A6EB00
:1038380002064ADBFDF710FB013FD8D107EE906A7C
:10384800F8EEE76A07EE905AB8EEE77A07EE904A84
:10385800DFED1F5A9FED1F5A1F4EF8EEE77A85EEEF
:10386800A66A0022104670231E21C5EE876A85EEDF
:10387800277AB0EEC66AF0EEE66AF0EEC77A86ED11
:10388800016AC6ED026AC6ED037AFFF7EBFB202357
:1038980001221E210020FFF7E5FB00231846022223
:1038A8001E21FFF7DFFB642004F056FAB9F1000F80
:1038B80004D14FF07E537360B360F360012003B00E
:1038C800BDE8F0834FF0000988E74FF00009B5E73D
:1038D80000406F4601C05E460000002001F0FFFF77
:1038E80000B583B0002000920A466821FFF714FE55
:1038F80003B05DF804FB1749174B184A184810B471
:10390800D1F8884044F47004C1F888401C6844F039
:1039180001041C605C6822405A601A6822F08472B4
:1039280022F480321A601A6822F480221A605A68D7
:1039380022F4FE025A60DA6A22F00F02DA621A6B87
:10394800002410404FF0006218639C608A605DF8A4
:10395800044B704700ED00E0001002400CC07FF8F7
:10396800CCFC00FF2DE9F04F05462DED028BB0F998
:10397800080008815FFA80F897B040460C469146E7
:1039880002F0E6FC40B101231A461846628117B0DE
:10399800BDEC028BBDE8F08FA8F10A03E72B00F21B
:1039A800EA80DFE813F0B206E800E800E800E80083
:1039B800E800E800E800E800E800E800E800E800BF
:1039C800E800E800E800E800E800E800E800E800AF
:1039D800E800E800E800C506E800E800E800E406BA
:1039E800E800E800E800DC05E800E105E800220658
:1039F800E8003B06E8004706E8004C06E8007206C7
:103A0800E800E800E800B601BD01E800C501E800EB
:103A1800E800D301E800DB01E800E800E800A901BC
:103A2800E800E800E800E8000402E8001F02E800F7
:103A38005F028502E800E800E800E800E800E80026
:103A4800E800A902E800EC02E8001903E8004903CD
:103A5800E8009E03E800E800E800E800AE03ED0394
:103A6800280431047B04E800E80062048D04E800BF
:103A78009B04D404E800E800E800E800F104E8004A
:103A8800E800FD04E800E800E8001F0530054905E6
:103A98008D05E800E800E800CB05E80041071307BA
:103AA800E800E800E800E800E800E800E800E800CE
:103AB800E800E800E800E800E800E800E800AE03F5
:103AC800E800E800E800E800E800E800E800E800AE
:103AD800E800E800E800E800E800E800E800E8009E
:103AE800E800E800E800E800E800E800E800E8008E
:103AF800E800E800E800E800E800E800E800E8007E
:103B0800E800E800E800E800E800E800E800E8006D
:103B1800E800E800E800E800E800E800E800E8005D
:103B2800E800E800E800E800E800E800E800E8004D
:103B3800E800E800E800E800E800E800E800E8003D
:103B4800E800E800E800E800E800E800E800E8002D
:103B5800E800E800E800E800E800E800E800E8001D
:103B6800E800E800E800E800E800E800E800E8000D
:103B7800E80034078706B8F1740F54D0B8F1770F0E
:103B88000DD12B686A689A421EBF5A1C2A601978A0
:103B9800A54A08BF002120462DF070FDF3E6B8F1D4
:103BA800F50F4ED069682E68A8F121038A1B362BC1
:103BB80000F26887DFE813F01607660766076607EE
:103BC80066076607660766073607660766076607B5
:103BD8006607660766076607660766076607660775
:103BE8006607660766076607CF06660766076607FD
:103BF8006607660766076607660766076607660755
:103C08006607660766076607660766076607660744
:103C1800660766076607660766076607E0066607BB
:103C2800AD06660749062B686A689A421EBF5A1C89
:103C38002A6019787D4A08BF002120462DF01EFD14
:103C4800A1E62B686A689A4241F04B87784BFF22BD
:103C58001A704FF00008774D17F068F94146202296
:103C6800754885F8008031F014FB8DF818809DF8B0
:103C78001830072B02F26080704F6F4E42469DF855
:103C8800183003EB430307EBC3035B7CE3B19DF8F8
:103C9800183003EB430307EBC30320215B699BB197
:103CA8009DF8183003EB430307EBC303586946F844
:103CB8002200FDF7F6FE2B7856F82300FEF791F95F
:103CC8002A780132D2B22A709DF818300133DBB25B
:103CD8008DF818309DF81830072BD0D92368591C57
:103CE80021601A70B9F1000F3FF44DAE544BC9F87A
:103CF800003001231A4648E6236800255A1C226032
:103D0800294620461D70FEF783FE29462046FEF709
:103D18007FFE00212046FEF77BFE01231A4634E68B
:103D2800216801200A1822600346024608702CE622
:103D3800444B22689978501C20601170216858788B
:103D48004A1C012322601A4608701EE608223E49D2
:103D58002046FEF746FE01231A4616E623683B4A2C
:103D68003B4D11783B4A581C206019701168204659
:103D7800FEF74EFE2368344A591C127A21601A70E5
:103D880029882046FEF75BFEA9882046FEF757FEE5
:103D980029892046FEF753FE00212046FEF74FFEF4
:103DA80000212046FEF74BFE01231A46EDE5236865
:103DB800294D591C2A7921601A7023686A79591C7F
:103DC80021601A7029882046FEF739FE2368AA79EF
:103DD800591C21601A7069882046FEF730FE216858
:103DE800E879ADE71D4E3378002B3FF4CCAD1C4D80
:103DF8000027A846236815F81720591C21601A7057
:103E080098F8011001EB810101EB810101F2EE212B
:103E180089B22046FEF713FE337801379F4208F136
:103E28000208E7DBAFE500BFBD0B03082D1503084B
:103E3800202400203B8E00203C8D0020847B002025
:103E480039FB02083029002054500020088900203E
:103E58000C3B0020D43C00208C3200204C48002031
:103E6800088E00202368AE4D01269A1922601E7024
:103E780020F02CFC002841F02B86AA4B2268511C0C
:103E880021601070226841F2B410511C185C216046
:103E980041F27811107059582046890AFEF7B8FD8A
:103EA800A96A20464908FEF7B3FD01231A466CE5C6
:103EB80023689D4E01255A1C22601D702368B27824
:103EC800591921601A7028F079FC2368974A984993
:103ED8005F1927601870B1F90010B2F90000FEF7F9
:103EE80039FF23685A192260187031882046FEF776
:103EF800A6FD2B462A4648E51CF06EF9FF28064623
:103F080001F0438616A9002501F84A5D0DF10D0060
:103F18008DF80D501CF040F916A800F8495D1CF00A
:103F28002FF916A800F8485D1CF01EF916A820F80D
:103F3800405D1CF00DF923685A1C22601E7023682E
:103F48009DF80D20591C21601A7023689DF80E20D9
:103F5800591C21601A7023689DF80F20591C216094
:103F68001A7023689DF81020591C21601A70BDF83A
:103F780018102046FEF763FD01231A4605E5DFF811
:103F8800B88198F80330002B01F094852368082243
:103F9800591C21601A7023680122991821601A702F
:103FA8002368644D591C2A7921601A702368AA78FD
:103FB800591C21601A7029882046FEF740FDE989BE
:103FC8002046FEF73CFD236898F80720591C21601D
:103FD8001A702168E878B3E6574E23687279574D0E
:103FE800591C21601A702B682046198CFEF727FD92
:103FF8002B682046D98BFEF722FD71892046FEF7F3
:104008001EFDB1892046FEF71AFD2B682046598C03
:10401800FEF715FD2B682046998CFEF710FDF189F7
:104028002046FEF70CFD318A2046FEF708FD2B6876
:10403800216893F8260083E600212046FEF7FFFC5E
:1040480000212046FEF7FBFC00212046FEF7F7FC86
:1040580023683A4D00265A1C22601E7023682A687D
:10406800591C92F82C2021601A7023682A68591C60
:1040780092F8362021601A7023682A68591C92F831
:10408800372021601A7023685A1C22601E7023682A
:104098005A1C22601E7023685A1C22601E702B68EE
:1040A8002046598FFEF7CBFC2B682046198FFEF768
:1040B800C6FC23682A68591C92F82E2021601A70C1
:1040C80023685A1C22601E702B682046598EFEF702
:1040D800B6FC2B682046998EFEF7B1FC01231A46E0
:1040E80053E42368164A1749D078174A5D1C25609F
:1040F800187023684979581C206019702168D07895
:104108001EE60DF1180900250695DFF844A00F4BAF
:1041180004950595C9F8045001214FF6FF7B1FE06F
:10412800D8820020F8580020A48A00206687002042
:1041380068870020447C0020747F0020EC3F00202A
:104148001C790020308C002078890020BC3F00209A
:10415800C054030801350B2D01F0FD831AF9011F26
:104168004F1C4BFA05F2F5D0D607F3D51A882A4129
:10417800D007EFD548460193FEF748FE019BE9E7D3
:10418800B54B9B8AB3F5006F01F29184B3F5806F4C
:1041980001F21985B3F5007F34BF01270227AF4D1F
:1041A80005F10C0655F8041B91FBF7F1204689B27E
:1041B800FEF745FCAE42F5D1A94DAA4F05F10C0614
:1041C800B5EC010AD7ED087A80EE270A2EF054FFE5
:1041D80081B22046FEF733FCAE42F1D1A24D05F183
:1041E8000C0655F8041B204689B2FEF728FCB54298
:1041F800F7D1FFF7C8BB10229C492046FEF7F1FB18
:1042080001231A46FFF7C1BB994D9A4EDFF8A882E1
:10421800DFF8A8929FED988A05F120070EE0FCEEE2
:10422800E77ACDED017ABDF8041020460435FEF793
:1042380006FCBD4206F118063FF4A5AB717C0029C7
:10424800F3D098F80030D5ED007A012BE7D1D9F8F2
:104258000030DB0441F12184F5EE407AF1EE10FAEA
:1042680041F0D88440F2DC51DFE7844D20462988AC
:10427800FEF7E5FB69882046FEF7E1FBB5F9043057
:104288007F49DA1781FB0313C2EBA30399B22046D7
:10429800FEF7D5FB01231A46FFF777BB794E337833
:1042A800002B3FF470AB784F002537F8021F2046EB
:1042B800FEF7C5FB337801359D42F6DBFFF763BB9C
:1042C800724B20461968FEF7A3FB714B20461988EC
:1042D800FEF7B5FB01231A46FFF757BB6D4D236860
:1042E8002A68591C127821601A702B6822689978FC
:1042F800531C2360002311702A6821681A44013373
:104308005279481C032B20600A70F5D123682A686B
:10431800591C127A21601A7023682A68591CD278AD
:1043280021601A7023682A68591C127921601A7052
:104338002B6820465989FEF782FB23682A68591C96
:10434800527A21601A702B6821685878F8E4524F25
:1043580000232268386803EB4301551C405C256044
:1043680010703A6820680A44451C5278256002702B
:104378003A6820680A4401339278411C0A2B21606C
:104388000270E6D1FFF7FFBA444952232268501C55
:104398002060137011F8013F002BF7D1FFF7F3BA33
:1043A8003F4D05F16006A9882046FEF748FBE988DD
:1043B8002046FEF744FB29892046FEF740FB236888
:1043C800AA7A591C21601A702368EA7A591C21605C
:1043D8001A7055F80C1B2046FEF71AFBAE42E2D1C4
:1043E800FFF7D1BA2F4D20462988FEF728FB6988A8
:1043F8002046FEF724FBA9882046FEF720FB012370
:104408001A46FFF7C2BA2268274B26491878551C66
:104418002560107022685878551C25601070226835
:104428009B78501C20601370C9882046FEF707FB54
:1044380001231A46FFF7A9BA23681C4A1C491078B9
:104448001C4A5D1C2560187023688978581C2060F8
:1044580019702168907873E4B0470020E84700207D
:104468008C7F002028700020F84700201C8700203F
:104478002C870020847B002000004042CC3F002095
:10448800676666664C480020CE6E0020C88A002009
:10449800FC3F00200C290020EC3F0020905403082A
:1044A800F49100207032002040240020747F002006
:1044B8001C79002078890020687C0020987F0020E3
:1044C800DFF804E30027FEB2714600232268501C7F
:1044D800206016702268501C20601370226811F842
:1044E800010F0133551C062B25601070EED10137E2
:1044F800062F0EF1060EE6D1A54900232268501CAE
:10450800206017702268501C20601370226811F810
:10451800010F0133551C0B2B25601070EED1236859
:104528009C4A581C07212060197023680021581CD8
:1045380020601970216892F8F00001E4964D204639
:10454800298AFEF77CFA698A2046FEF778FAA98A52
:104558002046FEF774FA01231A46FFF716BA8F4B66
:1045680022681978FFF7E7BB8D4D23682A7A591C12
:1045780021601A70A98B2046FEF761FA298B204624
:10458800FEF75DFA698B2046FEF759FA2368EA7C44
:10459800591C21601A70A98C2046FEF750FAE98C44
:1045A8002046FEF74CFA2368AA7F591C21601A702E
:1045B800236895F82020591C21601A70698C2046C0
:1045C800FEF73DFA2368EA7A591C21601A70E968F7
:1045D8002046FEF71DFA23682A7C591C21601A70B0
:1045E800216895F82100FFF7ABBB6A4D05F140063D
:1045F800B5F880102046FEF722FA236895F8822045
:10460800591C21601A70236895F883200435591CB9
:10461800B54221601A70EBD1FFF7B5B9614D05F1CC
:10462800800655F8041F2046FEF7F2F9B542F8D186
:10463800FFF7A9B95A4B2168587DFFF781BB5A4B40
:1046480003F15A0522685979501C206011702268BC
:104658001978501C2060117022685978501C20600D
:10466800117022689978501C206011702268D978DE
:10467800501C20601170226819790633501C9D4225
:1046880020601170DED1FFF77EB9484D484E05F124
:10469800300795F90210474B93F906208A4203F137
:1046A800080301F03A81B342F6D10835BD42F0D192
:1046B800FFF769B9404B03F1700522681978501C5F
:1046C8002060117022685978501C2060117022688F
:1046D8009978501C206011702268D978501C20608D
:1046E800117022681979501C20601170226859795C
:1046F800501C20601170226899790733501C9D4224
:1047080020601170D9D1FFF73EB92C4D28462DF005
:10471800F5FA00287FF737A92B460544226813F8D5
:10472800011B501CAB4220601170F7D1FFF72BB969
:10473800234D05F1500628782CF0F4FF2368027AFF
:10474800591C21601A7023686A78591C21601A70F4
:104758002368AA78591C21601A702368EA780435FE
:10476800591CAE4221601A70E5D1FFF70CB9154DFE
:1047780020462988FEF763F9A9882046FEF75FF9E5
:1047880029892046FEF75BF901231A46FFF7FDB891
:10479800633F0020803E0020447C002008890020E0
:1047A800545000207C3E002098300020488600208D
:1047B80008810020D88000205C8F0020D43F002092
:1047C8000C8900200C3B00203F3F00202368A04FAD
:1047D800591C3A7821601A703B78002B3FF4D3A813
:1047E8000025EEB230461EF09BF923684278591C2A
:1047F800216030461A701EF093F901892046FEF7B1
:104808001EF93B7801359D42EBDBFFF7BCB8914DB3
:104818002046E989FEF713F9A9892046FEF70FF922
:1048280001231A46FFF7B1B88B4B8C49B3F9003016
:1048380081FB0321DB17C3EBA10189B22046FEF7F8
:10484800FEF801231A46FFF7A0B8731C30462B6008
:1048580010F8377B0DF1170201332B6013F8011C98
:1048680002F8011F9842F7D1DFF8109299F800502A
:10487800002DFDD1DFF808A20126042089F8006088
:1048880022F070FBDAF80000FDF7A6FB744B28460F
:104898001E7022F091FA284622F08EFA092022F0A2
:1048A8008BFA384622F088FA06AF3D460DF14E08DD
:1048B800EE1BF6B20A2022F07FFA304622F07CFA8C
:1048C80015F8016B0B2022F077FA304622F074FAC3
:1048D8000020FCF7C1FA4545EAD1082022F06CFA1D
:1048E800A02022F069FAA02022F066FA002022F027
:1048F80063FA10F02005F6D1DAF80000FDF771FB35
:10490800022022F02FFB012389F800501A46FFF7F6
:104918003CB8731C2B603778FF2F01F0E681FE2F1F
:1049280001F065812846FEF74CF895E80C009B1AC3
:10493800002B06DD531C2B60137813B90B2F41F2A3
:10494800B781242F00F2AA82464A012322F81700D1
:104958001A46FFF71AB8731C2B6033780A2B01F03C
:1049680035812846FEF738F82846FEF735F82846F8
:10497800FEF732F8FFF707B8731C2B60307803286E
:1049880000F28C82431E384E3849DBB203EB4303F6
:1049980006EB430308705E7800283EF4F4AF531E1C
:1049A800DBB2B34240F07A820022C1F80620C1F897
:1049B80002208A725BB1581C2B6808444A1C0133D8
:1049C8002B6013F8011C02F8011F9042F7D1284B05
:1049D8001B78002B3EF4D7AF27F032FC01231A4690
:1049E800FEF7D3BF3346721C2A60224F13F8022BFE
:1049F8007A702B6073783B70F31C2B60B378BB70B4
:104A08002846FDF7DEFF2B6838811A46591C2960B5
:104A180012F8021B79712A605B78BB7101231A4670
:104A2800FEF7B3BF731C2B6033780A2B01F0C580E7
:104A3800502B40F0E8832846FDF7C3FF0E4E308028
:104A48002846FDF7BEFF012370801A46FEF79DBF7A
:104A58000D4900201C790020788900206766666669
:104A680042430020288A0020746903082C83002010
:104A7800383B0020948A0020203300203B4300204C
:104A880034860020A8F10B00EF2800F2078201A36A
:104A980053F820F021540008A54E0008A54E000840
:104AA800A54E0008A54E0008A54E0008A54E000812
:104AB800A54E0008A54E0008A54E0008A54E000802
:104AC800A54E0008A54E0008A54E0008A54E0008F2
:104AD800A54E0008A54E0008A54E0008A54E0008E2
:104AE800A54E0008A54E0008A54E0008A54E0008D2
:104AF800A54E0008D1530008A54E0008B75300087A
:104B0800A54E000895530008A54E0008A54E0008BC
:104B1800A54E00086D530008A54E00081353000861
:104B2800A54E0008E1520008A54E0008BB52000837
:104B3800A54E0008A9520008A54E000855520008C5
:104B4800A54E00085D4E0008A54E0008A54E0008B9
:104B5800A54E0008A54E00088F390008A54E00088C
:104B680039520008A54E0008A54E00081F5200083B
:104B7800A54E0008CD510008A54E0008A54E000816
:104B8800A54E0008A54E0008A54E0008A54E000831
:104B9800A54E0008A54E000849510008A54E00087A
:104BA800FB500008A54E0008A54E00081158000843
:104BB800A54E0008A54E0008A54E0008A54E000801
:104BC800A54E0008A54E0008A54E00082B57000862
:104BD800A54E00081B560008A54E0008B155000850
:104BE800A54E000809550008A54E0008A354000862
:104BF80085540008A54E0008A54E0008A54E0008DB
:104C0800A54E0008A54E0008A54E0008A54E0008B0
:104C1800A54E0008A54E0008A54E0008A54E0008A0
:104C2800A54E0008A54E0008A54E0008A54E000890
:104C3800A54E0008A54E0008A54E0008A54E000880
:104C4800A54E0008A54E0008A54E0008A54E000870
:104C5800A54E0008A54E0008A54E0008A54E000860
:104C6800A54E0008A54E0008A54E0008A54E000850
:104C7800A54E0008A54E0008A54E0008A54E000840
:104C8800A54E0008A54E0008A54E0008A54E000830
:104C9800A54E0008A54E0008A54E0008A54E000820
:104CA800A54E0008A54E0008A54E0008A54E000810
:104CB800A54E0008A54E0008A54E0008A54E000800
:104CC800A54E0008A54E0008A54E0008A54E0008F0
:104CD800A54E0008A54E0008A54E0008A54E0008E0
:104CE800A54E0008A54E0008A54E0008A54E0008D0
:104CF800A54E0008A54E0008A54E0008A54E0008C0
:104D0800A54E0008A54E0008A54E0008A54E0008AF
:104D1800A54E0008A54E0008A54E0008A54E00089F
:104D2800A54E0008A54E0008A54E0008A54E00088F
:104D3800A54E0008A54E0008A54E0008A54E00087F
:104D4800A54E000859540008A54E0008C15800088F
:104D5800A54E0008A54E0008A54E0008A54E00085F
:104D6800A54E0008A54E0008A54E0008A54E00084F
:104D7800A54E0008A54E0008A54E0008A54E00083F
:104D8800A54E0008A54E000865580008A54E000865
:104D9800D7580008A54E00088F5600080959000882
:104DA80049580008A54E0008E1500008A54E000823
:104DB800B9500008A750000849500008A54E00083F
:104DC8001F500008A54E0008A54E0008FD4F00081A
:104DD800CF4F0008BB4F0008934F0008734F0008DF
:104DE800514F0008A54E0008394F0008A54E00088D
:104DF800A54E0008A54E0008A54E0008A54E0008BF
:104E0800A54E0008A54E0008A54E0008A54E0008AE
:104E1800A54E0008A54E0008A54E0008A54E00089E
:104E2800A54E00081F4F0008A54E0008A54E000813
:104E3800C74E0008A54E0008A54E0008A54E00085C
:104E4800A54E0008A54E0008A54E0008A54E00086E
:104E5800AF4E00080723B2FBF3F3C3EBC301521AAA
:104E68001CD1DBB203F1FF385FFA88F8002B3EF45F
:104E78008AADDFF80C9308F101081746731C2B6004
:104E8800BF4B96F90010002693F902208A4203F1DD
:104E9800080300F0DF860136062EF5D14FF0FF3308
:104EA8001A46FEF772BDB74B1B78DB07F6D401F044
:104EB800CDFD02F0CDFB01231A46FEF766BD731C3B
:104EC8002B6033780F2BE9D8B21C2A60C3EBC303DD
:104ED800AD4A7178D154F11C29601344B2785A70E4
:104EE800321D2A60F2789A70721D2A603279DA705F
:104EF800B21D2A6072791A71F21D2A60B2795A714C
:104F080006F108022A60F2799A712BF071F90123EF
:104F18001A46FEF73ABD2846FDF753FD9B4EF08131
:104F28002846FDF74EFD0123B0811A46FEF72DBD38
:104F38002846FDF746FD964900EB80004200012314
:104F48000A801A46FEF721BD2846FDF73AFD914E24
:104F580030822846FDF735FD70822846FDF731FD81
:104F68000123B0821A46FEF710BD3346721C2A6030
:104F780013F8020B2B60F31C71782B60B2781AF0CF
:104F8800B7F800287EF4FFAC88E73346721C2A6025
:104F9800814A13F8021B11702B607C4A7378937056
:104FA800F31C2B607A4BB2789A7001231A46FEF7ED
:104FB800ECBC7A4B7A4918684E222DF053FE012337
:104FC8001A46FEF7E2BC3246731C2B60754B12F88A
:104FD800021B19702A6072785A70F21C2A60B27823
:104FE8009A702846FDF7EDFC6F4A0123D0801A46D7
:104FF800FEF7CBBC2846FDF7E4FC6B4E3080284614
:10500800FDF7DFFC70802846FDF7DBFC0123B0804C
:105018001A46FEF7BABC654F3B78002B3EF4B3AC9A
:10502800DFF8988100262846FDF7CBFC14F010FD28
:105038003B78A8EC010A01369E42F4DBFEF7A3BCDC
:105048000D2A7FF42BAF731C2B603678072E3FF6A2
:1050580025AFDFF86C8128460C27FDF7B2FC07FB6B
:1050680006F708EB0706B0802846FDF7AAFCF08093
:105078002846FDF7A6FC2B6830811A46591C296082
:1050880012F8021BB1722A605B78F3722846FDF7AA
:1050980081FC012348F807001A46FEF776BC28462B
:1050A800FDF78FFC424A012310801A46FEF76DBCBB
:1050B800731C2B603078060600F1FC86314B1B7898
:1050C800DD073EF560AC032828BF002001F0A2FCF4
:1050D80001231A46FEF759BC2A4B1B78D8073EF520
:1050E80052AC01F083FD02F0B3FA01231A46FEF731
:1050F8004CBC731C2B6096F80080B8F1110F3FF67A
:10510800CDAEB31C2B602B4F737807F818302846A8
:10511800FDF757FC40F6CA039842A8BF184640F26C
:10512800EE23984207EB4807B8BF18460123A0F2C0
:10513800EE211A46192091FBF0F17970FEF725BC93
:105148003346721C2A601C4F13F8022B3A712B60ED
:1051580073787B712846FDF734FC2B6838805A1C1D
:105168002A601B78BB712846FDF72BFC2B687880DA
:105178005A1C2A601B78FB7101231A46FEF705BCEE
:1051880048860020C04F00205C8F00201C7900203A
:1051980078890020447C0020747F0020EC3F0020A8
:1051A800F469030840240020703200200D490020D3
:1051B8003C240020088E00208C320020C4310020BE
:1051C800F4910020731C2B60BE4B3278BE4F1A70CE
:1051D80000233B602846FDF7DDFB2A683B68BB4996
:1051E800BB4E0343501C3B60286013780B72284663
:1051F800FDF7E7FB30602846FDF7E3FB70602846C3
:10520800FDF7DFFBB0602846FDF7DBFB2846FDF71E
:10521800D8FBFEF7B8BBAF4B06F1080201362E608B
:1052280016F8011C03F8011FB242F7D1FEF7ABBB19
:105238003346721C2A60A84A13F8021B91702B602F
:105248007378537001231A46FEF79FBB731C2B60BB
:1052580033780E2B3FF622AEB21C2A6070780328F2
:105268003FF61CAE9D49062202FB03F28B18F71C81
:1052780058712F60B0788854321D2A60F2785A70BD
:10528800721D2A6032799A70B21D2A607279DA70BA
:10529800F21D2A60B2791A7101231A46FEF775BB0E
:1052A800731C2B60894B32785A7501231A46FEF716
:1052B8006CBB731C2B6036781F2E3FF6EFAD052AAA
:1052C8007FF4ECAD2846FDF765FB854B43F82600D7
:1052D8001AF0F6FCFEF757BB814E06F14007284648
:1052E800FDF76FFB2B68A6F88000591C1A46296049
:1052F80012F8021B86F882102A605B7886F88330E1
:105308000436B742EBD1FEF73EBB731C6F4F2B60E0
:1053180033783B722846FDF754FBB8832846FDF7DF
:1053280050FB38832846FDF74CFB2A687883531CCA
:105338002B601278FA746A68D31A032B00F3758508
:105348002B68D11A052900F35F85D21A002A7EF747
:105358001AAB5A1C2A601B7887F8213001231A4699
:10536800FEF713BB731C2B60564832780270C91ABB
:1053780000297EF708ABB31C2B607278003218BF87
:105388000122012342701A46FEF7FFBA2846FDF7AC
:1053980018FB4F4E30602846FDF713FB7060284617
:1053A800FDF70FFB0123B0601A46FEF7EEBA464E32
:1053B800002333602846FDF7EDFA326801230243E3
:1053C80032601A46FEF7E1BA731C2B603778132F48
:1053D8003FF664ADB31C2B6070782CF089F9002877
:1053E8003FF45CAD3F4B027803F82720F21C2A609B
:1053F80003EB8703B2785A70321D2A60F2789A70EC
:10540800721D2A6038493279DA7008680EF098FC03
:1054180001231A46FEF7B9BA3449102A13464FF049
:10542800000228BF10230A604A608A60CA600A74B2
:10543800002B3EF4A8AA2A680139134401322A60D5
:1054480012F8010C01F8010F9342F7D1FEF79BBA4D
:105458003346721C2A6013F8027B2B60F31C7078A9
:105468002B60B178002F00F0A484012F7EF48BAA62
:1054780015F0DCFF3B463A46FEF787BA1C4B1B7813
:1054880013F001017FF40AAD731C2B60307815F01E
:105498000FFF01231A46FEF778BA3346721C2A60BA
:1054A800144A13F8021BD1702B60134A7378537196
:1054B800F31C2B60114BB278DA7001231A46FEF701
:1054C80064BA00BF08890020D43C00205450002052
:1054D8000C3B002053500020302900209830002039
:1054E800803E00200C890020EC3F0020D43F0020A3
:1054F800C04F00201C790020308C002078890020C3
:105508002846FDF75EFA2846FDF75BFA2846FDF7C0
:1055180058FA2846FDF760FA2B68B44F1946581C0C
:105528003A68286011F8020B82F82C002960597833
:1055380082F83610D91C29609B7882F837302846C3
:10554800FDF74AFA2846FDF747FA2846FDF744FAD8
:1055580028463E68FDF735FA708728463E68FDF70D
:1055680030FA2B686A683087D11A01290ADD591C7C
:105578003A6829601B7882F82E302846FDF72CFA05
:105588002B686A68D31A032B09DD28463E68FDF7A5
:1055980018FA708628463D68FDF713FAA886386819
:1055A8002BF0D8F9FEF7EFB9731C2B608F4FDFF89B
:1055B8005082337888F8053028463E68FDF701FAAE
:1055C800308428463E68FDF7FCF96A682B68F0834A
:1055D800D11A072900F30084D11A032900F3EF83B5
:1055E800D21A002A05DD591C3A6829601B7882F80E
:1055F800263001F035FA25F0ADF97D4B38681B6887
:10560800002B00F0C2832AF087FE01231A46FEF71A
:10561800BCB93346721C2A60DFF8E48113F8022B08
:1056280088F802202B60734A73781370F31C2B6080
:10563800714FB3783B71331D2B60F378092BA8BFEA
:1056480009232846BB70FDF7BCF92B686A683880C7
:10565800D11A012905DD2846FDF7B3F92B686A68D8
:10566800F8819A4240F09C8301F0FAF92B686A6845
:105678009A423EF488A95A1C2A601B78FB700123C1
:105688001A46FEF782B9092A7FF708ACDFF8748159
:105698003346721CD8F800702A6013F8022B3A704F
:1056A8002B607378BB70F31C2B60B378642BA8BF96
:1056B8006423321D7B712A60F378642BA8BF6423AE
:1056C800721DBB712A603379FB71B31D2B6073792E
:1056D800642BA8BF6423F21D3B722A60B379FB7068
:1056E80006F108032B60F3793B712846FDF769F949
:1056F8006A682B687881D11A00290CDD591CD8F802
:1057080000002960521A002A1978417203DD9A1C98
:105718002A605B7843700EF085FB01231A46FEF77A
:1057280034B92846FDF74DF906461AF055FDFF280D
:105738003EF429A93F2E00F211830DF158090023E8
:1057480009F8403DF708494604A88DF8103001379C
:105758001AF022FD9DF81030FFB206F00706BB4292
:1057680006F1010603D19DF81830B34203D0314643
:1057780038461AF01DFD2B686A68D21A012A7EF78E
:1057880002A95A1C16A82A6000221E7800F8482D83
:105798001AF0F6FC9DF81030B3420AD0174B1B687C
:1057A8003BB19A79B24204D31B681B690BB13046EE
:1057B80098472B685A1C2A60484600221D788DF8A5
:1057C80018201AF0D1FC9DF81830AB423EF4DBA843
:1057D8000A4B1B68002B3EF4D6A81B685B69002B9C
:1057E8003EF4D1A828469847FEF7CDB8EC3F0020F4
:1057F800F08800200C910020447C0020E83F002025
:10580800747F00200C290020BF4B1B78012B3EF62B
:10581800BAA83246731C2B60BC4F12F8023BBB700F
:10582800F31CC91A2A60012972782B6040F3368369
:105838002846FDF7C6F8012338801A46FEF7A5B8B2
:10584800B34B1B78DA073EF59EA8B2490A780123C4
:1058580042F004020A701A46FEF797B8C2F34706E8
:10586800122E3FF61BABBEB116AB0DF1160803EBBB
:1058780046094746A9F142092846FDF7A2F827F844
:10588800020FB945F8D1A44B38F8022F23F8022F9C
:105898004745F9D1112E09D8A04A7300023B134499
:1058A8000021223223F8021F9A42FBD19C4901228F
:1058B80013460A70FEF769B89A4E002328463360EB
:1058C800FDF768F8012330601A46FEF75EB8964B7C
:1058D8001868F31C02462136991E296013F8031C28
:1058E8001170591E296013F8021C51702B6013F8AF
:1058F800011C91700333B34202F10302ECD14FE66D
:10590800834B1B78D9073EF53EA8884A4FF4C871E7
:10591800012311801A46FEF738B823685A1C226002
:10592800197029882046FDF78AF82368EA78591CF7
:1059380021601A7023682A79591C21601A7023681B
:10594800AA79591C21601A7023686A79591C216048
:105958001A70FEF7AABEDFF800B200254FF0080A59
:105968000135C5F120020AFA02F2A5F120032BFA4B
:1059780005F616432AFA03F31E43252D06F0010205
:105988004FF000030BD01343EAD0E8B20EF0D2F97F
:105998000028E5D029464846FDF738FAE0E75C4B91
:1059A8001B78DA0700F1F9800025614E2F4602E0E6
:1059B8000135252D0DD029463046FDF736FA002849
:1059C800F6D029464846FDF730FA002860D101375D
:1059D800EEE7584B584DB3F850102046FDF72FF816
:1059E800564B1988204689B2FDF729F8544B1A6896
:1059F800530103F02001C2F340030B43C2F38001BB
:105A080043EA4103C2F3C00143EA8103C2F34011F0
:105A180043EAC10102F0100211432046FDF70FF8D6
:105A280004A904222046FCF7DCFF23682978454AAC
:105A3800581C2060197011886429A8BF6421204669
:105A4800FCF7FDFFB8F1960F00F0AC80002120466E
:105A5800FCF7F5FF2168B7F1190348BFA7F1120356
:105A6800A3F3C4034A1C226020461A460B7005A9FA
:105A7800FCF7B7FF2368344A581C102120601970BE
:105A880011882046FCF7C4FF01231A46FDF77DBFA5
:105A9800394604A8FDF7BAF999E7F4EEC87AF1EEA9
:105AA80010FA80F210814FF47A71FEF7BEBB082716
:105AB800FEF775BB236898F80210244A581C20602A
:105AC800197023681278591C21601A70FEF768BA99
:105AD80095F824201E4B002A40F0E1803046FEF75E
:105AE800CDB95A1C19462A601A4811F8022B0270BF
:105AF80029605B784370042A30D9FF2A3EF4A9A8AC
:105B080021680020FEF71CB9C13C0020A48A0020AF
:105B1800C04F0020908A0020428C0020448C002036
:105B2800688C00208C300020EC3F00202C290020BD
:105B38003C93002050000020F03F00204C2A002019
:105B4800E88A0020502A0020EC8A00200C910020CE
:105B5800F85800202024002090E33FF4C349097836
:105B6800994203D8022ACBD1FF2BC9D1226801233D
:105B7800D11821601370B9F1000F3DF404AFBC4A8D
:105B8800C9F800201A46FDF700BF21680123CA188A
:105B980022601A460870FDF7F8BE069B43F0010321
:105BA800069301E723680322591C21601A702368B1
:105BB8006A78591C21601A704CE72846FCF701FFE7
:105BC800AC4EFEF73CBF0427FEF7E9BAB31C2B60C6
:105BD800A94B72781A70F21C2A60B2785A70321D7A
:105BE8002A60F2789A7001231A46FDF7CEBEB31CDC
:105BF8002B607678022E3FF651A92846FCF7E1FE85
:105C08009E4A02EB46024FF0FF33A2F85C001A46A8
:105C1800FDF7BBBEF4EEC87AF1EE10FA3EF522AB02
:105C28009FED977AF4EEC77AFDEEE77AF1EE10FA77
:105C380017EE901A00F283806FF4F973303903FB82
:105C480001F140F2E73391FBF3F101F2DB5189B244
:105C5800FEF7EBBA09EBC60A28468AF80210FCF7E9
:105C6800B0FE2B6829F836001A46591C296012F82C
:105C7800021B8AF803102A605A788AF80420DA1C72
:105C88002A609A788AF806201E1D2E600137DB7874
:105C98008AF80530B8457FF4F1A8FDF774BE597845
:105CA800022943D003290CBF04203046FEF7E6B88A
:105CB800724B00301F4418BF0120012387F84A00A7
:105CC8001A46FDF762BEFDEEE77A40F2E73317EEBB
:105CD800901A303903FB01F140F2CF7391FBF3F1D5
:105CE80001F2E93189B2FEF7A0BAB31C2B60654B0B
:105CF80072781A70F31C2B60604FB37887F85B30AA
:105D0800331D2B60F37887F85A302846FCF759FE84
:105D1800A7F856002846FCF754FE2846FCF751FE23
:105D28000123A7F858001A46FDF72FBE042A34BFEE
:105D380002200320FEF7A2B84246FDF7CFBF40F28B
:105D4800F313A1F5836103FB01F140F2E73391FB03
:105D5800F3F101F2DD5189B2FEF767BA0DF11809C6
:105D680048461AF0F5F9BDF81830B3423FF403ADD0
:105D7800454B1B68002B3FF4FEAC1B689B69002B4E
:105D88003FF4F9AC30469847F5E4404B404A414867
:105D980041491A60012302600A601A46FDF7F5BD01
:105DA8005A1C2A601B78003318BF012388F8073073
:105DB8005AE42AF047FC01231A46FDF7E6BD2846B7
:105DC800FCF7FFFDA8F80E002846FCF7FAFD2B6843
:105DD8006A68A8F8100003E42846FCF7F2FDA8F862
:105DE8000A002846FCF7EDFDA8F80C0028463E6896
:105DF800FCF7E7FD708428463E68FCF7E2FD2B6857
:105E08006A68B084FFF7E8BB5A1C2A601B78FB72EB
:105E18002846FCF7BFFD2B68F8605A1C2A601B78DF
:105E28003B742B686A68FFF790BA2846FCF7C9FDEF
:105E3800B8842846FCF7C5FD2B686A68F884D11A2F
:105E480003297FF77EAA1A46591C296012F8021BFB
:105E5800B9772A605B7887F820302846FCF7B1FDCF
:105E68002B686A687884FFF76CBA00BF0D49002078
:105E780099620008D8240020933B0020288A00203B
:105E880000E082443C860020E83F00204C9000203F
:105E9800C3060008A0900020089100200B4BB078A2
:105EA8001988012311FB02F11A4691FBF0F13980A0
:105EB800FDF76BBD00F07F00032828BF002015F018
:105EC800D1FA01231A46FDF760BD00BF668700209E
:105ED80038B50B4C23688BB15A68821A002A0546DC
:105EE80004DA0CE05A68AA1A002A07DB9A682260CA
:105EF80018461A6890472368002BF3D138BD38BD7F
:105F0800F07400200B4B002210B4027203F18C04D1
:105F1800012102E0072A09DC9979890702D5197954
:105F2800815401329C4203F11403F3D15DF8044B10
:105F3800704700BF507A030824230370704700BFDE
:105F480001231021112241704271037003717047BF
:105F58002DE9F0410B78057BDB43DFB200F113023A
:105F680000F11D0302F8015F9342FBD1DFF890E0D6
:105F780000F12701002203F8012F9942FBD11421D7
:105F88000524002647FA04F303F00103002B1E44FE
:105F980014BF4FF019084FF00A0814F0010FF6B2B9
:105FA80014BFAC464FF0000C0023CA1810FA82F256
:105FB8000133434582F814C0F7D15A1E92B2013218
:105FC800013C8B18621C9BB201D01946DAE716F027
:105FD800010F14BF19240A240022991810FA81F11C
:105FE8000132A2420D75F8D113449BB25A1C0344E6
:105FF800002192B21975AEF800200261BDE8F08167
:10600800242400202DE9F04FDFF890A0BAF80230E0
:106018000B3383B01FFA83F901F1060B4FF0010827
:106028004FF0000C002711F801EB3E464C460122C8
:10603800A4F10B039BB2019105E001339BB2017BF4
:1060480029759C4208D0C518002AF6D1C518013315
:106058009BB29C422A75F6D103190136092F019982
:1060680083F814C0F6B20CD0092E15D008FA07F33D
:1060780013EA0E0F14BF012200220C34A4B2013718
:10608800D6E709F1780959451FFA89F9CAD1AAF85A
:1060980002C003B0BDE8F08F0022EEE72424002000
:1060A8002DE9F047DFF85C80B8F8043004331FFAB4
:1060B80083FC01F109094FF0010E11F8017B6446D8
:1060C8000026231F0EFA06F29BB23A40C2B1B0F87E
:1060D8000CA0C51801339BB29C4285F814A0F5D1D9
:1060E80001360434082EA4B2EBD10CF1200C49453A
:1060F8001FFA8CFCE1D10023A8F80430BDE8F08732
:106108009246E6E72424002010B40268047B116854
:106118000223A340194209D00649406800240C70A4
:1061280001684FF6FE742140016053605DF8044B2E
:10613800704700BF28830020436A8269D154436AAC
:106148000169426B01338B4228BF00234362002A56
:106158002FD0EFF31181502383F31288436B1A6811
:10616800D2072CD470B45E686EB9456A826A9542CB
:1061780017D084691444DC600ED9AA1A5A60856263
:10618800002280F850201A6842F00102C9B21A6051
:1061980081F3118870BC70470469A21A5A6086623C
:1061A800EEE7012380F85030C9B281F3118870BC42
:1061B8007047C26C136843F0800313607047C9B21C
:1061C80081F31188704700BF026B10B462B1036C91
:1061D800C2684469D11A013B615C5DF8044B08BF91
:1061E80013460364C8B27047016A4369C4685B5CBC
:1061F8000131A14228BF114601625DF8044BD8B2B3
:10620800704700BF436B13B190F850007047836A22
:10621800406A181AB0FA80F040097047416A836AE8
:1062280099420AD3CB1A416B026961B14968501E81
:106238000B4483420AD2C01A704702691144CB1A30
:10624800416B0029F2D1501EC01A704700207047D8
:10625800036B43B1026C5B6893422FBF981AC06806
:106268009B1AC0187047C269036A9A422FBFD01A96
:10627800C0688018C01A704708B513F06BFC024B51
:10628800024ADA60FEE700BF00ED00E00400FA050C
:10629800024A034B1278197819F0BABF202400205B
:1062A800212400202DE9F0470569C3681D4028D046
:1062B8000F4606464FF000484FF00009B5FA85F33F
:1062C80028FA03F2D2431B3B32611540042B16D83F
:1062D800DFE803F03129211903007B6A002B32D053
:1062E80003F1FF3A1FFA8AFAC7F824903C6A34B1DE
:1062F80023682046514698476468002CF8D1002D41
:10630800DCD1BDE8F0873868716B036889B29847BB
:10631800002DD3D1F5E77868B16B036889B2984747
:10632800002DCBD1EDE7B868F16B036889B29847C7
:10633800002DC3D1E5E7F868316C036889B2984746
:10634800002DBBD1DDE7F36A1FFA83FACEE700BF61
:10635800442800F07C822DE9F0470C4642D9812878
:1063680000F01B8200F28D80542800F0C38040F2B8
:10637800A1816E2800F07182802840F00B82B84B12
:1063880093F8009009F1020919F0FF0900F08D80D7
:10639800B44BB54FB54EDFF818A3994403F1010883
:1063A8000A2516E0322D00F09B82A5F13C00C0B210
:1063B800132840F29B8200232268511C216015702B
:1063C8002268C84502F10101216013706DD018F8E8
:1063D800015B0A2DE6D1BAF80030FF2BA8BFFF23D6
:1063E800DBB2E9E7052800F020821AD8022879D024
:1063F80040F2FF80032800F0BC81042840F0CA81E5
:1064080002469B492046FCF7ECFA20460021FCF79F
:1064180016FB23680222591C21601A700120BDE86E
:10642800F087242856D040F2F780282800F05F81B2
:10643800382840F0AF810A688E4B0120511C21603A
:1064480010702268052115182560117022680A212C
:106458001518256011702268002115182560117023
:10646800226819781518256011702268597815184E
:106478002560117022689B78111821601370BDE89F
:10648800F087A02814D040F28480B82800F06981F1
:10649800FE2840F07F81784D05F1080635F8021B8B
:1064A8002046FCF7CCFAAE42F8D10120BDE8F087CF
:1064B800724B08461968FCF7ABFA714B204619680D
:1064C800FCF7A6FA6F4B20461968FCF7A1FA0120E1
:1064D800BDE8F0876C4B08461968FCF799FA01206B
:1064E800BDE8F087084604226849FCF77AFA0120DB
:1064F800BDE8F0870B68664A664F581C112120607A
:10650800197023681278591C21601A70236897F84B
:106518005B20591C21601A70236897F85A20591C6F
:1065280021601A70B7F856102046FCF788FA002147
:106538002046FCF784FAB7F858102046FCF77FFA93
:10654800BD1E07F1480635F8021F2046FCF777FA0A
:10655800AE42F8D12268504B0C21501C20605D18C7
:106568001170226813F8011F501C9D4220601170A1
:10657800F7D123680222591C21601A70B7F85C1001
:106588002046FCF75CFAB7F85E102046FCF757FA8D
:106598008BE7822840F0FE800B68404A404D117816
:1065A800404A581C2060197011892046FCF747FAA8
:1065B8003D4B22681B88FF2B02F10101A8BFFF2376
:1065C80021601370A96881F31001204689B2FCF795
:1065D80036FA296801F30F01204689B2FCF72FFA31
:1065E8002368324A591C127821601A700120BDE8CC
:1065F800F087012840F0CE800B680022591C2160EA
:106608001A7023685A1C2260187023682422591CA7
:1066180021601A70BDE8F087202840F0BB800B6825
:10662800204D591C6A7821601A7023682A78591CF1
:1066380021601A702368AA78591C21601A70298968
:106648002046FCF7FCF923686A79591C21601A7006
:106658002368AA79591C21601A700120BDE8F087C7
:106668000D490020D0540308676666664033002051
:10667800F53F0020933B002030490020ACF7FF1F76
:10668800B0F7FF1FB4F7FF1FD43C00209481030824
:106698003C860020288A0020718A0020C93F0020FB
:1066A800B4490020948A0020C0490020DC8A0020D8
:1066B8006C33002052286DD10A68A44E531C032164
:1066C800236006F10C071170334606200121226869
:1066D800551C2560117022689F4202F1010121605A
:1066E800107000F0DA809979D8790633EFE70B68F3
:1066F800DFF89882964E591C022221601A7023688E
:1067080006275A1C22601F7023680A22591C216020
:106718001A70236801255A1922601D70B8F80010F4
:106728002046FCF78CF9B8F802102046FCF787F9E8
:1067380023685A1922601F70236850225919216052
:106748001A7023680022591921601A70318820466E
:10675800FCF775F920467188FCF771F92846BDE801
:10676800F0877C4B08461968FCF752F90120BDE810
:10677800F0870B685A1C0A6018700B680222591CB3
:1067880021601A7023680022591C21601A700120A8
:10679800BDE8F0870020BDE8F0876F4B1E78033610
:1067A80016F0FF063FF481AE6C4B6D4F1E4403F1AB
:1067B80001094FF00A0820E0B8F1500F00F08E8070
:1067C800B8F1320F00F0A780A8F13C00C0B213283E
:1067D80040F2A4800025294623685A1C22602046DE
:1067E80083F80080FCF72BF929462046FCF727F9A7
:1067F8004E453FF45AAE19F8018BB8F10A0FDBD1B8
:10680800584B9D68196805EB85054FF6FF736D00B9
:106818009D42A8BF1D469942A8BF194625EAE575BD
:1068280021EAE171ADB289B2D6E720460B224E4982
:10683800FCF7D7F8204608224C49FCF7D2F8204646
:1068480007224B49FCF7CDF80120BDE8F087002A64
:1068580042D0484B136001207047474B0A681B8899
:10686800464DFF2BA8BFFF23511C21601370A96858
:1068780081F31001204689B2FCF7E1F8404B20462D
:106888001988FCF7DCF8296801F30F01204689B262
:10689800FCF7D5F80120BDE8F0873A4B21681A7853
:1068A800481C20600A70002A3FF4FFAD013AD2B2BA
:1068B80002EB420206EB42025278002A3FF4F5ADA1
:1068C8000132D5180133226813F8011F501C9D426C
:1068D80020601170F7D1E8E5012070472A4B90E756
:1068E8003388FF2BA8BFFF23DBB265E51CF018F93E
:1068F80000283FF460AD03780A2B25D8B0F90230A0
:1069080087FB0312DB17C3EBA2039BB2FF2BA8BFC5
:10691800FF23DBB250E597E8220074E71CF000F98A
:1069280000283FF457AF03780A2B3FF653AFB0F96E
:106938000430B0F9061003EB830383F3500521EA12
:10694800E171ADB289B247E70023E2E77469030851
:10695800203300208C3000200D490020E05403082B
:1069680030330020EC3200209C810308A881030802
:10697800B481030881620008C0490020B44900209E
:10698800C48A00202C83002024330020D82400202F
:106998001C4C08B501210220FBF732FB237803F0D9
:1069A8000502052A2AD003F00903092B08D0002183
:1069B8000120FBF725FB00210846FBF721FBFEE73A
:1069C800114A124B11681A680B68114C4FF6FE7089
:1069D80003400B601388206823F001031B041B0C81
:1069E800138018B1292200238271C37102224E211B
:1069F800FAF786FE2068FBF7EFFAD8E713F03CF9C0
:106A08002378D0E7D43A0020742A0020782A00207E
:106A1800EC2A0020022828BF022010B4084C094B99
:106A2800207000EB8002C0EBC20207495DF8044BFE
:106A3800013003EB4203C0B20B602AF0BDBF00BFB8
:106A4800F03F0020A83B0020EC3F002008B522F0D2
:106A5800DDF9FBF7AFFDBDE8084022F0BFB900BF84
:106A680038B5434B5A899989914224BF00225A81EB
:106A7800198ADA89914224BF0022DA81DA788AB346
:106A8800072A2FD03B493C4D91F85700012400219B
:106A98000A282C709C70D9713DD00C2865D0DFED88
:106AA800377A8ABB364C9FED370AA278002918BF7F
:106AB800F0EE407A062A04D8334901EB820191EDC1
:106AC800080A217959B3013A032A4DD8F7EE007A1A
:106AD80087EE800A2CF0D0FA2388984228BF1846FF
:106AE800208038BDD97921B198780428B8BF04200E
:106AF8009870204890F857000A280CD00C28CED15E
:106B0800DFED227A002ACDD0072ACBD00A282CD153
:106B1800DFED1F7AC6E70A20DFED1E7AC1E79B7812
:106B2800154A07EE103A1178B8EEC77A27EE277A99
:106B380007EE901AF8EEE77A67EE877AB4EEE70A7E
:106B4800F1EE10FA10DDC0EE077AFDEEE77A17EEE7
:106B5800903A102BA8BF1023012BB8BF0123DBB23A
:106B68008B4238BF0B46137038BDDFED0B7A99E7BF
:106B7800747F0020287000200C9100206F120339C8
:106B8800447C00206F120338D05403080AD7A33975
:106B98000F506E3A5304E9386F12833A38B50C4CEB
:106BA8000C4DAC4206D2616820461434FBF78EFCCB
:106BB800AC42F8D3084A094B094C14600022094931
:106BC8001A705A7008480860BDE8384019F078B85B
:106BD800C8BE030878C30308EC3F0020F03F00203C
:106BE800A83B00200C2900208C47002008B5FFF79F
:106BF800D5FF22F00BF9FBF7DDFCBDE8084022F0D9
:106C0800EDB800BFF0B50C292BD8DFE801F06F2AEA
:106C18002A2A4C2A2A2A2B2A2A2A0700046AB2F886
:106C28000CE097881668674D24F480540462036A60
:106C38004468C16923F4005343EA0E3321F4E64162
:106C4800A84243EA073341EA062100F0B58005F57A
:106C58000065A84200F0B08092684460C161026497
:106C68000362F0BD046A96899588D2F800E0554F12
:106C780024F480740462036A4468C16923F40073CD
:106C880043EA062321F07301B84243EA052341EAA7
:106C98000E017ED04C4DA8427BD092684460C16101
:106CA800C2630362F0BD046A96899588D2F800E051
:106CB800444F24F010040462036A4468816923F095
:106CC800200321F0807143EA061321F4E641B8421B
:106CD80043EA051341EA0E2148D03B4DA84245D06E
:106CE80092684460816182630362F0BD046A93899B
:106CF800B2F804E01768334E24F001040462056A10
:106D08004468816943EA0E0321F4803125F00205C5
:106D18009BB221F07301B04243EA050341EA07013F
:106D280014D0294DA84211D005F54065A8420DD0D0
:106D380005F58065A84209D005F58065A84205D00B
:106D480092684460816142630362F0BDD689158A06
:106D5800578A23F0080333433D43D68824F440740C
:106D680023F00403ADB233432C43E9E7D589178AEE
:106D7800D68823F0800343EA051324F44064558A37
:106D880023F0400344EA870443EA061344EA8504EF
:106D9800A6E7D589178AD68823F4006343EA052332
:106DA80024F44054558A23F4806344EA071443EAE0
:106DB800062344EA051470E7158A24F4804444EA5B
:106DC800851449E7002C0140003401402DE9F04FBB
:106DD800F022002183B07948794CDFF80892794D88
:106DE800794E7A4FDFF800822EF053FA78487949C5
:106DF800DFF8F8E1DFF8F8C100221359834200F008
:106E0800C280B3F1804F00F0CA80AB4200F0C98065
:106E1800B34200F0C880BB4200F0C780734500F061
:106E2800C680634500F0C580434500F0C480DFF8A4
:106E3800C4A153457AD00AF5806A534508BF09238F
:106E480075D01432A02AD8D15D4C634D634E614F82
:106E580004F1A00802E01434A04564D0A379002B03
:106E6800F9D023794FEA131909F1FF39B9F1050F60
:106E780003F00F03EFD835F8190040FA03F2D207F0
:106E8800E9D54FF0010A0AFA03F3013B18402BF049
:106E98004FFC16F809305249184411EBC002DAD0F9
:106EA80051F83000DFF850E1217A00F138439B0AAD
:106EB8001EF8033003F01F0E5B09022B0AFA0EFAC4
:106EC80063D0032B66D0012B58D093880093B3FA74
:106ED80083F3C3F11F039BB2DA0800EB820203F0CD
:106EE8000703D2F820E09B004FF00F0C0CFA03FCCC
:106EF8002EEA0C0EC2F820E0D2F820E001FA03F3E3
:106F080043EA0E03136269460023022214348DF803
:106F180004208DF805308DF806308DF807301EF006
:106F2800C3F8A0459AD103B0BDE8F08F082309EB58
:106F3800C3034FF0010B93F840A00AF01F034FEA78
:106F48005A1ABAF1020F0BFA03F311D0BAF1030F70
:106F580008D0DA457FF475AFD1F814A043EA0A03E4
:106F68004B616EE7D1F81CA043EA0A03CB6168E7DE
:106F7800D1F818A043EA0A038B6162E77B694AEA01
:106F880003037B61A1E70023D1E7BB694AEA030356
:106F9800BB619AE7FB694AEA0303FB6195E70123B2
:106FA800C5E70223C3E70323C1E70423BFE705239B
:106FB800BDE70623BBE70723B9E700BFE48100204C
:106FC800507A030800040040000800400010004008
:106FD800002C0140001002400C7D0308187D0308B6
:106FE800547A0020D05403080040014000140040A7
:106FF8000034014000440140487A0308014902482E
:10700800FFF750B9AC820020004001400149024816
:10701800FFF748B984820020003401400149024842
:10702800FFF740B98482002000340140014902483A
:10703800FFF738B95C820020000800400149024887
:10704800FFF730B9348200200004004002494FF0B5
:107058008040FFF727B900BF0C8200200149024891
:10706800FFF720B9E4810020002C014001490248C3
:10707800FFF718B9E4810020002C01402DE9F04108
:1070880004684E4DA30AAB427AD00AD94C4DAB42A4
:107098005FD00335AB4277D0053DAB425DD0BDE84C
:1070A800F081B3F5801F67D0013DAB4259D14FF055
:1070B800700E022647794FEA970C002968D0B00075
:1070C800634685190227D4F80C809F400CEB4503D2
:1070D800BFB23C4D03F1040C47EA080745F82310FA
:1070E80045F82C20E760EFF31181502282F31288D3
:1070F800821905EBC2021369002B34D013620433E2
:10710800821905EBC202576917B11F60536904332E
:10711800821905EBC202976917B11F60936904339E
:10712800821905EBC202D76917B11F60D36904330E
:107138000027CAB21F6082F31188304405EBC000F3
:10714800036A9BB9E3684FF6FE721340E360BDE83B
:10715800F0814FF0C00E0426ACE74FF0200E002659
:10716800A8E7BDE8F08105EB0E03C9E7E36843F043
:107178000103E360BDE8F0814FF0480E012699E76E
:107188004FF0980E032695E74FF0E80E052691E795
:10719800BF08022306FA03F0BB40DB43E768094D4A
:1071A8009BB23B4087190CEB470CE3600CF10403DE
:1071B80045F82C1045F8232095E700BF0200100081
:1071C8004D001000E481002030B503685C4D18883C
:1071D8005C4CB4FBF2F20139013AAB4294B283B091
:1071E80089B282B266D05848834263D0B3F1804FE7
:1071F80060D0A0F5983083425CD000F5806083426F
:1072080058D0524883425BD000F5806083427DD0DD
:1072180022F4407200F58C3092B283421A80D9620F
:107228001C850ED0484A93420BD002F54062934227
:1072380007D002F58062934203D002F58062934240
:1072480001D100221A8601225A611A883C4992B259
:1072580042F001028B421A8062D0B3F1804F61D0B4
:107268003B4A934260D002F5806293425ED002F5B9
:10727800006293425CD002F5806293425AD002F5D4
:107288009032934258D002F54062934256D002F5AC
:10729800806293421ED002F58062934208BF0922A1
:1072A80019D002A84FF0012340F8043D1DF0CEFB91
:1072B80003B030BD254822F07002834292B2A3D1B8
:1072C80001201A80D9621C8558611A8892B202433B
:1072D8001A80C5E708221F4B03EBC20301A893F8E5
:1072E80041408DF80440012300228DF805308DF8C7
:1072F80007308DF806201DF0A9FB1B2CD8D1164BA2
:10730800019301A81DF0A2FB03B030BD01201A8033
:10731800D9621C8558611A8892B202431A809CE788
:107328000022D8E70122D6E70222D4E70322D2E7D7
:107338000422D0E70522CEE70622CCE70722CAE7D7
:10734800002C014000A24A04003401400010004013
:1073580000040040D054030819010001204B984252
:107368002DD0B0F1804F2CD0A3F5943398422AD079
:1073780003F58063984228D003F50063984226D02D
:1073880003F58063984224D003F59033984222D0C5
:1073980003F54063984220D003F58063984207D0F4
:1073A80003F58063984208BF092202D00020704785
:1073B80008220C4B03EBC20393F8400070470022ED
:1073C800F7E70122F5E70222F3E70322F1E70422B7
:1073D800EFE70522EDE70622EBE70722E9E700BF22
:1073E800002C0140D05403082DE9F04F013085B03E
:1073F800C3B203938E4D8F4F8F4C904E0A23029346
:10740800DFF8409223F0FEFF4FF4FA7A4FF0100CA9
:107418004FF47A70D9F80430C3F30803002B40F016
:10742800C880EFF31183002B40F0C3802968A2685D
:1074380000BF2B689942F9D1D7F800E000FB0EF3A2
:107448009B1AB3FBFEF300FB01314FF0010E0191D3
:10745800D9F80430C3F30803002B40F08E80EFF313
:107468001183002B40F089802B68A16800BF2A682F
:107478009342F9D1D7F800B000FB0BF2521AB2FBD5
:10748800FBF200FB0323019A9B1AB3F57A7FDFD343
:10749800BAF1010ABED1039B002B40F0C4804FF41F
:1074A8007A7ADFF8A09150464FF0100CD9F80430E2
:1074B800C3F30803002B40F09980EFF31183002BEE
:1074C80040F094802968A26800BF2B689942F9D1DE
:1074D800D7F800E000FB0EF39B1AB3FBFEF300FBAA
:1074E80001314FF0010E0191D9F80430C3F30803BC
:1074F8003BBBEFF3118323BB2B68A16800BF2A684D
:107508009342F9D1D7F800B000FB0BF2521AB2FB44
:10751800FBF200FB0323019A9B1AB3F57A7FE3D3AE
:10752800BAF1010AC2D1029B013B02937FF468AF12
:107538004349444B4448454A0860DA6005B0BDE811
:10754800F08FEFF311888CF31288A1682368DB03AE
:1075580044BFC6F800E0A1682B6832685FFA88F873
:1075680088F31188D7F800801A4400FB08F35B1AE7
:10757800B3FBF8F300FB0233CDE7EFF311888CF38C
:107588001288A1682368DB0344BFC6F800E0A1683D
:107598002B6832685FFA88F888F31188D7F800807A
:1075A8001A4400FB08F35B1AB3FBF8F300FB023341
:1075B80069E7EFF311828CF31288D4F808E02368A6
:1075C800D90303D501233360D4F808E02B68316868
:1075D800D2B282F311883A68194400FB02F3A3EB94
:1075E8000E03B3FBF2F300FB01312EE7EFF3118238
:1075F8008CF31288D4F808E02368D90303D5012353
:107608003360D4F808E02B683168D2B282F311886D
:107618003A68194400FB02F3A3EB0E03B3FBF2F341
:1076280000FB01315DE718461FF0C2FC37E700BFD9
:10763800E4720020E872002010E000E0E072002010
:10764800FC9F002000ED00E0EFBEADDE0400FA056F
:107658002DE9F047AB4FAC4E21F0D8FBBE421ED20D
:10766800DFF82C83DFF82C934446258862197DB116
:107678004A450DD2052D0BD933886188C3F30B0316
:10768800994200F0EE80144625886219002DEFD14A
:10769800716830461436FAF719FFBE42E4D39B4AA4
:1076A8001378A3F1170102290FD9994911F833006A
:1076B800002840F0F880D8000144497829B195495C
:1076C80011F83330002B00F01681934C6378022BAD
:1076D80084BF002363702378022B84BF00232370A8
:1076E8008E4B9A78042A00F0FD8032B91A88B2F5D8
:1076F800F07F84BF4FF4F0721A80894D894A2B6855
:107708001A40002A00F0FA80D80700F1E6805904F0
:1077180000F1DE801A0700F1D6809B0400F1CC80CE
:10772800814D2B685A8C998C914224BF00225A842F
:10773800FFF796F923F018FD10B97C480EF002FB0C
:107748008020FAF7F9FE4FF40070FAF7F5FE4FF0D3
:107758000070FAF7F1FE4FF08060FAF7EDFE6378FB
:10776800022B06D8724A734903EB430302EB8303E7
:107778000B602378022B07D803EB83016E4AC3EB17
:10778800C10302EB43032B600CF04CFB00213022B9
:107798006A482DF07EFD286828F070FF684B2E6837
:1077A80003F1500102E0043399427AD01A78002A92
:1077B800F9D19C78D8788442F5D26249624B91F825
:1077C80004E06248624D5C6B624B2860C827642104
:1077D80011FB0E71DFF8C0E159605F4F30F8061CED
:1077E8005E4DAEF8001000219960D96019615961A9
:1077F8009961D96183F8201083F821103A702E60BE
:107808000CB121F065F9564B9FED565A1B88564A24
:107818009FED566A557B564C56495748086006EE08
:10782800903AF8EEE66A1389C5EE265A07EE103A42
:107838005389127BC4ED005A07EE903AB8EEC77A26
:107848004E4BF8EEE77A1D725A7227EE067A67EE0B
:10785800867ABDE8F04783ED017AC3ED007A21F01E
:10786800BDBA63799B077FF40EAF716894F804A0E2
:107878003046FAF72BFE3388BAEB133F04D01436A0
:10788800BE42FFF4F1AE0AE773887068AA1FC3F31B
:107898000B039A4204F10601A8BF1A462BF0E2F93D
:1078A800EDE7012289E7D8000C186468002C7FF402
:1078B80003AF17241470FFE63148FAF73DFE402065
:1078C800FAF73AFE2CE72F48FAF736FE2B6824E73A
:1078D8002D48FAF731FE2B681CE72C48FAF72CFEE6
:1078E8002B6814E79A8AB2F57A7FBFF406AF4FF493
:1078F8007A729A8201E718231370E6E643F00103CF
:107908002B6001E778C30308C8BE03080889002074
:10791800E8760308307E0308F03F0020447C00200E
:10792800D43C002009600002EC3F0020488600207B
:107938008C4700200C290020A83B0020A825002007
:107948000C8900208C320020B047002022790020CA
:10795800149300200C4800204C000020DC25002057
:1079680074240020C0C9FB482424002017B7D1384C
:1079780078240020643000203661023D4030002029
:1079880009400002016000020920000208600002AC
:1079980002F0030800000408AC78002008B521F0C4
:1079A80035FAFAF707FE21F019FAFFF751FE012020
:1079B800BDE808402AF000B82DE9F04F013085B045
:1079C800C3B203930B4602918B4C8C4E002B00F0F4
:1079D80099808B4D8B4FDFF8309223F013FD4FF4D5
:1079E800FA7A4FF0100C4FF47A70D9F80430C3F3D8
:1079F8000803002B40F0DE80EFF31183002B40F0EA
:107A0800D9802968A26800BF2B689942F9D1D7F8B4
:107A180000E000FB0EF39B1AB3FBFEF300FB013101
:107A28004FF0010E0191D9F80430C3F30803002B7D
:107A380040F08780EFF31183002B40F082802B68A1
:107A4800A16800BF2A689342F9D1D7F800B000FBBB
:107A58000BF2521AB2FBFBF200FB0323019A9B1AAA
:107A6800B3F57A7FDFD3BAF1010ABED1039B002BAD
:107A780040F0BD804FF47A7ADFF88C9150464FF091
:107A8800100CD9F80430C3F30803002B75D1EFF3B9
:107A98001183002B71D12968A26800BF2B68994215
:107AA800F9D1D7F800E000FB0EF39B1AB3FBFEF305
:107AB80000FB01314FF0010E0191D9F80430C3F3F6
:107AC800080313BBEFF31183FBB92B68A16800BF50
:107AD8002A689342F9D1D7F800B000FB0BF2521A8A
:107AE800B2FBFBF200FB0323019A9B1AB3F57A7FE2
:107AF800E3D3BAF1010AC4D1029B013B0293002BE4
:107B08007FF467AF05B0BDE8F08FEFF311888CF311
:107B18001288A1682368DB0344BFC6F800E0A168A7
:107B28002B6832685FFA88F888F31188D7F80080E4
:107B38001A4400FB08F35B1AB3FBF8F300FB0233AB
:107B4800D2E7EFF311888CF31288A1682368DB036E
:107B580044BFC6F800E0A1682B6832685FFA88F86D
:107B680088F31188D7F800801A4400FB08F35B1AE1
:107B7800B3FBF8F300FB023370E7EFF311828CF3E9
:107B88001288D4F808E02368D90303D501233360A9
:107B9800D4F808E02B683168D2B282F311883A68C9
:107BA800194400FB02F3A3EB0E03B3FBF2F300FB53
:107BB80001317FE7EFF311828CF31288D4F808E0E3
:107BC8002368D90303D501233360D4F808E02B6870
:107BD8003168D2B282F311883A68194400FB02F383
:107BE800A3EB0E03B3FBF2F300FB013118E71846D1
:107BF8001FF0DEF93EE700BF10E000E0E072002071
:107C0800E4720020E872002000ED00E0204B5B6881
:107C1800C3F3080330B4BBB9EFF31183A3B91D4B09
:107C28001D4C1868A16800BF1A689042F9D11B4B17
:107C38001C684FF47A7202FB04F3591AB1FBF4F191
:107C480030BC02FB00107047EFF31182102383F35E
:107C5800128811498C680B6813F4803F104B02D0CE
:107C6800012018608C680B49D2B20D68186882F33D
:107C780011880A4B19684FF47A72284402FB01F301
:107C88001B1B30BCB3FBF1F302FB0030704700BF95
:107C980000ED00E0E472002010E000E0E87200204F
:107CA800E07200202DE9F84F8046FFF7AFFF254E20
:107CB8002549DFF8A0E0254A254D844610274FF4D2
:107CC8007A740120DEF80430C3F30803D3B9EFF364
:107CD8001183BBB90B68D2F808A000BFD1F8009097
:107CE8004B45F7D1D6F800B004FB0BF9A9EB0A090C
:107CF800B9FBFBF904FB0393A3EB0C034345E1D366
:107D0800BDE8F88FEFF3118A87F31288D2F808B02C
:107D18001368DB0344BF2860D2F808B00B68D5F8B5
:107D280000905FFA8AFA8AF31188D6F800A099447D
:107D380004FB0AF3A3EB0B03B3FBFAF304FB0933CD
:107D4800DAE700BFE8720020E472002010E000E0EB
:107D5800E072002000ED00E02DE9F04FDFF830C1BF
:107D6800474A4849484E494D8046102718F1FF3880
:107D7800C0F08480DCF80430C3F30803002B5CD126
:107D8800EFF31183002B58D10B68946800BF086883
:107D98008342F9D1D6F800904FF47A7000FB09FEBF
:107DA800AEEB040EBEFBF9FE00FB03EEDCF804307C
:107DB800C3F308034FF47A740120FBB9EFF311837E
:107DC800E3B90B68D2F808A000BFD1F800904B4582
:107DD800F7D1D6F800B004FB0BF9A9EB0A09B9FBF7
:107DE800FBF904FB0393A3EB0E03B3F57A7FBDD233
:107DF800DCF80430C3F30803002BDFD0EFF3118A5B
:107E080087F31288D2F808B01368DB0344BF2860F0
:107E1800D2F808B00B68D5F800905FFA8AFA8AF3AE
:107E28001188D6F800A0994404FB0AF3A3EB0B03CE
:107E3800B3FBFAF304FB0933D5E7EFF3118487F3B7
:107E48001288D2F808901368D80303D501232B6051
:107E5800D2F808900B682868E4B284F31188D6F841
:107E680000A04FF47A7400EB030E04FB0AF3A3EBB3
:107E78000903B3FBFAF304FB0E3E97E7BDE8F08F66
:107E880010E000E0E4720020E8720020E0720020B8
:107E980000ED00E030B4EFF31183102282F3128872
:107EA8000649074C0A680748013200250A60256020
:107EB800DBB2026883F3118830BC7047E47200209B
:107EC800E072002010E000E00F4B1B88014643B928
:107ED8000E4B0F4A1B7810680BB981F00101FAF7B5
:107EE80085B80C4B5A691AB118B91A6810605874D9
:107EF8007047094A18681188084A92FBF1F2012173
:107F080002605974704700BFBC720020BE72002026
:107F1800C0720020C4720020DC72002020A107007B
:107F28001D4B70B59C68E36C226BDD69C2B1636B55
:107F38002BB12B0702D5E36C08221A6270BD2A0602
:107F4800F7D5A26A616A8A421FD0511CA069A16252
:107F5800825C2069E66C81423285EAD3A362E8E755
:107F6800A906E4D5E26A1AB1988C80B29047DEE798
:107F7800E1699B8C6069DBB24E1CE6614354E169A0
:107F8800E368994228BFE261D1E7E26C136823F005
:107F980080031360CDE700BFE03A00201D4B70B5A9
:107FA8005C68E36C226BDD69C2B1636B2BB12B0794
:107FB80002D5E36C08221A6270BD2A06F7D5A26AB8
:107FC800616A8A421FD0511CA069A162825C206943
:107FD800E66C81423285EAD3A362E8E7A906E4D5D4
:107FE800E26A1AB1988C80B29047DEE7E1699B8C0F
:107FF8006069DBB24E1CE6614354E169E36899426B
:1080080028BFE261D1E7E26C136823F080031360B4
:10801800CDE700BFE03A00201D4B70B51C68E36C4B
:10802800226BDD69C2B1636B2BB12B0702D5E36C00
:1080380008221A6270BD2A06F7D5A26A616A8A42C6
:108048001FD0511CA069A162825C2069E66C814244
:108058003285EAD3A362E8E7A906E4D5E26A1AB151
:10806800988C80B29047DEE7E1699B8C6069DBB24F
:108078004E1CE6614354E169E368994228BFE26116
:10808800D1E7E26C136823F080031360CDE700BFEB
:10809800E03A002070B4EFF31186502383F312887E
:1080A800436B1A68D20720D45D686DB9446A826A46
:1080B800944217D081691144D9600ED9A21A5A6026
:1080C8008462002280F850201A6842F00102F1B25E
:1080D8001A6081F3118870BC704701698A1A5A6066
:1080E8008562EEE7012380F85030F1B281F3118800
:1080F80070BC70472DE9F04F2DED028BD54B1B78E6
:1081080091B0072B069001F0148200230893D24CFB
:10811800D4F800B01BF4806F40F00587CF4B1B6884
:1081280007931F0700F1A986CD4BCE4DB3F80090F9
:10813800CD4CCE4BCE491E68B1F906807289904568
:1081480080F2AB81CB4B4FF07E521A60DFF834A33C
:1081580094F90820B1F900E0BAF81870207994F879
:1081680005C0AEEB0703002A14BF01224FF0FF320F
:10817800002BB8BF5B42B3F5FA7FA8BF4FF4FA7380
:108188009842059380F286811B1A07EE903AF8EE22
:10819800E77A7745C5ED007A03DDF1EE677AC5ED3C
:1081A800007AB1F902E0AEEB0703002BB8BF5B42DF
:1081B800B3F5FA7FA8BF4FF4FA739842059380F29B
:1081C8007F811B1A07EE903AF8EEE77A7745C5EDFE
:1081D800017A03DDF1EE677AC5ED017AB1F9041091
:1081E800CB1B83EAE370A0EBE370B0F5FA7FA8BF7E
:1081F8004FF4FA706045CCBFA0EB0C0C4FF0000CAC
:1082080002FB0CFC07EE90CAF8EEE77AB942C5ED1E
:10821800027ABCBFF1EE677AC5ED027A1BF480538F
:10822800059300F0F480B8F5FA6F4246A8BF4FF402
:10823800FA62B2F57A7F237BB8BF4FF47A72A2F55F
:108248007A72002B40F0FB808B49DFF83CE281FB1F
:108258000230D317C3EB6013581C6FF0630C3EF960
:1082680010003EF913E00CFB0323A0EB0E0003FB08
:1082780000F381FB0321DB17C3EB61139E440FFA64
:108288008EFE07EE90EA059BB8EEE78A85ED038A35
:10829800002B40F06F8519F04003099340F0AE843D
:1082A800079B13F0140F03D019F4027F40F04786A0
:1082B800724B1B7823B1BAF81A30434580F2818497
:1082C80094F83A701FB119F0030F40F03B8794F807
:1082D8004020002A40F07B859AF81E70002F00F09D
:1082E800F280022F00F02787032F40F00D879AF8BD
:1082F8002030C3EB431103EB8101C90089B29AF81E
:108308001F300233DBB2002A00F00787002900F093
:1083180004875B480768B1FBF7F10FB2A4F87070E7
:10832800ABB307EE907AF8EEE77AF7EE006A86EEDE
:10833800A77A012BD5ED007AD4ED216A77EEE67A9B
:1083480067EE877AC4ED1D7A21D0D5ED017AD4ED98
:10835800226A77EEE67A022B67EE877AC4ED1E7AF8
:1083680015D0D5ED027AD4ED236A77EEE67A032BA1
:1083780067EE877AC4ED1F7A09D0D5ED037AD4ED7C
:10838800246A77EEE67A67EE877AC4ED207A314977
:108398000978092901F07D84002F40F3998093B36F
:1083A80094ED217AD4ED1D7A77EE877A012BC4ED0E
:1083B800217AC5ED007A21D094ED227AD4ED1E7A87
:1083C80077EE877A022BC4ED227AC5ED017A15D0B3
:1083D80094ED237AD4ED1F7A77EE877A032BC4EDD8
:1083E800237AC5ED027A09D0D4ED247A94ED207A67
:1083F80077EE877AC4ED247AC5ED037A013B022B28
:10840800B8BF0223DBB2002A18BF022361E0BAF822
:108418001A209045C0F2D383B8F5FA6FD4BFC2EBE7
:108428000803C2F5FA634FF47A7101FB03F1207B6C
:10843800C2F5FA63B1FBF3F200283FF405AF637BA2
:108448000D4902FB03F281FB0213D217C2EB631240
:10845800FAE600BF2C490020987F0020E88A002017
:10846800BC3F0020803F00203C2400200C29002035
:10847800D06E00200C2700201F85EB514C000020F7
:10848800F08800205450002010290020000000002F
:108498000AD7233C5FED037A7BE6B8F5FA6FC0F2A2
:1084A8008283337AC3F1640307EE903A1FED087AAA
:1084B800CA4BF8EEE77A67EE877AC3ED007A45E6AD
:1084C800DFEDC77A82E6A4F87070002A00F06F81A9
:1084D80002233278DFEDC36AB17807EE902AF8EE0E
:1084E800E77AB0EE007A67EEA67ABF4AF4EEC77A6A
:1084F800F1EE10FA107840F30C84DFEDBC6A37EE29
:10850800C77AB0EE676AA7EE266AF0EE466A95ED7E
:10851800007A9FEDB76ADFF8FCE2DFF8FCC227EECD
:10852800066AF0EEC65ACEED005A8CED006A99B193
:1085380007EE101AB8EEC75A9FEDAA7A66EE064AF9
:1085480025EE075AB7EE007A37EE457A64EEA54A6B
:10855800A5EE247A26EE076A9FEDA67A727926EEB2
:10856800877A27EE067AAAB1DFED9E6A9FEDA26AA6
:1085780065EEA65A06EE902AF8EEE66A66EEA56A59
:10858800F4EEC66AF1EE10FA40F38E859FED9B6A11
:1085980027EE067A0C289FED9A8ADFED9A6ADFF8B3
:1085A8007C8200F05C85B4EEC87AF1EE10FA98BFD0
:1085B800B0EE478AB4EEE68AF1EE10FAB8BFB0EE34
:1085C800668A88ED008A002B00F0E680B0EE007A1B
:1085D800F4EEC77AF1EE10FA05DD37EEC77ADFED73
:1085E800836AE7EE267A95ED017ADFED816A27EE58
:1085F800267AF0EEC75A8CED017ACEED015A99B180
:1086080006EE901A9FED776AF8EEE66A27EE075AAB
:1086180066EE866AB7EE006A36EE666A25EE255A79
:10862800A6EE856A27EE067ADFED726AB27967EE02
:10863800A67A67EE877AFAB107EE102AB8EEC77AFB
:108648009FED686ADFED6C6A27EE257A27EE067AD9
:10865800B4EEE67AF1EE10FA00F32285B5EEC07AB0
:10866800F1EE10FA00F1A087B7EE006A36EE477A0D
:10867800C6EE076A67EEA67A0C2800F0D184DFED13
:10868800606A9FED607AF4EEE67AF1EE10FA88BF40
:10869800F0EE667AF4EEC77AF1EE10FAB8BFF0EEB3
:1086A800477A012BC8ED017A76DD7378DFED4D6AE4
:1086B80007EE903AF8EEE77AB0EE007A67EEA67A1F
:1086C800737AF4EEC77AF1EE10FA05DD37EEC77A61
:1086D800DFED466AE7EE267A95ED027ADFED446A29
:1086E80027EE267AF0EEC75A8CED027ACEED025AC2
:1086F8009BB106EE903A9FED3B6AF8EEE66A27EEEC
:10870800075A66EE866AB7EE006A36EE666A25EEA6
:10871800255AA6EE856A27EE067ADFED366AF379E2
:1087280067EEA67A67EE877AFBB107EE103AB8EEE5
:10873800C77A9FED2C6ADFED306A27EE257A27EE9F
:10874800067AB4EEE67AF1EE10FA00F3A584B5EEF7
:10875800C07AF1EE10FA00F12387B7EE006A36EE20
:10876800477AC6EE076A67EEA67A0C2800F05084AE
:10877800DFED236A9FED237AF4EEE67AF1EE10FA44
:1087880088BFF0EE667AF4EEC77AF1EE10FAB8BF59
:10879800F0EE477AC8ED027A092800F030849AF89A
:1087A8002150002D40F0E683002384F84030164D18
:1087B800164F95F82420164E05F14009531E082B34
:1087C80000F20781DFE813F023014C01A90005013D
:1087D8005A002C009D010501880100BF0C270020CC
:1087E800000000000AD7233C2C490020D7A3684189
:1087F8006F12033B00004843A4707D3F0000C8424D
:1088080000C0F94400C0F9C4D8820020E4720020F6
:10881800D4820020382700202C270020142700208D
:108828002B68287A4FF4807203EB002000211EF099
:1088380053FA2B7A0133DBB2022B2B7240F0D7812B
:1088480000201EF08BFA00201EF088FAFF201EF090
:1088580085FA00F01F00052801F063821BF0ECFE8A
:10886800D5F80C80B8F1000F00F0C58100222B6903
:1088780069680120C04795F824209FE74FF40071EC
:10888800286818F0C1F8012800F0A484C0F03D86DB
:10889800022840F0AC811BF007FF1BF0CDFED5F895
:1088A8000C80B8F1000F00F0A681002210462B6959
:1088B8006968C04795F8242080E71021484618F0D9
:1088C800A3F88346002840F0F48001217F201DF0A2
:1088D80087FD0128804640F0EC80584602211DF0B3
:1088E8007FFD002801F0C680012840F0E2801621B3
:1088F8003A201DF075FD431C9B02AB621BF0D4FEB1
:108908003068F9F769FB00210A2018F09BF8002865
:1089180040F08584032385F8243010210CA818F032
:1089280073F8002840F063819DF83A209DF83900DB
:108938009DF83C109DF83D309DF83BE0120442EA5A
:1089480000620A431B019DF83E109DF83100DBB21E
:1089580043EA111342EA0E2203F5FA636A636B874E
:108968009DF832209DF8383042EA002201F00F01CC
:10897800180903F00F0385F83C10AA859DF83010FC
:108988009DF8332085F839309DF8343085F82E105D
:1089980085F82F209DF835109DF8362085F8303061
:1089A8009DF8373085F8333085F8380085F8311070
:1089B80085F832201BF078FEAB7E002B00F0E380B8
:1089C800D6481EF0A9FA002304222B6285F8242039
:1089D8000323DBB2022B74D9042A00F0AE80082AE4
:1089E80000F0AB80CE4B1B7823B9CE4EB378002B6A
:1089F80040F0DD8306980DF033FACB4B1B78072B3C
:108A080000F0DF8411B0BDEC028BBDE8F08F306858
:108A1800F9F7E2FA0021084618F014F880461BF02E
:108A280043FEB8F1010F40F0E28030684FF0000BD0
:108A380085F819B0F9F7D0FA40F2AB11082018F010
:108A480001F8052800F0D283012800F077851BF093
:108A58002BFE6B7E002B01F07581022385F82430F4
:108A68003068F9F7B9FA6B7E022B14BF4FF0000893
:108A78004FF080480021372017F0E4FF41462920B5
:108A880017F0E0FF80461BF00FFEB8F1000F40F032
:108A9800AE806B7E022B00F0B28385F81A803068B6
:108AA800F9F79AFA0021092017F0CCFF00283FF4C3
:108AB80004AF1BF0F9FD95F82420531EDBB2022BFE
:108AC8008AD89A4B69691B685B1AC82B87D91BF02F
:108AD800B3FD95F824207FE74FF00808FF201EF02B
:108AE8003DF9FF2800F07884B8F10108F6D16B69E8
:108AF8003A68FA3393427AD21BF09EFD95F8242007
:108B08005CE6FF201EF02AF9FF284FF0080807D07E
:108B1800B8F10108EBD0FF201EF020F9FF28F7D1AB
:108B28002B6A0022012B2A765AD9EA69013B0132C5
:108B38002B620823EA6185F824307D4D19F04AF844
:108B48006B78022B00F05484032B7FF44BAF41F277
:108B5800B813EB5C002B40F0A98741F2A403EB5C4F
:108B6800002B40F0AD8741F2E803EB5C002B40F0AE
:108B7800A28741F22C13EB5C002B3FF433AF6D4816
:108B880020F0ECFC2EE73068F9F726FA4FF4007174
:108B9800102017F057FF80461BF086FDB8F1000F34
:108BA8003FF40EAFA8E7307AA8EB020303FB00F30B
:108BB800C2F5FA6293FBF2F3C3F1640374E4194655
:108BC80035E45D4B1B78012B00F05E83192B00F018
:108BD8005B830E2B3FF474AB082B3FF471AB58E367
:108BE80001F0E083042385F824301BF05DFD95F83F
:108BF8002420531EEDE695F82420DFE54F4B50491D
:108C0800B3F90430A28ADFED4F6A9FED4F7A81FBFA
:108C18000301DB17C3EBA1039B1A1BB207EE903AC3
:108C2800F8EEE77A67EEA67A77EE876ABDEEE66A2F
:108C380016EE103A2033402B40F22084DFED436AD1
:108C4800BDEEE77A17EE103A2033402B00F2E083AE
:108C58009FED3F7AF4EEC77AF1EE10FA40F34487BD
:108C6800DFED3C5A9FED3C6A01E0F0EE477AF4EE06
:108C7800C67AF1EE10FA37EEE57AF6DCDFED377AF0
:108C8800B4EEE77AF1EE10FA40F13287DFED315AAF
:108C98009FED336A01E0B0EE677AB4EEC67AF1EE82
:108CA80010FA77EE257AF6D49FED277AF4EEC77A94
:108CB800F1EE10FA00F395829FED2A7AF4EEC77A66
:108CC800F1EE10FA44BF9FED257A77EE677A67EEEA
:108CD800A75A9FED255A9FED256A9FED257AA5EEA7
:108CE800856A27EEA55AA5EE867AE5EE077A95ED10
:108CF800016AD5ED005A27EEC67A65EEA77AA5EE89
:108D0800A67AE6EE267A85ED007AC5ED017AFFF7B8
:108D1800C7BAF0EE676AFFF7FABB00BF0038004039
:108D28003A430020A48A00202C490020E472002045
:108D3800F8580020246A002008890020CC3F002031
:108D48006766666635FA8E3CDB0FC93F0000000097
:108D5800DB0F4940DB0FC940E4CB1641DB0F49C0AC
:108D6800E4CB16C1DB0FC9BF92E741B99730083C85
:108D780015A82ABE1D21D048FAF757F800283FF455
:108D88008AAACE4BDB78002B7FF485AADFEDCC7A5C
:108D9800CC4938EE678AC7F5FA63FDEEC87A1BB28C
:108DA800CDED097ABDF92420120381FB0201D21707
:108DB800C2EBA11203FB02F343F30F333B4407EE6C
:108DC800903AF8EEE77AC5ED037AFFF764BABE4940
:108DD800B94BD1F8EC101B6844F620608142A8BF5B
:108DE8000146B1F57A7FB8BF4FF47A7189B2D806D7
:108DF800A4F8421040F1FD81059B002B40F0D88378
:108E0800B24BD3F800E0BEF93270AE48636CD5EDD2
:108E1800037AA0FB01018809642191FBF0F1142970
:108E2800BDEEE77A04EB430CA8BF142101338B4253
:108E3800636417EE108AA4BF0023636404EB430342
:108E4800ACF84880B3F9483007EE103AB8EEC77A64
:108E580077EEC77AFDEEE77ACDED057ABDF9141005
:108E680081EAE173A3EBE173BB4200F32E86984BD2
:108E78004FF07E511960FFF72FBA964D964BD5EDFE
:108E8800027AB3F80090954B954AB3F90430954CA3
:108E9800B2EE0E7AF0EEE76AF4EEC76AF1EE10FA77
:108EA80082FB03124FEAE37338D519F0040F35D06B
:108EB8002188C3EBA2035B1A9BB21AB212F1B30F5B
:108EC800BCBF03F5B4731AB2B32AC8BFA2F5B47312
:108ED8008549C8BF1AB2237A0978002B4FF6FF7369
:108EE80018BF01230E077FF524A97849096812FBEA
:108EF80003F30A7E7D499BB212FB03F381FB031245
:108F08001A44DB17C3EB221307EE103AB8EEC77A00
:108F180077EEC77AC5ED027AFFF70BB9C3EBA20368
:108F28002380FFF706B972488368002B3FF4F6A840
:108F380000F150019847D4F800B0FFF7EFB86A4B3A
:108F48001B7813F0100300F07281227EE36995ED1F
:108F5800017A002A0CBF01224FF0FF3203FB02F313
:108F680007EE903AF8EEE77A77EE877AC5ED017A60
:108F7800FFF79EB91E215048F9F757FF00283FF424
:108F880013AC099B002B7FF40FAC94F89430AB42E0
:108F980040F0DC85574BD4ED267AD3ED006A98ED86
:108FA800025ADFED555A9FED556A27EEC57A68EEED
:108FB800277AA8EE267AE5EE267AB4EEE57AF1EE7F
:108FC80010FA88BFB0EE657AB4EEC67AF1EE10FA00
:108FD800F4EEE57AB8BFB0EE467AF1EE10FA88BF43
:108FE800F0EE657AF4EEC67AF1EE10FAB8BFF0EE5C
:108FF800467A88ED007AC8ED027AFFF7D5BBFDEE18
:10900800C87A3F4A17EE903A9780D380FFF7C7BBDC
:10901800BDEEE77A3A4B17EE102A9A80FFF7A8BB05
:109028009FED357ADFED356A3549F4EEC77AF1EE12
:1090380010FA98BFB0EE677AFDEEE77AB4EEE67AFA
:10904800F1EE10FA17EE902AB8BFB0EE667A012B4F
:1090580088ED017A4A803FF728ABFFF7A0BBB4EE52
:10906800C87AF1EE10FA98BFB0EE478ABDEEC77A1B
:10907800B4EEE68ADFF88890F1EE10FA17EE102ABF
:10908800B8BFB0EE668A88ED008AA9F80020002BE8
:109098007FF49CAAFFF783BBDFED1A6AFFF763BB77
:1090A800DFED186AFFF7E6BAF7EE005A75EEE66AE2
:1090B80085EEA66AFFF76CBAE08A00200C4800200B
:1090C80000007A44D34D621050000020EC3F00208D
:1090D80040000020803F0020BC3F0020CC3F002003
:1090E800676666663C240020908A00208988888804
:1090F800287000202400002000C0F94400C0F9C4F2
:10910800304900200000C842C34B59889AF81F30E4
:109118000233DBB2002A7FF4F9A8B4F87070013F7B
:109128003FB2002FA4F870703FF739A9002A7FF4E6
:10913800CFA9FFF73CBBB4F8421001F57A7189B2A8
:10914800FFF7DDB8B54BDFEDB67A93ED080AB4EE5C
:10915800E70AF1EE10FA40F20A822AF023F8D4ED79
:109168000F7A20EE270A29F087FFB0F5617F00F318
:10917800268207EE900AF8EEE76ADFEDAA7A66EE35
:10918800A76A07EE907AB8EEE77AFDEEE67A17EE70
:10919800903A2033402B40F21D869FEDB70A29F004
:1091A8006BFF00B207EE900AB8EEE77AE1E19E4F56
:1091B8003A78013A0A2A00F2C880DFE812F0800201
:1091C800720266024C02C600C6003802C702A50237
:1091D8008F0279006B693A6864339342FFF45BABA2
:1091E80005E59FED9F7A77EE677A70E585F8198037
:1091F8002DE41BF0805F7FF4FFADFFF76DB830689A
:10920800F8F7EAFE41463A2017F01CFC0422834690
:109218000CA940461DF060FDBBF1000F3FD01BF0CC
:1092280043FA1BF009FA95F82420FFF7C7BAE27948
:10923800002A40F0DD81B4F92070A179A8EB07037A
:1092480083EAE370A0EBE370884240F3558403EBB4
:10925800D37301225B10236384F8342084F8282018
:10926800E3691F44B7F5FA6FA8BF4FF4FA67B7F57B
:109278007A7FB8BF4FF47A7707EE907AF8EEE77AFC
:10928800C5ED037AFFF714B8684B9B7B002B7FF47E
:1092980017A8674A0023AB609360FFF711B81BF06B
:1092A80003FA0C9B1BBAC3F38073AB76FFF7F7BBCB
:1092B800022B38D15F4BDFF894A11B78002B40F0CC
:1092C800C087DAF8005045B32B7833B395F82820D7
:1092D800002A40F056812B7EAA6385F83C200422A0
:1092E80085F8282013F008036A6AEA622A6303D023
:1092F800514A41F29413D3586B634FF00008C5F8F4
:109308002480C5F80880C5F80C8028461DF024F88C
:109318000523C5F8408085F8283000220423CAF8C0
:1093280000208AF81430454B454A5B681268C833F8
:10933800934204D313F0DAFE002800F0B081B3782A
:10934800032B01F0198001223A70022B00F01981D9
:10935800F278002A3FF44EAB3A4A1278D20706D484
:10936800059311F017F8059B002840F0B484344D9C
:10937800D4F8A4102A68914200F2B4843B78012BF7
:109388003FF438AB94F8A020002A3FF433AB0B2B02
:109398000DD801229A4040F6030112EA01060BD1CA
:1093A80012F4C06F03D0093B012B41F25E80234BBE
:1093B8002A685A600B233B70002384F8A030FFF71B
:1093C80019BBFEF723FC089A1F4B801A988011B02E
:1093D800BDEC028BBDE8F08F1BF066F9042385F81D
:1093E8002430154D18F0F6FB6B78022B7FF4ACABEC
:1093F800AB784FF00109072B3FF6F4AADFE813F02A
:10940800E20216030A03FF027C0266027002FB02F4
:10941800DFED197A6BE400BF4C48002018300020BB
:109428008FC2753CD06D393AC13C00208479002048
:1094380014270020D4880020F8580020E488002051
:10944800E4720020C04F002030490020AC8A002080
:10945800E4CB1641DB0FC940E4CB16C1DB0FC93F93
:10946800DB0F494092E741B99730083C15A82ABE5E
:10947800DB0FC9BFDB0F49C000000000F4EEC77A5C
:10948800F1EE10FA40F345845FED0E5A1FED106AB5
:1094980001E0F0EE476AF4EEC66AF1EE10FA36EE35
:1094A800E57AF6DC5FED0D6AB4EEE67AF1EE10FAD5
:1094B80040F12B845FED195A1FED196A01E0B0EEF7
:1094C800667AB4EEC67AF1EE10FA77EE256AF6D42B
:1094D8001FED1E7AF4EEC76AF1EE10FA3BDD1FEDC0
:1094E800207A77EE666A66EEA65A1FED225A1FEDBD
:1094F800226A1FED227AA5EE856A26EEA55AA5EE08
:10950800867AE5EE076AFFF79BBB1BF0CDF8EE689D
:109518000423002085F824302876002E3FF40DAB74
:109528002B692A686968B04795F82420531EFFF70D
:1095380050BAFEF76BFB0890FEF7E9BD58460422C7
:109548000CA91DF0C9FB9DF83330AB2B04BF0223D7
:109558006B76FFF77CBA1FED3A7AF4EEC76AF1EE44
:1095680010FA44BF1FED3D7A77EE666ABBE71FED40
:109578003E7AD5ED037A77EE877AC5ED037AFEF762
:10958800A6BEA74A41F2B513D35C002B00F028878A
:1095980094F8A03001223A70002B3FF42BAA0BE775
:1095A800F7EE006AFFF7DFB8F7EE006AFFF762B878
:1095B8009C4BD3F800E0BEF832707F0825E407EE34
:1095C800907ADFED996AB8EEE77A66EEA65A9FEDD3
:1095D800975A9FED976ADFED977AA5EE856A26EE92
:1095E800A55AE5EE867AE5EE276A26EE870AD6E5DD
:1095F800B4F92020A179A8EB020787EAE770A0EB6D
:10960800E770884240F386829045C8BF494207EE1A
:10961800901A95ED037A6362F8EEE77A012077EE07
:10962800277A84F82800C5ED037AFEF741BE13F0C7
:109638001FFD814B002105208DE80300A3F10802DE
:109648000291532023F0F6FB48BB7C4AB3781060A4
:1096580008223A7079E613F00BFD794A0292A2F1DA
:109668000C03292101930091A2F10A035021163A13
:10967800492023F0DFFB90B9704AB37810604FF0AF
:10968800FF31516007223A705FE66C4D13F0F0FC31
:109698006C4A6B68126864339342C0F08D85B37866
:1096A80053E6022B00F03284664A644912684A6025
:1096B800654800220A6003210260397045E6634A62
:1096C8001278D2077FF541AE80201CF0E3FB08B189
:1096D8000DF066F823F078FCB37836E65C4B1B781F
:1096E800002B00F01A831A200AF024FB002840F00F
:1096F800148394F8A030002B40F00F8309233B70AB
:1097080023F062FBB37820E61A200AF013FB002846
:10971800F6D0504B1B88002BF2D14F4B45201D68CB
:1097280013F026FD0E2013F023FD284622F054FFE7
:10973800069D284622F050FF484A494B12681A6095
:1097480028460A233B7023F04FF8D9E713F090FC22
:10975800444B93ED000A29F08FFC434B93ED000A2C
:10976800804629F089FC8146402013F063FC0028DC
:1097780095D1324D3D4A2B6892F801E04C2B00F20E
:109788004685DFE813F0DD06EA06E30673076D0792
:109798006507F506B607AF07A807A10791078A0767
:1097A8008307790768085A0853084C0845083A0897
:1097B8002F08240819080E080308F807ED07DC0726
:1097C800CC07BC07150A050AF509E509D509C50935
:1097D800BD09AD09A4099C0994098C0984097B0970
:1097E8007209690961095909500947093F09370987
:1097F8002F092709AD08A708A008990892088A0820
:1098080082086F08D006C906C206BB06B406AD06B4
:10981800A6069F06980691068A0683064B063F060B
:10982800F8580020EC3F002084F9223F92E741B924
:109838009730083C15A82ABEA0570308E4880020E2
:10984800C2550308E4720020783D0020C04F002074
:109858005C890020608700205C87002050870020FA
:109868004C8700207487002064320020F03F0020DD
:109878002B690622652BAA7032D92A78032A14BFCD
:109888006FF0FF026FF07F02A3F1650303EA0203A2
:1098980003F1010314BF4FF4807280229A422B61B6
:1098A8001ED23268EE6802329F19974280F05F85B7
:1098B800C94A6E60D16FAF60490203FB01F305210D
:1098C800166042F81C3C42F8183CA970AA68C349C3
:1098D800012017F055FB012840F03F850623AB70A7
:1098E8000021BF4817F08AFA012840F03685AB7886
:1098F8000133DBB2AB707EE52A782B7DB94EDFF8F9
:10990800DC82032A14BF4FF480778027002B44D0D1
:10991800012BFBD1B44B6A681968306800234FEA01
:10992800412E4FF0FF31B1FBFEF112EB010B43F179
:10993800000C0021614500F1020008BF584538BFFE
:1099480083465A46A949022017F04CFC032800F226
:10995800FD8101A353F820F0ED89000871990008F2
:10996800ED890008719900086968D5F808E02B6945
:10997800AEEB01029A4284BFE9602A6103283FF4F2
:1099880077AF0EF10103B3FBF7F207FB12320AB10E
:109998003B449B1A00226B602A75326841460232AA
:1099A800002017F01FFC032800F2D08101A353F810
:1099B80020F000BFED890008719A0008ED890008C1
:1099C8007998000800230DF130084146184609220D
:1099D80017F068F801287FF405A80C9B93F8FE217E
:1099E800552A00F0B58141F2B41202210123A9548D
:1099F8006B70FEF7F7BF03236B70FEF7F3BF41F2FE
:109A08007013EB5C002B3EF4EDAF75481FF0A6FD1C
:109A1800FEF7E8BF764B00930320A8703023052299
:109A280074496F4818F044F8FEF7DCBF0DF13008B0
:109A380041F2FC164146A8590023092217F032F8D2
:109A480001287EF4CFAF00230C9A2B70B2F80B30AC
:109A5800B3F5007F00F0208441F2B4120321012302
:109A6800A9546B70FEF7BEBF6B6885F8149001337C
:109A7800AB604FE704212C201CF0B2FC0321834685
:109A88004E201CF0ADFC0C21059036201CF0A8FCE3
:109A9800059B421C02339A4008FA0BF8A2FB080106
:109AA800420A42EAC152AA62FEF728BF52481FF092
:109AB80055FDFFF752B851481FF050FDFFF759B850
:109AC8004F481FF04BFDFFF74EB8BEF834309FEDFE
:109AD8004D7A07EE903AF8EEE77A4B4B67EE877AC5
:109AE800C3ED007AFEF7F8BBB0EE677AFFF7C6B8A9
:109AF800F0EE477AFFF7D8B894F82830002B3FF4F7
:109B0800AFAB424B84F834201B6884F82820E3620A
:109B1800FFF7A6BB94F8281021B13C4984F82830F7
:109B28000B68E362E3691344B3F5FA6FA8BF4FF417
:109B3800FA63B3F57A7FB8BF4FF47A7307EE903AB9
:109B4800F8EEE77AC5ED037AFEF7B2BB07EE905A56
:109B5800DFED2F6A9FED357A84F89450F8EEE77AB6
:109B680067EEA67A77EE876ABDEEE66A16EE103AD9
:109B78002033402B40F27481DFED266A264BBDEE80
:109B8800E77AC3ED006A17EE103A2033402B00F253
:109B9800AE819FED277AF4EEC77AF1EE10FA40F322
:109BA800FE83DFED1E5A9FED1E6A01E0F0EE477A54
:109BB800F4EEC67AF1EE10FA37EEE57AF6DCDFED70
:109BC800197AB4EEE77AF1EE10FA40F1E583DFEDA9
:109BD800135A9FED156A35E08C6A0020FC58002066
:109BE800686A0020006B0020086B002000590020E4
:109BF800E1060208C0810308B06A0020E06900207D
:109C08009C6900206F12833A40000020C88A002017
:109C180035FA8E3C0000000024000020DB0FC9400C
:109C2800E4CB1641DB0F49C0E4CB16C1DB0FC93FBB
:109C3800DB0F494092E741B99730083C15A82ABE86
:109C4800B0EE677AB4EEC67AF1EE10FA77EE257ABE
:109C5800F6D41FED0A7AF4EEC77AF1EE10FA40F363
:109C680049811FED0D7A77EE677A67EEA75A1FEDE7
:109C78000F5A1FED0F6A1FED0F7AA5EE856A27EEC2
:109C8800A55AA5EE867AE5EE077AC4ED267AFFF79F
:109C980086B995ED000A0793059229F0EDF9A649D2
:109CA800DFF8C8E2D1F8EC10DFF8C4C2059AACF8C6
:109CB80000008EFB013EC917C1EBAE1107EE901AEA
:109CC800F8EEE77A079BFDEEE77A17EE901AACF804
:109CD8000210FEF761BB994A126802F59C520832DD
:109CE800C4F8A4203A78012A7EF484AE94F8A0201F
:109CF800002A7EF47FAE032B00F0758323F064F90D
:109D0800012384F8A030FEF775BEF0EE476AFFF72E
:109D1800DFBBB0EE667AFFF7C5BB069822F064FD9C
:109D2800EEE4864BEE681B686B61072385F82430E8
:109D3800002E3EF457AE2B692A6869680120B047A7
:109D4800FEF755BF85F82430FEF74CBE2B7DDDE5C8
:109D580093F8FF21AA2A7FF446AED3F8C61149B179
:109D680093F8C221A2F10B0001282DD902F0F702C5
:109D7800062A29D0D3F8D61149B193F8D221A2F1F5
:109D88000B00012820D902F0F702062A1CD0D3F8CC
:109D9800E61149B193F8E221A2F10B00012813D989
:109DA80002F0F702062A0FD0D3F8F61100293FF483
:109DB8001AAE93F8F231A3F10B02012A04D903F089
:109DC800F703062B7FF40FAE41F2FC120123A950D2
:109DD800AB702DE6DFED5A7AF4EEE76AF1EE10FA91
:109DE80040F35183DFED575A9FED576A01E0F0EEDB
:109DF800676AF4EEC66AF1EE10FA76EEE57AF6DCFA
:109E0800DFED526AF4EEE67AF1EE10FA40F10C83D7
:109E1800DFED4C5A9FED4E6A01E0F0EE667AF4EE03
:109E2800C67AF1EE10FA77EEA56AF6D4DFED497A34
:109E3800F4EEE76AF1EE10FA05DDDFED417A77EE30
:109E4800E66AFFF7C2BBDFED447AF4EEE76AF1EEAB
:109E580010FA44BFDFED3D7A77EEE66AFFF7B5BB4F
:109E6800F4EEC77AF1EE10FA40F3B782DFED355A17
:109E78009FED356A01E0F0EE476AF4EEC66AF1EE4E
:109E880010FA36EEE57AF6DCDFED306AB4EEE67A03
:109E9800F1EE10FA40F17D82DFED2A5A9FED2C6A2F
:109EA80001E0B0EE667AB4EEC67AF1EE10FA77EE1B
:109EB800256AF6D49FED277AF4EEC76AF1EE10FA18
:109EC80040F3B3819FED1E7A77EE666A66EEA65A76
:109ED8009FED225A9FED226A9FED227AA5EE856AB0
:109EE80026EEA55AA5EE867AE5EE076A46E6DFED88
:109EF8001E7ACAE69FED187AF4EEC77AF1EE10FAE8
:109F080044BF9FED127A77EE677AAEE6DFF864A079
:109F18009AF81430052B3FF6C2AB01A252F823F091
:109F28000DA10008A79600084BA10008D39F0008C0
:109F380009A0000807A1000850000020E4720020D2
:109F4800DB0F4940DB0FC940E4CB1641DB0F49C0AA
:109F5800E4CB16C1DB0FC93FDB0FC9BF92E741B99C
:109F68009730083C15A82ABE00000000D34D6210A7
:109F780030490020AC8A0020DAF8041091F91A2040
:109F8800551C5C460AD0B44B02F5817203EB0213F0
:109F9800FF20DA796FF30002DA71887691F91B30C5
:109FA800581C0FD0AC4803F5817300EB0310FF2554
:109FB800C379C3F34502013A22EAE27262F3460327
:109FC800C371CD7603238AF81430A448DAF8041054
:109FD8000378002B7FF463AB002900F0288291F806
:109FE8002830002B7FF45BAB2838442228F03AFE57
:109FF8000021DAF8040016F0A9FF0023CAF804309B
:10A00800DAF81050DFF87492DFF874E2DFF874C2FF
:10A01800934B05F1010BA9FB0B58ACFB0B5CAEFB9A
:10A028000BE507958F4DA5FB0BE50995079D0FCB14
:10A03800AD090795099D4FEAD80E4FEA5C1C6D0BD8
:10A048000DF13008CDF814C00995A9FB0EC5C4461A
:10A05800ACE80700059A07988CF80030A9FB0221A4
:10A06800ED08A9FB00020998079B05EB8505A9FBEC
:10A078000009C908AEEB4500D208059D0EEB8E0E0F
:10A0880001EB810102EB8202A5EB4101ABEB4E0B28
:10A09800A3EB420241F2A40E099B6F4D4FEAD90986
:10A0A80009EB8909A3EB490915F80E30303001F1A5
:10A0B800300E0BF1300B303209F1300901218DF8E7
:10A0C80036008DF837B08DF835E08DF834208DF8EE
:10A0D80033908AF81410002B00F06F8141F2E803E6
:10A0E800EB5C002B00F0688141F22C13EB5C002B39
:10A0F80000F0A48104238AF81430FFF7D0BAB378AB
:10A10800FFF7D2BA544D6B78032B7FF4C8AA41F2FB
:10A11800A4020123AA5C8AF81430002A00F0A08166
:10A1280041F2E802AA5C002A00F08B8141F22C136C
:10A13800EB5C002B00F0848100238AF81430FFF7D1
:10A14800AEBADFF84491DFF84481474DA3460BAA25
:10A158004946DAF8040016F0E5FD012841464FF0BB
:10A16800030240F026810B9C2046002C3FF404AFEC
:10A178002378002B3FF400AF2BF0FDF8032229468B
:10A188000028E4D104F108002BF0F5F80346002874
:10A19800DDD154F8030F0C9022798DF834200CA8E7
:10A1A8008DF8353028F036FDDAF81030834238BFA4
:10A1B8000346CAF81030CAE7402012F03BFF0028D7
:10A1C8007FF46DAA2B68DFF8C880DFF8C8A04FF0CD
:10A1D80040090DE012F0CCFFDAF800202B68013AB4
:10A1E8000133B9F10109CAF800202B6000F0A281FF
:10A1F80018F803301846002BECD100234FF0FF323B
:10A208002B6004233B706A60B378FFF79EB812F0A6
:10A218006DFF00283FF443AA144A154B12681A60D0
:10A228000A233B70B378FFF790B89FED127AF4EEEB
:10A23800C76AF1EE10FA44BF9FED0F7A77EE666AAF
:10A2480044E60021DAF8000016F080FE00287FF4CA
:10A2580064A8FFF724BA00BFF8580020D86A002085
:10A26800CC8603085917B7D1D88103085087002036
:10A278004C870020DB0FC9BFDB0F49C0CDCCCCCC4D
:10A28800D34D62101F85EB51B48A0020D481030896
:10A298005C550308783D0020137C022B7FF4DCAB6F
:10A2A80092F8FE31552B7FF4D7AB92F8FF31AA2BE9
:10A2B8007FF4D2ABB2F80EE0AF59B64B77441F60CB
:10A2C800567B41F21021731E7F2B6E503FF6C4ABB4
:10A2D800734236EA03037FF4BFAB730241F21821DD
:10A2E800013B6B50D08A00B9506AAB4941F2042354
:10A2F800E850B2F811305B0103F2FF135B120B60F8
:10A30800B2F8131001B9116A0EEB030C4000844433
:10A31800A1EB0C0141F2082E40F6F47CB1FBF6F1FA
:10A32800614545F80E1069D94FF6F476B14261D906
:10A3380003212970D26A99493B44184441F20C26FA
:10A3480041F21C230978A851EA5009B91FF0D8F83E
:10A35800AB780133AB70FEF745BB02287EF442AB05
:10A3680041F2B4120123AB546B70FEF73BBB16F0FD
:10A37800D1F92B69FFF79CBA894D28680CF0E4F9EC
:10A38800884B1B780022022B2A606BD0B378FEF72B
:10A39800DABFF0EE476A8DE5F0EE477A59E4B0EEA1
:10A3A800677A0CE416F00CFB02287EF420ACFEF76A
:10A3B8001CBC5C46FFF773B90B4603EB031305EBB4
:10A3C800830000F58550784B009341463C232022BA
:10A3D800043017F06DFBFFF762B9B0EE667A53E50B
:10A3E8000223FEF7B5BF80201BF054FD00287EF441
:10A3F80001AB83E402222A7000229CE701232B7020
:10A40800FFF72ABB694B6A491A686A4822F062F961
:10A418002A68B37801322A60FEF797BF92786449B8
:10A42800654822F057F9F3E7F0EE676AFEE41FF09B
:10A4380067F800287FF4DCADFFF731B90223BCE7E9
:10A448000223442202FB035303F585505B4B009320
:10A45800102213235A49043017F02AFBFFF71FB9BB
:10A468001346EEE70CF01CFE90E7452012F080FE44
:10A47800FF2012F07DFE534812F04CFE304612F0D9
:10A4880077FEFEF794BFF0EE667AB9E44E4B484982
:10A49800DA894E4822F01EF9BAE74B4B44491A882C
:10A4A8004B4822F017F9B3E7474B41499A78494896
:10A4B80022F010F9ACE7444B3D491A79464822F09E
:10A4C80009F9A5E79AF808203949444822F002F921
:10A4D8009EE7BAF822203649414822F0FBF897E770
:10A4E8009AF8202032493F4822F0F4F890E79AF889
:10A4F8001E202F493C4822F0EDF889E73B4B2C49B8
:10A508001A783B4822F0E6F882E73A4B2849DA788D
:10A51800394822F0DFF87BE7384B25495A79384823
:10A5280022F0D8F874E7374B2149DA78364822F018
:10A53800D1F86DE718F80330002B7FF4B0A85CE67B
:10A54800324A3349334822F0C5F861E7324B334A7F
:10A558003349344822F0BEF85AE7334A334B019264
:10A568000093334A334B3449344822F0B3F84FE769
:10A5780022F024F9324A334BB2F900108046B3F97D
:10A588000000F8F7E7FB4246C3B22F492F4822F0F4
:10A59800A1F83DE7F86A0020186B0020D86A00206F
:10A5A8007C3D0020ED88002001C30108D43C002038
:10A5B80074820308B4860308A8860308F5CF010847
:10A5C800CC810308C0860308447C002094860308D5
:10A5D80084860308708603085C8603084886030897
:10A5E8002C86030810860308FC8503083029002000
:10A5F800E485030878890020D4850308308C00207E
:10A60800C48503081C790020B4850308DC8103088D
:10A61800E8810308EC810308A88103089C810308EA
:10A628003C8203084482030834820308B481030887
:10A6380004820308FC8103081082030820820308AF
:10A648006887002066870020848203088C820308BC
:10A65800A64BA749B3F90020A64822F03BF8D7E655
:10A66800A54AA649A64822F035F8D1E6A54AA34945
:10A67800A54822F02FF8CBE6A448A549837842786C
:10A6880000780090A34822F025F8C1E6A24B1B6889
:10A69800D90412D40F232B60BAE6A04BA0499A8A9A
:10A6A800A04822F017F8B3E61FFA89F31FFA88F2D8
:10A6B8009D499E4822F00EF8AAE69D4B98491A78C3
:10A6C8009C4822F007F8A3E64FF07E529A499B482F
:10A6D80022F000F89CE69A4B85495A8A994821F05D
:10A6E800F9FF95E6964B82491A8A974821F0F2FFBE
:10A6F8008EE632887E49954821F0ECFF88E6944B37
:10A708009449D3F800E094489EF804309EF803205A
:10A718009EF805E0CDF800E021F0DCFF78E68C4BF0
:10A728008C49D3F800E08D489EF801309EF800204F
:10A738009EF802E0CDF800E021F0CCFF68E6884BF7
:10A74800844988480C2202FB0E3E9EF806309EF88B
:10A7580005209EF807E0CDF800E021F0BBFF57E6A2
:10A768007F4A634980480C2303FB0E2EBEF80A205B
:10A7780021F0B0FF4CE67A4A5D497C480C2303FB84
:10A788000E2E9EF8082021F0A5FF41E6744A58498C
:10A7980077480C2303FB0E2E9EF8042021F09AFF25
:10A7A80036E66F4A524973480C2303FB0E2E9EF877
:10A7B800032021F08FFF2BE6694A4D496E480C2390
:10A7C80003FB0E2E9EF8092021F084FF20E6644A40
:10A7D80047496A480C2303FB0E2E9EF8012021F0FE
:10A7E80079FF15E65E4A424965480C2303FB0E2EA5
:10A7F8009EF8022021F06EFF0AE60C2303FB0EFEF2
:10A80800574B3B4913F80E205E4821F063FFFFE5E4
:10A818005D4B37491A785D4821F05CFFF8E55C4BE1
:10A8280033499A785B4821F055FFF1E55A4B304996
:10A838001A685A4821F04EFFEAE5344B9B79012B00
:10A848007FF4E6ADB4F99C30B4F99E2036495448FB
:10A8580021F040FFDCE5534B31491A88524821F07A
:10A8680039FFD5E5514B9FED527A1B882049514855
:10A8780007EE903AF8EEE77A67EE877AFDEEE77A28
:10A8880017EE902A21F026FFC2E5414A2649138A8D
:10A898004948928921F01EFFBAE53D4A2249D389E9
:10A8A8004648528921F016FFB2E5394B10495A79CA
:10A8B800434821F00FFFABE5354B0D491A79414864
:10A8C80021F008FFA4E5324B0949DA783E4821F027
:10A8D80001FF9DE5627906493C4821F0FBFE97E5BA
:10A8E800227903493A4821F0F5FE91E56687002070
:10A8F8007482030878820308D43F0020E8810308A3
:10A90800688203082800002054820308948A0020E3
:10A91800F4820308008303086C870020B0470020F6
:10A92800CCB60308E0820308CC820308D48203086B
:10A93800933B0020E8820308B8820308C08203081A
:10A94800447C0020AC820308A08203089882030894
:10A95800EC3F0020B0830308CC830308C4830308BA
:10A968008C470020BC830308A08303089483030852
:10A9780088830308808303087483030868830308B3
:10A9880060830308588303080C910020448303085C
:10A99800747F002034830308887F002028830308FD
:10A9A8001883030870870020108303081C7900208F
:10A9B8000000C842A8850308948503088485030815
:10A9C80074850308608503085485030844850308D3
:10A9D800488503087E4B7F491B687F485A8D21F0C4
:10A9E80079FE15E57A4B7B491B687C481A8D21F066
:10A9F80071FE0DE5764B77491B6879485A8F21F02F
:10AA080069FE05E5724B73491B6876481A8F21F079
:10AA180061FEFDE46E4B6F491B68734893F837205D
:10AA280021F058FEF4E46A4B6A491B686F4893F8B2
:10AA3800362021F04FFEEBE4654B66491B686C48F5
:10AA48009A8E21F047FEE3E4614B62491B6869482E
:10AA58005A8E21F03FFEDBE45D4B5E491B68664879
:10AA680093F82D2021F036FED2E4594B59491B6842
:10AA7800624893F82C2021F02DFEC9E4544B554927
:10AA88001B685F4893F8272021F024FEC0E4504B50
:10AA980050491B685B489A8C21F01CFEB8E44C4B6B
:10AAA8004C491B6858485A8C21F014FEB0E4484BB6
:10AAB80048491B685548DA8B21F00CFEA8E4444B42
:10AAC80044491B6852481A8C21F004FEA0E4404B0C
:10AAD80040491B684F4893F8262021F0FBFD97E476
:10AAE8003B4B4D49D3F800E04C489EF81C309EF88B
:10AAF8001B209EF81DE0CDF800E021F0EBFD87E477
:10AB0800334B34491B6846481A7E21F0E3FD7FE445
:10AB18002F4B4149D3F800E042489EF816309EF882
:10AB280015209EF817E0CDF800E021F0D3FD6FE482
:10AB3800274B3949D3F800E03B489EF813309EF87C
:10AB480012209EF814E0CDF800E021F0C3FD5FE488
:10AB58001F4B3149D3F800E034489EF810309EF876
:10AB68000F209EF811E0CDF800E021F0B3FD4FE48E
:10AB7800174B2949D3F800E02D489EF80D309EF870
:10AB88000C209EF80EE0CDF800E021F0A3FD3FE494
:10AB98000F4B2149D3F800E026489EF80A309EF86A
:10ABA80009209EF80BE0CDF800E021F093FD2FE49A
:10ABB800074B1949D3F800E01F489EF807309EF864
:10ABC80006209EF808E0CDF800E021F083FD1FE4A0
:10ABD800EC3F0020748203083085030820850308B1
:10ABE8001485030804850308EC840308D08403084B
:10ABF800BC840308A48403089084030880840308A1
:10AC0800708403085C8403084C84030840840308A8
:10AC1800308403081C840308B083030814840308E1
:10AC28000C84030800840308F8830308F0830308EE
:10AC3800E8830308E0830308D88303082DE9F04F6D
:10AC4800724B734A1C7893B000F59C4120318146C1
:10AC580007911160002C00F0F2846E4A126890424D
:10AC680040F22B826C4A6D491768DFF8E8B104920C
:10AC7800013C1C706A4C039107F48057002F40F088
:10AC88002982039B5B7D002B40F0A584049B1B68F5
:10AC98001D0400F1FC86634B9945A37800F27D837F
:10ACA800002B40F07D83604B0593049B1F6817F4CD
:10ACB800805940F00484039BBBF906605B8B9E427D
:10ACC800B4BF00260126594B1B6813F0805300F0CF
:10ACD8000B82059A127812F0010200F00C82039898
:10ACE8005349408C91ED037A07EE900AF8EEE77A23
:10ACF800B4EEE77AF1EE10FA80F2C387002E40F046
:10AD080001824C4D95F8A010002940F0FB814A487B
:10AD18004A49056895F82D50002008604860886009
:10AD28004749002D40F0EF810D70002A40F0F08176
:10AD3800444B1A78002A50D10399BBF900E04F8B95
:10AD4800898BBBF90200BE45CCBF8025002545F0A4
:10AD580040038E45A8BF2B469B0843F08005B842A8
:10AD6800C8BF2B4643F040058842A8BF1D46BBF923
:10AD780004E0BBF90600AD0845F08003BE45C8BF36
:10AD88001D4645F040038E45A8BF2B469B0843F05F
:10AD9800800E284DB842C8BF734643F0400E95F860
:10ADA800A2708842B8BF73469F4201F00281A5F89D
:10ADB800A42085F8A620244985F8A2300F78002F12
:10ADC80001F04F805F2B01F0DA806F2B00F0B18724
:10ADD800059B1B78DB0740F17387049B1B4A1B68A4
:10ADE800069203F00403002B40F0E0840DF14008C4
:10ADF800174D0023C8F8043005F15009109340F6A8
:10AE0800330A192740F2833629E000BF3079002041
:10AE1800D47400202C790020987F00205450002002
:10AE28000C480020404B4C00C04F0020E08A002016
:10AE3800803F0020F8240020EC3F0020D886002026
:10AE480054270020483D00204C000020E88A0020BC
:10AE58000C890020D06E002004354D4520D0AA78FA
:10AE6800EB789A4217FB0260F6D26978043117FB37
:10AE780003623BF911305345A8BF5346B3F5617FD0
:10AE8800B8BF4FF461739842E6DA9A42E4DB297856
:10AE98002429E1D840460435F7F7B8FF4D45DED1FF
:10AEA800B24B98E803001F78B14B83E80300002FEA
:10AEB80000F007840121AE48F7F7B7FF002840F0FB
:10AEC800A481E378002B40F0A081AA4C23881DB20E
:10AED80025F00105AEB2B342268000F06B86A64D80
:10AEE80002270E204FF014094FF0FF082F7085F845
:10AEF800019085F8028026F07FFC39469C48268818
:10AF0800F7F793FF002841F0078026F002039BB271
:10AF1800B34223800AD0984B1421FF2202250E2029
:10AF28001D7059709A7026F067FC2688DFF898A281
:10AF3800924B9AF8001058680393B50708BF81F040
:10AF48000201C1F34001F7F751F824218848F7F7C7
:10AF58006CFF30B9059A1378590744BF23F00403EE
:10AF68001370069B1B6813F00A0F24D00521804834
:10AF7800F7F75BFF002800F0518625886F0740F13E
:10AF88004B877B480621F7F750FF002800F03386EF
:10AF98006E0640F15E8707217548F7F746FF50B106
:10AFA800774B784AB3F90430774982FB0302DB1701
:10AFB800C3EBA2030B800C216D48F7F736FF2288FC
:10AFC800002800F03E8142F480739A42238009D021
:10AFD800694B02251421FF220E201D7059709A70AA
:10AFE80026F00AFC694B1B78082B00F036810E2BE3
:10AFF80000F03381049B1B685D0544D5644B1B79C5
:10B00800002B00F0E78014215948F7F70EFF0028BD
:10B0180040F0E58023F038F801200CF00BF890B3ED
:10B02800DFF8A88100254FF0CC0902E0DDB2022D3F
:10B0380029D809FB05F76B1C58F80760002EF5D1D5
:10B04800C378544A90F9020052F82330019603223B
:10B058000092012132460BF0BBFB034605EB45008D
:10B0680000EB0010049353B1314608EB8000CC226A
:10B078002AF00FF9049B48F807300135EDB221F0AA
:10B0880083F90028D3D1059B1B78D80740F1F880B5
:10B098004149424A01230B701370039B9AF8001030
:10B0A800186801F00101F6F7A1FF069B1B685B0712
:10B0B80000F1568113B0BDE8F08F394B394A1F684B
:10B0C800049307F480570392DFF804B1364C002F3D
:10B0D8003FF4D7AD00212648F7F7A7FE00287FF4F4
:10B0E800D0AD0DF077F8CCE578023FF5F2AD059AD2
:10B0F800127802F001022D4D002185F8A010002ED3
:10B108003FF405AE2A4901200870002A3FF410AE2A
:10B11800F9067FF50DAE274A1278D2063FF508AE3C
:10B12800B9F1000F7FF404AE002B7FF401AE7D026D
:10B138003FF5FEAD204B1B78002B01F01F831F4B02
:10B148009B78002E41F02A833BB11D4A1D4B1268A3
:10B158001B689B1A002BC1F2C6831020134D26F0E2
:10B168004BFB012385F8A130E2E500BF3A430020FC
:10B17800E08A0020BC3F002094320020B0720020FA
:10B18800CC3F0020676666665024002008890020AE
:10B19800B44B0020C87D0308C14F00207C24002048
:10B1A800987F0020545000200C480020F8240020EC
:10B1B80054270020908A00204C00002030290020CD
:10B1C800E472002004300020AC720020206B0020C4
:10B1D800D06E0020059B1B78D9077FF51BAF3C205C
:10B1E8001AF058FE00283FF44EAF0BF0D9FA3C2075
:10B1F8001AF0F2FD00283FF446AF0BF0D1FA3C20DC
:10B208001AF0EAFD0028F0D13DE7069B1B689A0773
:10B218007FF55BAEBF4C2688F3073FF576AE46F068
:10B2280001039E4223803FF470AEBB4B1421FF22E2
:10B2380002250E201D7059709A7026F0DDFA2688B6
:10B2480063E622F480739BB29A4223807FF4C0AEF7
:10B25800B24B1B78082B7FF4CAAE228822F0400339
:10B268009BB29A4223803FF4C5AEAB4B0225142112
:10B27800FF220E201D7059709A7026F0BDFAB9E6AB
:10B28800A74B93F80090B9F1000F5FD1DFF8E48283
:10B29800A44F18F8030C3E784146A8F1030508F0BE
:10B2A8001FFD002800F09C83002E40F0EE8305F17E
:10B2B8000801687908F014FD002841F071819A4965
:10B2C800A87A08F00DFD002800F09D83022E41F0B9
:10B2D8006B819649E87B08F003FD002841F06881FE
:10B2E8009349287D08F0FCFC002800F09D83042E7B
:10B2F80041F062818F49687E08F0F2FC002841F035
:10B308005F818D49A87F08F0EBFC002800F09D8341
:10B31800062E41F02881894995F8230008F0E0FCC1
:10B32800002840F0F186864995F8280008F0D8FCF6
:10B33800002800F09D83082E40F0D086814995F8BA
:10B348002D0008F0CDFC002840F09D837E4B0122A3
:10B358001A7008F048FF069B1B685B077FF5AAAECA
:10B36800032008F0E7FC002800F01E86238813F06D
:10B3780008047FF49FAE082026F04EFB7348744DF6
:10B388007449754A754BBBF8066000682E800860E2
:10B3980014601C6013B0BDE8F08F0BB90123A370D3
:10B3A8006F4B05931B201F7894F8216008F0C2FCAE
:10B3B800012E07F00109824600F0DD8507F002033F
:10B3C800069394F82030DFF8B081664D052B69D8D4
:10B3D800DFE813F05B004F000600DC00FF008D0083
:10B3E800012E04BF052384F82030B9F1000F00F0C6
:10B3F8001381039B5C4FB3F91810B8F80030002292
:10B4080061F30F0263F31F42002361F30F0361F33B
:10B418001F43CBF8042039686269CBF800308A42B0
:10B42800C0F01684012E41F0D781032294F8203011
:10B438000692CBE708F0AAFC012807D14A4FB8F8D2
:10B4480002303A68642101FB03232361BAF1000F3B
:10B4580004D098F80630002B40F09080012E21D0BF
:10B46800414F22693B689A42C0F0EC85012384F879
:10B478002030012E3BD098F80730012B00F0D58002
:10B488000FF082F894F82030A0E7B9F1000FD1D17D
:10B498004FF48060BAF1000F00F0AA8326F0BCFADE
:10B4A80000232361069B002B3FF4FFAB069826F090
:10B4B800A3F9049B1F6817F480593FF4FCAB1D21C6
:10B4C8002A48F7F7B2FC00287FF4F5AB284A039B1B
:10B4D800D2881B8BBBF90660991A8E4240F3AF8560
:10B4E80013449E42B4BF00260126FFF7ECBB1E4F53
:10B4F8003A68B8F80230642101FB03234FF48060F6
:10B508000022236184F82020E27026F06DFA94F876
:10B5180020305BE7BC3F00209432002008890020DF
:10B52800C14F00203C0000208C31002091310020C8
:10B53800963100209B310020A0310020A531002049
:10B54800AA310020AF3100207C240020C88A0020C6
:10B558005C24002068240020602400205824002057
:10B56800C04F0020EC8A0020E4720020E08A00200E
:10B5780070320020823100208C3200200FF004F855
:10B5880003224FF47A7384F82020E361994F2B88C3
:10B5980043F002032B800CF01DFE3A68E369134464
:10B5A8000422A36184F82020012E40F055853B68D1
:10B5B800A2699A42BFF476AF8F4B187820B908F089
:10B5C800B9FB00287FF46EAF2B8823F002032B8091
:10B5D8008EE7884FE8E7039A013BD27D3BF91330A9
:10B5E800002A40F03083A3F57A73B3F57A7FA8BFB9
:10B5F8004FF47A7323EAE37307EE903A9FED7F7A6C
:10B60800F8EEE77A67EE877A7D4AFCEEE77A17EE7E
:10B61800903A1380FFF73FBB764F3B6847F23052B2
:10B628000323E26184F82030B1E70EF0ADFF032276
:10B6380040F6B83384F82020E3616E4FA7E7714FD6
:10B648003B78002B00F044876F4BDFF8D481DFF89C
:10B65800D4B1DFF8D4A1039345465E4604909946D9
:10B668000EE019F804109847032C28DC88B93B78B9
:10B678002AF8020F01349C4205F1040580F2DA80B1
:10B68800072CE1B23046DBF80430EADD984700B217
:10B69800EDE738F824206B88801A4FF47A719B1AEA
:10B6A80001FB00F040F6CA0290FBF3F00844904218
:10B6B80040F2EE23A8BF10469842B8BF184600B221
:10B6C800D5E7DFF868A1DFF86881504D0AF15A061E
:10B6D8004FF0010951461AF8010C08F001FBF8B1C6
:10B6E8009AF804009AF802309AF803E000EB400157
:10B6F80005EB8101013BD1F8B42003EB430343443C
:10B7080093420DD095F8E02081F8B0E009FA00F0F6
:10B7180022EA0000C1F8B430C1F8B87085F8E0003A
:10B728000AF1060AB245D5D13949324A394B3A4D60
:10B7380009681B78D2F8009008910793A5F1B00A20
:10B7480000266B685BB31F784FB3AA68A9EB0202A7
:10B75800002A0ADB9AF8E0200121B14022EA01021E
:10B7680009F5FA718AF8E020A960079ABAB12A782F
:10B7780059780432D2B2002940F0898203993BF902
:10B788001220098B01F1C800824240F32A849AF8FA
:10B79800E0109A7841FA06F3D80740F19A84013606
:10B7A800042E05F10C05CCD1FFF784BB174D95F895
:10B7B800AA3053B1059B1B78DE0706D5039BBBF95E
:10B7C80006205B8B9A4200F35A8411211348F7F73D
:10B7D8002CFB002800F0438295F8AE302BB995F881
:10B7E800A83013B93223A5F8AC30012385F8AE3060
:10B7F800FFF7FCBAE47200204C000020AAF1823F57
:10B80800C48A0020BC8D002054500020F824002059
:10B818000C2900207D3F0020A8250020E08A002078
:10B82800D48D00204C480020F624002099300020B8
:10B83800C0570308DDF81090C44A04921146C44A60
:10B848000968A2FB092A42F201020A404FEA9A1A41
:10B85800059200F00082BF4DBF48C04CC04A95F821
:10B8680000E0007884F800E01070BEF1000F04D00A
:10B87800BB4A92F800E08EF0010EBA4D0F2085F811
:10B888002400002B00F0FA82B74B039E0C931B7820
:10B89800B6F826C00B931C463B78B78C039EB34A78
:10B8A800368B0E962646A2FB0442520802EB420251
:10B8B800B21AD2B2CDF824C001F48051089295F89A
:10B8C8002580DFF8C0B2DFF8E8C20A900AF5967260
:10B8D80076460F9105F1280400200692CDF83490A1
:10B8E800AE46002E00F03A823EF910201FFA82F987
:10B8F800B9454FEA400103D3099DA94540F2728238
:10B908005CF82020924580F032823BF90120059DA9
:10B91800002D40F04682013098422BF8012004F1B6
:10B928000604DEDB0A98924ADDF834908EF825800A
:10B938000F280CBF012100218EF82400117000F09F
:10B94800A4828C4C8C4E8D4F35883868A16862680B
:10B95800E06045F00405401A90427F4F3580804DE5
:10B968004FF0010188BF00223970297088BF84F820
:10B978002120002B00F09B82049A03991768804EBF
:10B98800B1F824C0B1F818E07E4817F4805735465E
:10B9980040F0D38239460EE06A7802EB820202EB6D
:10B9A800820202F2EE2292B20131994220F8022B71
:10B9B80005F102050ED016F81120002A00F01682B3
:10B9C800022AE9D00131028820F8022B994205F1B8
:10B9D8000205F0D10C9A137801331370FFF74EB9B2
:10B9E80008F10501687908F07BF900283FF467AC95
:10B9F800012E40F0D58505F10D01A87A08F070F9FF
:10BA0800002840F0D1856049E87B08F069F90028F2
:10BA18003FF466AC032E40F0CB855C49287D08F0E6
:10BA28005FF9002840F0C8855949687E08F058F940
:10BA380000283FF466AC052E40F0C2855549A87F22
:10BA480008F04EF9002840F08E85534995F82300F8
:10BA580008F046F900283FF466AC072E40F05483FE
:10BA68004E4995F8280008F03BF9002840F0368345
:10BA78004B4995F82D0008F033F900283FF466ACDF
:10BA8800092E3FF463AC4FF009094B4629E3354DC5
:10BA9800D5F88830A9EB0303002BFFF6FCA8414A30
:10BAA80095F88C30517C079AC5F8882001333E4AB6
:10BAB800039E32F81120B17D03F00F0385F88C3016
:10BAC8002B4492B292FBF1F283F8902095F89010F3
:10BAD80095F8912095F8923095F89C000A4495F8CD
:10BAE8009310134495F89420194495F895300A4416
:10BAF80095F89610134495F89720194495F89830BE
:10BB08000A4495F89910134495F89A20194495F821
:10BB18009B300A44134495F89D1095F89F201844CB
:10BB280095F89E3001440B441A4442F30B12642AE0
:10BB3800F17DA8BF642213B209B1C2F1640307EE14
:10BB4800903A9FED1A7AF8EEE77A5BE5987F002045
:10BB5800D34D6210B0740020702100207D3F00207A
:10BB680071210020F8240020698D0020ABAAAAAA20
:10BB78004A4800200C480020EC8A0020E47200208B
:10BB8800088E0020D06E00209131002096310020D0
:10BB98009B310020A0310020A5310020AA310020CF
:10BBA800AF310020AC6F0020C86F002014AE2341D5
:10BBB8006C8D00200221C648F7F737F900283FF4BA
:10BBC800A4A92580B7073FF5B1A946F00203B342FF
:10BBD80023803FF4ABA9BF4B02201421FF22187029
:10BBE8000E2059709A7025F007FE2688FFF79EB937
:10BBF80025F0FAFE54E425F040039BB2AB422380C3
:10BC08003FF4C9A9B34B02251421FF220E201D7051
:10BC180059709A7025F0F0FDFFF7BDB9238823F01D
:10BC28000405ADB2AB4225803FF4ABA9A94B022570
:10BC38001421FF220E201D7059709A7025F0DCFD2A
:10BC48002588FFF79EB9C3F53B6308331BB2CAE4E6
:10BC580003230693E2E4A04A92F800E005E695F88B
:10BC6800A830002B3FF4C2A8059B1B7813F00103F2
:10BC78007FF4BCA8012285F8A83085F8A920FFF731
:10BC8800B5B8964D012185F8A010FFF73BBA0129F8
:10BC980000F0D8839AF8E0200123B340013613431B
:10BCA800042E8AF8E03005F10C057FF44AADFFF761
:10BCB80001B9059B8A4A1B781060D80700F1ED810D
:10BCC80095F8A61000297FF488A8B5F9A430322B7E
:10BCD8007FF783A895F8A2200120572A85F8A600A7
:10BCE80000F02684049B1B6813F0040302D05A2A30
:10BCF80000F031855D2A00F0A9845B2A00F0CB842E
:10BD08005E2A00F0D584562A00F00A85972A00F0AA
:10BD18001685A72A40F062847249049B0A781B683A
:10BD280042F004020A70704A069203F00403FFF717
:10BD38005AB8B2F5FA7FFFF650A895F8A620002A5F
:10BD48007FF44BA8059B1B78012185F8A610D9071D
:10BD580000F13A840BF02AFCFFF73FB8002F3FD0E0
:10BD68005CF8202092454FEA4001FFF4CEAD5F4ACF
:10BD78005E4D525C05EB0109002A00F09D80022A05
:10BD880047D199F8012002EB820202EB820202F20B
:10BD9800EE2292B2032833DD059D12B2002D3FF446
:10BDA800BAAD089D24F81520B8F1000F03D10B9DFA
:10BDB800022D7FF6B0AD2288B4F80290B4F8048062
:10BDC8004A4490444A4A0FFA88F882FB0852494D7F
:10BDD800A2EBE87225F8018012B24FF001089AE54B
:10BDE8003A464100069D4CF8205090E5CAB2022A16
:10BDF80004D9032A7FF4E6AD6246D5E57246D3E559
:10BE0800012505FA00F90A9D25EA090512B20A95E5
:10BE18007DE53BF80120BDE745F004039D42238002
:10BE28000AD02C4B02251421FF220E201D705970B8
:10BE38009A7025F0E1FC25882F4B304AB3F904307D
:10BE48002F4982FB0302DB17C3EBA2030B80FFF72A
:10BE580098B845F04003AB4223807FF4D3AEFFF798
:10BE68009AB839461A48F6F7E0FF00283FF421AFA0
:10BE780085F8A7700BF09AFBFEF7AABF2149224A62
:10BE88000C91DFF890B0012111701B211048059327
:10BE9800F6F7CBFF059B00287FF453AD1B4C1C4FD6
:10BEA800E2683B68A3609B1AC82B00F23383049BAB
:10BEB8001F6807F480578DE5C2B2022A40F2C0829B
:10BEC800032AA6D10E9A0F9D002D08BF3A4661E7B6
:10BED800E08A0020943200207D3F0020F8240020D2
:10BEE80008300020908A0020E88A0020088E002070
:10BEF8005655555568250020CC3F00206766666674
:10BF08003C240020698D00204A4800200C4800206D
:10BF1800E4720020D06E002026F001039BB2B342E9
:10BF280023803FF44FAE0E202F7085F8019085F8DE
:10BF3800028025F061FC268844E600210FE06A783B
:10BF480002EB820202EB820202F2EE2292B201318D
:10BF5800994220F8022B05F102053FF43BAD16F893
:10BF680011201AB1022AEAD00288F0E7CAB2032ADD
:10BF7800FAD87246EBE700230693FFF722BAB2F528
:10BF8800FA7FFEF62AAF95F8A630002B7EF425AF8F
:10BF9800059B1B7801210B4085F8A61000F09C82B8
:10BFA8000CF018F9FEF719BF082025F01DFDFFF762
:10BFB80081B8BB4ABB491068B5F9A420C76981FBA1
:10BFC80007018911FF17781A00F5FF407F30824278
:10BFD8003EF7F1AEC91B0A4412B2A5F8A420FEF739
:10BFE800EABEC8398A423DDA9AF8E0109A7841FAEE
:10BFF80006F3D9073FF5D3AB52420120099225F049
:10C00800DBFC7B1E099A162B00F2C280DFE813F0D6
:10C01800B001C6019701EF01DC01030282016D0145
:10C02800560131011A01C000EF0105010302820126
:10C038006D01EF00D900C300AE0096008000012614
:10C04800FEF741BE0EF0A0FA032240F6B83384F89A
:10C058002020E361FFF79BBA3A68E3691344A361C0
:10C06800FFF720BA9AF8E0300122B24023EA02032F
:10C0780009F5FA728AF8E030AA60FFF790BB002150
:10C088008948F6F7D2FE00287FF49FAB322385F863
:10C09800AA00A5F8AC30FFF798BB844B1B78002B9F
:10C0A8003EF49BAEE378002B7EF497AE95F8A7306C
:10C0B8000133DBB2032B85F8A7307EF68EAE7C4BBE
:10C0C8005B7813B9002E7EF488AE0CF083F8FEF787
:10C0D8007FBE002A0CBF012002208FE74FF008091D
:10C0E8004B4603EB83031D4487F80090A9786878D2
:10C0F80014F05EF8059B6F4A1B7801211170DA076E
:10C108007FF527A9FEF7C9BF4FF007094B46E8E7B7
:10C11800DAF8E400DFF8A08190F8361098F80230D9
:10C1280011446429A8BF642121EAE17180F836101E
:10C13800002B40F08B8324F00DFCABE5DAF8E4002B
:10C14800DFF8748190F8371098F802301144FE290E
:10C15800A8BFFE2121EAE17180F83710002BEAD050
:10C16800162007F045FEDAF8E400E4E70898DFF85F
:10C17800488141781144B1F5967FA8BF4FF4967174
:10C1880021EAE171417098F80230002B40F05883A1
:10C19800DAF8E400CFE7DAF8E400DFF81C81817808
:10C1A8001144C829A8BFC82121EAE171817098F813
:10C1B8000230002BBFD0142007F01AFEDAF8E40092
:10C1C800B9E7DAF8E400DFF8F08041781144C829CB
:10C1D800A8BFC82121EAE171417098F80230002B0C
:10C1E800A9D0132007F004FEDAF8E400A3E7DAF890
:10C1F800E400DFF8C48001781144C829A8BFC82129
:10C2080021EAE171017098F80230002B93D01220D6
:10C2180007F0EEFDDAF8E4008DE7DFF89C80089877
:10C2280098F80230417911446429A8BF642121EAB1
:10C23800E1714171002BABD00E2007F0D9FDDAF87F
:10C24800E40078E7DAF8E400DFF86C80017A98F81F
:10C2580002301144C829A8BFC82121EAE17101723E
:10C26800002B3FF468AF0B2007F0C2FDDAF8E400BA
:10C2780061E7DAF8E400DFF84080C17998F8023025
:10C288001144C829A8BFC82121EAE171C171002B56
:10C298003FF451AF0A2007F0ABFDDAF8E4004AE7B3
:10C2A800542A0020D34D6210E08A00207D3F0020F0
:10C2B800302900207C240020A48A0020DAF8E40039
:10C2C800DFF87885817998F802301144C829A8BF29
:10C2D800C82121EAE1718171002B3FF42CAF0920BC
:10C2E80007F086FDDAF8E40025E7DAF8E400DFF87D
:10C2F8004C85417998F802301144C829A8BFC82153
:10C3080021EAE1714171002B40F05382112F7FF433
:10C3180046AF10E7DAF8E400DFF82085017998F8ED
:10C3280002301144C829A8BFC82121EAE17101716E
:10C33800002B40F0D082102F7FF447AFFBE608991E
:10C34800DFF8F8840F791744642FA8BF642727EA19
:10C35800E7770F7107F066FD98F80230002B3FF47D
:10C3680017AF0320394607F043FDDAF8E400E2E6A8
:10C378000898DFF8C88401781144FA29A8BFFA217F
:10C3880021EAE171017098F80230002B3FF400AF08
:10C39800012007F02DFDDAF8E400CCE60898DFF874
:10C3A8009C84817811446429A8BF642121EAE17141
:10C3B800817098F80230002B3FF4EAAE022007F0B3
:10C3C80017FDDAF8E400B6E60898DFF87084C1795A
:10C3D80098F80230114481F30801C171002B3FF431
:10C3E800D7AE052007F004FDDAF8E400A3E6089BC1
:10C3F800DFF84884997998F8020011446429A8BFA5
:10C40800642121EAE1719971002840F0DA810D2F49
:10C418007FF405AFBCE6DAF8E400DFF82084C178E1
:10C4280098F802301144C829A8BFC82121EAE1714F
:10C43800C170002B40F05F820F2F7FF4DCAE7AE6EC
:10C448000E9AA7E43BF912209978B2F5617F4FF470
:10C45800966393FBF1F332DB40F633019142A8BFB8
:10C4680011460C2FA1F5617191FBF3F100F0F980F1
:10C47800182F7FF40FACC9B2C8290B46A8BFC82330
:10C48800DAF8E400C27DDFB297423FF403AC9A1AAF
:10C49800DFF8A883C77548BF0732D71098F802306D
:10C4A8000137FFB23BB9002F3FF4F4AB384625F013
:10C4B80083FAFFF7EFBB182007F09AFCF3E70C2F7D
:10C4C80000F0E680182F7FF4E5AB00210B46D7E794
:10C4D800C34A0392FFF7B0B9C249096811F40031A1
:10C4E80040F0EA800B46C048C65C0F2E03F10C03EF
:10C4F8003DD001311529F7D1049BBC491B68069131
:10C50800FA3AA5F8A420002203F0040385F8A6202F
:10C51800FEF769BCB64A049B1F68138823F004031E
:10C528001380012307F4805784F82130FFF752BAAB
:10C53800AE4AB04B069210461A68AF494FF47A7368
:10C54800B3FBF2F3C3EB431203EB82030268DB0095
:10C558005707A1F8B43000F1A280049B1B6803F0D0
:10C568000403FEF740BC4FF006094B46B9E5A34E5D
:10C57800D6F800E04B00BEF1000F07D05F1800EBC3
:10C5880087079EF801E07F787745B5D20B449C4F2A
:10C598009C4900EB8300002330603B800B60ABE7D5
:10C5A8004FF001094B469CE54FF002094B4698E5D0
:10C5B8004FF003094B4694E54FF004094B4690E5CC
:10C5C8004FF005094B468CE5049B8F491B680A60B0
:10C5D800864A069203F00403FEF705BC0021BB2A35
:10C5E800109100F09880B72A00F09180BE2A00F0E0
:10C5F8009580BD2A67D0792A00F05A817A2A00F0FE
:10C6080050819E2A00F047819D2A00F03D81AE2A84
:10C6180000F03381AD2A00F02981EF2A00F0208153
:10C62800FD2A00F01781FB2A00F04F81FE2A00F056
:10C638004681F72A00F067817B2A7EF4CEAB4FF45F
:10C64800FA6102200EF034FEFEF7C7BB6F4B0022E2
:10C6580001206F4D6F492A700B6025F0ADF9FEF788
:10C66800BCBBCFB26A4B09915B78BB423FF412ABBB
:10C67800DFF8C88138460EF0F5FE98F802300999BF
:10C688001BB1C9B20C2007F0B3FB0137FFB20AE7B0
:10C6980000273946E6E7604B01220220D9E7049BD0
:10C6A8005E4A1B680A21118003F00403FEF79BBB56
:10C6B8005B4B02220320CCE75A490978032900F092
:10C6C800868019460FE74FF6FE73574A4748968902
:10C6D8000690D089334401449381D1811CF096FBA4
:10C6E800F5F768FF1CF07AFBFAF7B2FF012025F096
:10C6F80063F9049BB5F8A4201B68FA3A0021A5F851
:10C70800A42003F0040385F8A610FEF76CBB0B46C3
:10C718004FF6FE71D9E70B460221D6E70223D4E78C
:10C728001CF074FBF5F746FF1CF058FBFAF790FF76
:10C73800012025F041F995F8A220FFF7E7BA049BFC
:10C748003A4A1B684FF4C8711180284A069203F0D0
:10C758000403FEF748BB95F8A820002A40F0DE80C5
:10C7680095F8AA3083F0010385F8AA30002B40F031
:10C77800D0800C2025F040F8FEF72FBB002E3EF4A9
:10C78800ECAC2B4D95F8A130002B3EF4D1AA25F046
:10C7980017F8002385F8A130FEF7CABA002BF0D0AD
:10C7A8002449254A09684FF47A7000FB0313136083
:10C7B800E7E71120099207F01BFBDAF8E400099A71
:10C7C800A4E50D20099207F013FB099A1FE624F04F
:10C7D800F7FFB5F9A4208FE603230693FEF766BE9C
:10C7E800545000208C300020D46D0308E88A0020C3
:10C7F800EC8A0020887F0020287000200427002071
:10C808009E270020A027002008300020A83B0020F9
:10C81800F03F0020EC3F0020F63B00202A290020B2
:10C82800443C0020DC8A00201C7900202C290020B0
:10C83800F8240020E472002004300020A48A00209C
:10C84800152007F0D5FADAF8E40074E4172007F0A9
:10C85800CFFA9DE4002101200EF02AFDFEF7BDBAB3
:10C86800002108460EF024FDFEF7B7BAFF2100208C
:10C8780026F0AEF995F8A220CFE60121002026F097
:10C88800A7F995F8A220C5E60021FF2026F0A0F917
:10C8980095F8A220BBE6012026F09AF995F8A22087
:10C8A800B2E6224A137A43F001031372FEF795BAEF
:10C8B8001E4A137A23F001031372FEF78EBA002181
:10C8C80003200EF0F5FCFEF788BA002102200EF0D6
:10C8D800EFFCFEF782BA1020099207F089FADAF81D
:10C8E800E400099A27E5124D0BF074FC002385F843
:10C8F800A130FEF71DBA0F20099207F079FADAF88D
:10C90800E400099A98E5002104200EF0D1FCFEF716
:10C9180064BA0B2024F070FFFEF75FBA054A85F869
:10C92800A81085F8A9000692FEF75DBA30480020E5
:10C93800F8240020E88A00202DE9F0478C4B1B786A
:10C94800DB07074644D58B4B8B4D1C788B4E012C4F
:10C9580059D01CD3022C07D189498A4A09881288E0
:10C96800914201D901241C70EB7AE3B12B89D3B130
:10C97800854B1B78BBB10FF0B5FA002800F09B80FF
:10C988002B7B83422CBF0121002131700CE07C49B4
:10C998007E4A098810886A7B801A8842E2DAEB7A34
:10C9A8000024002BE2D131782A79632A06D8022C98
:10C9B800774E00F0BA803378002B5DD1754AAB7A98
:10C9C8008C4238BF0C461470002B4CD1BDE8F08760
:10C9D8006B4B694D19885B88E878CB1A83EAE37258
:10C9E8008142A2EBE3721DD32B788B421AD3614BA1
:10C9F8001C78E01E012861D96749097802294FD0BF
:10CA0800012C5E4EA5D15F4A5D491288687B098872
:10CA1800121A914239DD5D4A12888A42A4D2002452
:10CA28001C70A1E7B1EB400FE1DC524B1C78E11E12
:10CA3800012940F29480022ADEDC57494F4E0878DB
:10CA4800DFF84481DFF844C1DFF838E1002103242E
:10CA5800022834701C7088F80010ACF80010AEF88A
:10CA6800001081D11FE0012C71D0022C0BD10720BE
:10CA7800BDE8F04724F0C0BE7068381A474B9842AA
:10CA880058DD72709AE7BDE8F08702241C706BE7E6
:10CA9800022AD2DD4049097802294FF0040464D102
:10CAA8003949364E09783E48022ACCBF0022012275
:10CAB800C28081804BE70221317075E7022A9BDC36
:10CAC80095F800C091FBFCFC0CF1010CBCF1080FBF
:10CAD800DFF8B4A0304EA87895F801E096F8008009
:10CAE8002A4CDFF8A090254EA8BF4FF0080C8AF812
:10CAF80000C01FFA8CFA10FB0AF01EFB0AFE80B277
:10CB0800DFF88CA02080A9F800E000244FF0640E24
:10CB1800B8F1020F34701C70CAF804408AF801E0BA
:10CB28007FF439AF0FFA8CF1BDE73078A0B9012353
:10CB380077603370C2F164021A4B00FB02F083FB8A
:10CB48000023C017A0EBA3506430707036E70820AC
:10CB5800BDE8F04724F050BE7368F81A8EE7032C3E
:10CB680096D10D49097802299AD0044EFCE600BFF7
:10CB7800C04F002038330020948A002068330020FA
:10CB8800C04900203C330020C93F00203A33002030
:10CB980048240020DC8A00202C4900207F96980039
:10CBA800304900206BCA5F6B2DE9F04F2DED0C8BDF
:10CBB800404B1B7893B0012B039001F0BC803E4C96
:10CBC80094F80021002A41F0C780072B01F0CE809D
:10CBD8004FF0000ADFF8ECB0DBF80430584698470D
:10CBE800002800F06F81BBF8B46000228BF8552054
:10CBF800002E40F06687BBF93C50DBF82410BBF9E7
:10CC08003E00DBF82820BBF94030691ACBF8301019
:10CC18002A490191821ADBF82C00CBF834200D4602
:10CC28001B1A9BF85610CBF838300BF130001BF06C
:10CC3800D1FE2B68990040F1E980DBED0D5ADBED60
:10CC48000C7A1F4A94ED416AD4ED426A94ED437A16
:10CC5800D4F810311268B8EEE58ADBED0E5AF8EE1A
:10CC6800E77AF8EEE58A013377EE867A38EE268A97
:10CC780078EE878A9342C4ED417A84ED428AC4ED06
:10CC8800438AC4F8103101F0F1820A4B1E78142E41
:10CC980002F0A1840023D4F818510293062D00F263
:10CCA800A880DFE815F0F712E6120B127B121100CC
:10CCB8002114BA132C490020E0250020987F002079
:10CCC8007475002028700020D44B1A78D4F81C7191
:10CCD800DFF8B8E39FEDD27AF8000EEB000383ED9E
:10CCE800007A002A7AD0CF49B0EE476AF0EE476A58
:10CCF8000023F1EC017A013367EEA77A05EE903A4A
:10CD0800B4EEE77AF1EE10FAF8EEE55AB8BFB0EEF5
:10CD1800677A9A4276EEA76AA7EEA56AE9D1F5EE98
:10CD2800C06A0EEB0003F1EE10FA83ED007A55DDD0
:10CD3800C6EE265ABC4BBD4A1288F7EE007A75EE4D
:10CD4800E75AD3ED007A65EEA77AFDEEE77A17EE9B
:10CD5800903A812B43F317839342A8BF134607EEFB
:10CD6800903AF8EEE77AB24BC11903EB810393EDE1
:10CD7800057AD3ED003A93ED066A93ED014AD3EDB7
:10CD8800046AD3ED034A93ED025AA3EEA77AA4EE00
:10CD9800276A66EEC76AA7EE646ABDEEC77AE5EE53
:10CDA800276A17EE101A812983ED056AC3ED066A12
:10CDB80043F3E6828A42A8BF0A4607EE902AF8EEB5
:10CDC800E77AFCEEE77ACDED047ABDF810300EEB89
:10CDD8000002938017B9132E03F0A687152E42F090
:10CDE800BF817044DFF8A882838828F81730D4F808
:10CDF8001851904B013583FB05235A19EB17C3EBE8
:10CE0800A203C3EBC303ED1AC4F818518A4B1B786D
:10CE1800002B01F0E380894DCDF808A0DFF874827B
:10CE2800DFF86C92DDF804A005F5BC770026844B8A
:10CE3800DBED087A1B78172B01F0258495ED007A35
:10CE4800B8EEC78A082B28EE278A07D1B0EE480A21
:10CE5800019326F011F9019B29F81600DAF8002051
:10CE680092000BD5002E04F0F080B0EE480ADBF8F3
:10CE7800143207F170009847B0EE408AB0EE480AC5
:10CE8800DBF83431A7F170009847DBF8A431384655
:10CE980098476B4B1B78032BB0EE408A01F0ED836B
:10CEA800D5F8F800DBF8B830B0EE480A98470136F4
:10CEB800032E07F12407A8EC010A05F10405B6D1F1
:10CEC800DDF808A05E4B1F78072F00F0BA8694F8AB
:10CED80028310493002B40F0C2865A4B5B79002B13
:10CEE80040F0E9850123564A84F828311278072A48
:10CEF80001F0748600230593534B94ED4C9A93EDFF
:10CF0800007A524BD4ED4BCAD3F800A0504B029391
:10CF1800F7EE007A37EEC9CA00252CEE07CA4D4B4A
:10CF2800DFF87491DFF874B1DFED4B8A9FED4BAAFF
:10CF3800DFED3BBADFED4A9A9FED4ABADFED4AAA28
:10CF4800DFF85C81494F0193B4EEE7CAF1EE10FABD
:10CF580088BFB0EE67CA2E46454B99ED008A2B4430
:10CF6800D3ED007AF5EE407AF1EE10FA17D0414B86
:10CF78002B44D3ED006A38EE667AB0EEC76AF4EE59
:10CF8800C67AF1EE10FA08D5B5EEC07AF1EE10FACD
:10CF9800CCBF37EEA68A36EEE78A83ED008A364B99
:10CFA8001A8893077ED0022E7CD09AF82E10334B25
:10CFB80007EE901A2B4493ED007A4B42F8EEE76A9D
:10CFC80007EE903A26EE877AF8EEE77AB4EEE77A3B
:10CFD800F1EE10FA0AD407EE901AF8EE677AF4EE3A
:10CFE800C77AF1EE10FA88BFF0EE477A244B25494C
:10CFF80003EB460331F91600B3F90C30C01A07EEFB
:10D00800100AB8EEC77AD007E7EE687A40F12F86A3
:10D018001D4B93ED008A27EE888A43E07A7500203D
:10D0280000000000E02500207C75002078750020B5
:10D03800B077002093244992717500205870002021
:10D048002C490020747F002060910020EC3F0020D4
:10D05800887F0020CC860020CDCCCC3DAE47813FD8
:10D068000000C84200003443610BB63BD88600205C
:10D078005491002020270020BC3F00202C270020AE
:10D088001C790020CC3F00203C910020987700209C
:10D09800304900208C7F0020142700204890002071
:10D0A800E4860020029B94F864212B44D3ED01DA36
:10D0B80038EE6DDA002A3DD0D34BD4F868210399B5
:10D0C8001B688A1A9A4235DD9AF84830022B01F01B
:10D0D800BC85022E03F05987CC4B1B68990740F199
:10D0E8006487CB4BCB49DFF8A0E331F916C09EED3E
:10D0F800008ADFF898E3C7ED00BA03EB460028EE94
:10D10800288AB0F90C00A0EB0C0007EE900AF8EEA4
:10D11800E77ADEF8000027EE888A904238EE6DDA6A
:10D12800C1F27980F7EE007AB4EEE79AF1EE10FAE0
:10D1380001F14880B84B2B4493ED000A019B2CEE7B
:10D14800800A022E20EE0D0AA3EC010A019303F0D7
:10D158003687B24B9BED007AD3ED007AB04BD7ED12
:10D16800006A93ED006AAF4B67EE277A2B4427EEEF
:10D178008C7AD3ED007A67EE277AF0EE665AEDEEF8
:10D18800275AB1EE467AF4EEC75AF1EE10FA08D4EF
:10D19800F4EEC65AF1EE10FA8CBFB0EE467AB0EE55
:10D1A800657A94ED4C6AF7EE007AB4EEE76AF1EE30
:10D1B80010FAACBF0123002343B1F0EEE66AF0EEAB
:10D1C800C77AF4EEE67AF1EE10FA01D587ED007A27
:10D1D800022E03F0D386944A944B52F826001B681B
:10D1E800B0EE6D0A9847924A924B52F826001B6897
:10D1F80098479AF8373023B18F4B1B88002B00F0E3
:10D20800BA85B0EE6B8A8D4B9BED007A38EE400AFA
:10D218002B4493ED008A83ED000A9AF8483030EEEB
:10D22800480AC0EE077A2BB3854B1B78DB0721D55C
:10D23800B7EE007AB4EEC79AF1EE10FA04DB94F870
:10D248006431002B00F06587D4F86831039AD31A4B
:10D258006D4A12689A420DDD7A4B93ED007AB0EE72
:10D26800CDDAB4EEC7DAF1EE10FA40F1F087002318
:10D2780084F86431744B94F874212B4493ED007A4C
:10D288002CEE877A67EE277AC8ED007A32B9019BCF
:10D29800C7ED00BA43ED01BAC8ED00BA0136032E56
:10D2A80009F1040908F1040807F1040705F1040568
:10D2B8007FF452AE654B1B78072B01F01482012BCB
:10D2C80001F091840023029394F87C31002B40F004
:10D2D80097855F4B5F4A1B68126813F4805C92F86D
:10D2E8002C2040F0A4865C495C4891ED006A408B94
:10D2F8005B4984ED636A91ED007A5A4984ED647A5A
:10D3080007EE900AF8EEE76AD1ED037A564984ED04
:10D31800616A37EE467A77EEE67AD1ED006A84EDF7
:10D32800607A012184F89411C7EEA65A4F485049F3
:10D3380090ED005A4F489FED506A90ED004A4F48D3
:10D34800DFED4F6AD0ED004A91ED007A35EE045AD0
:10D35800F7EE007AF4EEE75A35EE245AF1EE10FAB9
:10D3680088BFF0EE675A25EE065AF4EEE65AB1EE9B
:10D37800476AF1EE10FAB4EEC65AB8BFF0EE665A34
:10D38800F1EE10FAC4ED665A00F1FD87B4EEC75A03
:10D39800F1EE10FA88BFB0EE475A3449DFED366A2D
:10D3A800D1ED017A334991ED014A344977EE847A17
:10D3B800D1ED014A77EEA47A67EEA67AB4EEE76A71
:10D3C800F1EE10FA08DCB4EEE77AF1EE10FA8CBF51
:10D3D800B0EE676AB0EE476A2449DFED276AD1EDFF
:10D3E800027A2449D1ED024A264977EEA47A91EDD2
:10D3F800007A67EEA67AB1EE473AF4EEC37AF1EE18
:10D4080010FA4ED444E000BF68910020E88A00205A
:10D418001C790020CC3F0020109100204000002003
:10D42800849100201C910020509000204C900020F6
:10D43800A4900020A0900020BC3F00204C27002092
:10D44800C04F002074910020289100202C49002012
:10D45800987F0020EC3F0020748700205450002063
:10D4680064320020803F002078320020CC860020E3
:10D4780088910020D88600206F12833AE486002025
:10D48800000000008C9100203C9100206491002055
:10D49800F4EEC77AF1EE10FA8CBFB0EE473AB0EE70
:10D4A800673AED49497809B9B1EE433A002A41F0A3
:10D4B8003E82F7EE003ADFF8C8B39BF80020002A56
:10D4C80002F03782E549DFEDE66AD1ED024A91EDD7
:10D4D800017AD1ED037A66EE244AE5EE074AE3EED7
:10D4E800274A63EEA44AF4EEE64AF1EE10FAB4BF16
:10D4F800B0EE664AB0EE644A98BFF0EE646A012A5C
:10D50800CDED0A4A02F0368291ED067AD1ED052A70
:10D51800D1ED077A26EE077AA5EE227AA3EE277ACE
:10D5280023EE877AB4EEE67AF1EE10FAB4EEC47A16
:10D538008CBFF0EE667AF0EE477AF1EE10FA98BFFB
:10D54800F0EE676AB4BFF0EE447AF0EE477A022A4A
:10D558008DED0B7A00F0DE8091ED0A7AD1ED092A83
:10D5680091ED0B4A26EE077AA5EE227AA3EE047A0D
:10D5780023EE877AB4EEE67AF1EE10FAB4EEE77AA3
:10D588008CBFB0EE664AB0EE474AF1EE10FA98BF8B
:10D59800F0EE446AA8BFF0EE477A032A8DED0C7AC4
:10D5A80000F0B88091ED0E7AD1ED0D2A91ED0F4A79
:10D5B80026EE077AA5EE227AA3EE047A23EE877A7E
:10D5C800B4EEE67AF1EE10FAB4EEE77A8CBFB0EE7C
:10D5D800664AB0EE474AF1EE10FA98BFF0EE446A98
:10D5E800A8BFF0EE477A042A8DED0D7A00F09280FC
:10D5F80091ED124AD1ED112A91ED137A26EE044AE3
:10D60800A5EE224AA3EE074A23EE844AB4EEE64A80
:10D61800F1EE10FAB4EEE74A8CBFB0EE667AB0EEDF
:10D62800447AF1EE10FA98BFF0EE476AA8BFF0EE20
:10D63800447A052A8DED0E4A6CD091ED164AD1ED4B
:10D64800152A91ED177A26EE044AA5EE224AA3EE92
:10D65800074A23EE844AB4EEE64AF1EE10FAB4EE35
:10D66800E74A8CBFB0EE667AB0EE447AF1EE10FA73
:10D6780098BFF0EE476AA8BFF0EE447A062A8DED0F
:10D688000F4A47D091ED1A4AD1ED192A91ED1B7A2C
:10D6980026EE044AA5EE224AA3EE074A23EE844A60
:10D6A800B4EEE64AF1EE10FAB4EEE74A8CBFB0EEFB
:10D6B800667AB0EE447AF1EE10FA98BFF0EE476A57
:10D6C800A8BFF0EE447A072A8DED104A22D091EDDA
:10D6D8001E7AD1ED1D2A91ED1F4A26EE077AA5EE96
:10D6E800227AA4EE037A27EE237AB4EEE67AF1EEF4
:10D6F80010FAB4EEE77A8CBFB0EE666AB0EE476A0D
:10D70800F1EE10FA8DED117A98BFF0EE466AA8BFD7
:10D71800F0EE477A77EEE67AF7EE006AF4EEE67A0C
:10D72800F1EE10FAC4ED4C7A43F39A8286EEA77AAA
:10D73800022ADDED0B7A67EE244A67EE877ACDED93
:10D748000A4ACDED0B7A2DD0DDED0C7A67EE877A9B
:10D75800032ACDED0C7A25D0DDED0D7A67EE877AB8
:10D76800042ACDED0D7A1DD0DDED0E7A67EE877AAD
:10D77800052ACDED0E7A15D0DDED0F7A67EE877AA2
:10D78800062ACDED0F7A0DD0DDED107A67EE877A97
:10D79800072ACDED107A05D0DDED117A27EE877ACC
:10D7A8008DED117A2F49096811F0805800F096879D
:10D7B800F6EE005AC4ED665A002A02F0B18094F9D8
:10D7C8009401D4ED644A284D284994ED636A284EA3
:10D7D800284FDFF8B0E0B5F81AA0C978B6F9069076
:10D7E80097ED005A9EF800E0D4ED606AD4ED617AB6
:10D7F80007EE100AFDEEE44A1F4814EE905A00782E
:10D80800FDEEC64A03F0100603F4800300F001079A
:10D81800B8EEC77A14EE900A0193002941F0C68049
:10D828000E49002E40F07C8791ED006A9DED0A5A62
:10D83800124B25EE866AA5EE076AB0EE675AA6EE89
:10D84800265ABDEEC56A16EE10EA16EE106AAE4507
:10D85800A8BF2E4618E000BF08890020E431002048
:10D8680000000000E08A0020545000200C480020EE
:10D87800D06E0020C0310020C04F00202C8700202F
:10D888000D490020687C00207045C8BF064606EE9A
:10D89800106AB8EEC66A012A83ED006A00F0DC80DF
:10D8A80091ED046A9DED0B5A25EE866AA5EE076A8E
:10D8B800B0EE675AA6EE265ABDEEC56A16EE10EA15
:10D8C80016EE106AAE45A8BF2E467045C8BF06467C
:10D8D80006EE106AB8EEC66A022A83ED016A00F005
:10D8E800BB8091ED086A9DED0C5A25EE866AA5EE7F
:10D8F800076AB0EE675AA6EE265ABDEEC56A16EE5E
:10D9080010EA16EE106AAE45A8BF2E467045C8BF8D
:10D91800064606EE106AB8EEC66A032A83ED026A66
:10D9280000F09A8091ED0C6A9DED0D5A25EE866AFD
:10D93800A5EE076AB0EE675AA6EE265ABDEEC56A8E
:10D9480016EE10EA16EE106AAE45A8BF2E467045D0
:10D95800C8BF064606EE106AB8EEC66A042A83ED0A
:10D96800036A79D091ED106A9DED0E5A25EE866A0C
:10D97800A5EE076AB0EE675AA6EE265ABDEEC56A4E
:10D9880016EE10EA16EE106AAE45A8BF2E46704590
:10D99800C8BF064606EE106AB8EEC66A052A83EDC9
:10D9A800046A59D091ED146A9DED0F5A25EE866AE6
:10D9B800A5EE076AB0EE675AA6EE265ABDEEC56A0E
:10D9C80016EE10EA16EE106AAE45A8BF2E46704550
:10D9D800C8BF064606EE106AB8EEC66A062A83ED88
:10D9E800056A39D091ED186A9DED105A25EE866AC0
:10D9F800A5EE076AB0EE675AA6EE265ABDEEC56ACE
:10DA080016EE10EA16EE106AAE45A8BF2E4670450F
:10DA1800C8BF064606EE106AB8EEC66A072A83ED46
:10DA2800066A19D091ED1C6A9DED115A65EE865A69
:10DA3800E7EE055AE6EEA57AFDEEE77A17EE901ABC
:10DA48008D42A8BF0D468842C8BF054607EE905ACA
:10DA5800F8EEE77AC3ED077A2FB922B19200D349DD
:10DA6800D34825F0FFF8D34B1B68002B40F0A48463
:10DA7800D14B1B7893B19BF8000060B1CC4ECF4FCF
:10DA88000025E8B23B68B6EC010A98479BF800000D
:10DA980001358542F5DBCA4B1B689847C94B1B7893
:10DAA800072B00F03586012384F8003113B0BDEC54
:10DAB8000C8BBDE8F08FC44B1B78013BDBB2FFF742
:10DAC80012BAC24B02934FF47A751B68B5FBF3F395
:10DAD800C3EB4315BE49DFF8248391F80190B94997
:10DAE800B8F906000F7803EB8503DD00ADB2AE424E
:10DAF80001F08586DBF88810BBF93CE0DBF86C3078
:10DB08004A1C07EE90EA7344012ACBF88820CBF828
:10DB18006C30F8EEE77A01F07F86DBED1E5ADBED1C
:10DB2800206A07EE102A37EEE56AB8EEC75A012ECA
:10DB380086EE057A37EE257A77EEC77A8BED1F7A6F
:10DB4800E7EE866A8BED1E7AF0EE667ACBED216AF7
:10DB5800CBED206A02F05080DBF89C10BBF93EE068
:10DB6800DBF870304A1C07EE90EA7344012ACBF8C0
:10DB78009C20CBF87030F8EEE77A01F06886DBED90
:10DB8800235ADBED256A07EE102A37EEE56AB8EE70
:10DB9800C75A012E86EE057A37EE257A77EEC77AD0
:10DBA8008BED247AE7EE866A8BED237AF0EE667ABF
:10DBB800CBED266ACBED256A02F04780DBF8B01082
:10DBC800BBF940E0DBF874304A1C07EE90EA734476
:10DBD800012ACBF8B020CBF87430F8EEE77A01F0E0
:10DBE8005186DBED285ADBED2A6A07EE102A37EE5C
:10DBF800E56AB8EEC75A012E86EE057A37EE257A21
:10DC080077EEC77A8BED297AE6EE276A8BED287ACC
:10DC1800F0EE667ACBED2B6ACBED2A6A02F03E80F5
:10DC2800A8F80600BBF8B430664A013B1778ABF891
:10DC3800B43002990023072F4B608B60CB607FF4D0
:10DC480046A9F9F7E3FFDFF8B48194F82831049383
:10DC5800A0EB0A00A8F80000002B3FF43EA9013B06
:10DC680084F8283113B0BDEC0C8BBDE8F08F94ED2F
:10DC7800567AB1F90000D4ED576AB1F902E0554A75
:10DC8800F4EEC76A80EAE0738EEAEE71A3EBE07304
:10DC9800F1EE10FAA1EBEE71B8BFF0EE476A8B42D5
:10DCA800B8BF0B4607EE103A1378B8EEC77A27EEDE
:10DCB800287A002B40F0FE81474B93ED006AB4EEC2
:10DCC800CA6AF1EE10FA40F18487F7EE005A75EE51
:10DCD800C65A3BEE477A65EEAA5A404BA7EE256A2C
:10DCE80093ED007A26EE076AB5EEC06AF1EE10FAF7
:10DCF80040F2F084C9EE865AB7EE007AB0EE476A71
:10DD0800A6EEE56AF0EE466AF4EEC76AF1EE10FA9E
:10DD180088BFF0EE476AF5EEC06AF1EE10FAB8BFB8
:10DD2800F0EE6B6A2E4B93ED007A67EE877AA7EEDA
:10DD3800A68AFFF7B7B92B4B2B4C19682B4ADFF88B
:10DD4800BC8094F80031C9691288A8F80010A8F8B6
:10DD58000220002B3EF43CAFFAF7CCF9002384F8FC
:10DD68000031184B1B78072B7EF432AFF9F74EFFC2
:10DD78008246FEF72FBF1E4B1E4A2B4493ED007AB6
:10DD8800D2ED007A1C4B67EE277AF7EE006AF4EEC4
:10DD9800E67AF1EE10FA93ED007A88BFF0EE667A33
:10DDA80067EE877A27EE888AFFF72DBAC4310020FC
:10DDB8002C87002040900020707F00205C7C002091
:10DDC800647C00202C4900200C910020887F0020D2
:10DDD800747F002048910020509100204491002039
:10DDE80040910020542A0020E0250020502A0020DD
:10DDF8003827002038910020349100203049002035
:10DE0800D94BDFF8B8B31B789BF80020DD077FF506
:10DE180024AE002A3FF427AED4ED573A94ED564A83
:10DE2800D24BD4ED617A93ED005A94ED607AD4ED3B
:10DE3800545A94ED536ACE49CE4BF4EEC43AF3EEFD
:10DE4800046AF1EE10FA77EEA64A00F1578791EDD1
:10DE5800026A26EE656AB0EE674AA6EE074AB4EE95
:10DE6800E44A34EE666AF1EE10FA48BFB0EE456A4D
:10DE7800012A83ED006A3FF4F6AD91ED066A26EEBD
:10DE8800656AB0EE674AA6EE074AB4EEE44A34EE95
:10DE9800666AF1EE10FA48BFB0EE456A022A83EDD1
:10DEA800016A3FF4E0AD91ED0A6A26EE656AB0EECC
:10DEB800674AA6EE074AB4EEE44A34EE666AF1EE23
:10DEC80010FA48BFB0EE456A032A83ED026A3FF4B0
:10DED800CAAD91ED0E6A26EE656AB0EE674AA6EE07
:10DEE800074AB4EEE44A34EE666AF1EE10FA48BF27
:10DEF800B0EE456A042A83ED036A3FF4B4AD91EDB0
:10DF0800126A26EE656AB0EE674AA6EE074AB4EED4
:10DF1800E44A34EE666AF1EE10FA48BFB0EE456A9C
:10DF2800052A83ED046A3FF49EAD91ED166A26EE4C
:10DF3800656AB0EE674AA6EE074AB4EEE44A74EEA4
:10DF4800666AF1EE10FA48BFF0EE456A062AC3ED9C
:10DF5800056A3FF488ADD1ED1A6A66EEE56AB0EE5F
:10DF6800674AA6EE874AB3EE046AB4EEE44A74EE52
:10DF7800466AF1EE10FA48BFF0EE456A072AC3ED8B
:10DF8800066A3FF470ADD1ED1E6A66EEE55AE5EE1D
:10DF9800877AF4EEE74A77EEC67AF1EE10FAC8BF50
:10DFA800F0EE457AC3ED077A5DE5734BC7ED00BA2D
:10DFB8001B689342BFF6B6A8704B1A88002384F8F2
:10DFC8006431002A41F011846D4A6E4B117818684B
:10DFD80081F00101F4F70AF8FFF7ACB86A4EDFF8F0
:10DFE800E08106F5F47506F51577F6EC017A9BEDF8
:10DFF800080ADBF81432F8EEE77A284627EE800A9A
:10E008009847A5F1E000DBF834319847A5F1700096
:10E01800DBF8A4319847D6F8F400DBF8B830984715
:10E028002435AF42A8EC010ADFD1FEF74BBF4E49B9
:10E038000978C80703D45549098BA4F888115449AD
:10E048005448098890ED037A07EE901AF8EEE77ABB
:10E05800B4EEE77AF1EE10FA40F208864E480088EE
:10E0680007EE900AF8EEE77AB4EEE77AF1EE10FAE6
:10E07800C0F2CC8549484A49D0ED006A91ED006A62
:10E088004848C4ED636ABCEEC75A76EE665A15EE88
:10E09800101AC4ED616AC4ED605A84ED646AA4F88C
:10E0A80088110121D0ED006A84F8941177EE677A1F
:10E0B800FFF73AB93C4B93ED005AB5EEC05AF1EE72
:10E0C80010FA40F30783394BD3ED004AF5EEC04A06
:10E0D800F1EE10FA40F3FE8234EEC77A66EEE95AA2
:10E0E80087EE246AC5EE856AB7EE007AB4EEC76A91
:10E0F800F1EE10FA88BFB0EE476AB5EEC06AF1EEED
:10E1080010FA76EE876AB8BFB0EE6B6A66EE266ADA
:10E11800FAE5274A92ED007AF0EEE76AF4EEC76A6C
:10E12800F1EE10FA7FF790A8224A92ED007AF0EE0D
:10E13800CD6AF4EEC76AF1EE10FA7FF785A81E4A99
:10E1480099ED007AD2ED006AB0EEC77AB4EEE67ABD
:10E15800F1EE10FA7FF578A801220399C4F8681146
:10E1680084F86421FFF774B8C04F0020C031002044
:10E17800E43100202C87002064910020BC7200202C
:10E18800BE720020C0720020587000205450002039
:10E198007C320020803F00207E3200206832002040
:10E1A8006432002084320020449100204C910020E9
:10E1B80078910020749100207C9100200D49002066
:10E1C8008C7F00200299724BD1ED017A93ED007A91
:10E1D800F0EEE77AF4EEC77AF1EE10FA7EF5AAAF20
:10E1E800D1ED027AF0EEE77AB4EEE77AF1EE10FAC2
:10E1F8007EF7A0AFD1ED037AF0EEE77AB4EEE77AD6
:10E20800F1EE10FA7EF796AF624B1B689A077FF51E
:10E21800D3AE6149614BB3F90C20B1F900E0604815
:10E22800AEEB020E00688EEAEE72A2EBEE7282424C
:10E23800BEF680AFB3F90E30B1F90220D21A82EAE5
:10E24800E273A3EBE27398427EF774AFB4E6554BE2
:10E2580099ED007AD3ED006AB0EEC77AB4EEE67AAB
:10E26800F1EE10FA7FF706A8FFF701B807EE103AAB
:10E278004D4BDFF840811B78C4F81061B8EEC77ABF
:10E28800F7EE006A132B86EE879AB8F90400B4F803
:10E2980014519BED080A01F03482444B444A93ED33
:10E2A800001A93ED053A93ED122A93ED176AD3ED10
:10E2B800091A93ED0E4AD3ED015AD3ED063A93EDC0
:10E2C8000A7A93ED0F5AD3ED132AD3ED186AD3EDDA
:10E2D800044AD3ED030A67EE897A69EE288A29EEA3
:10E2E800088AA1EE273A02EB85060021A2EE286AE9
:10E2F800C4F80411C4F80811A1EE884AE5EEA73A5B
:10E30800A7EE085A93ED167AD3ED0D5A93ED021A3B
:10E31800D3ED0C1A86ED003AE2EEA86A64EEC34A21
:10E3280027EE467A93ED0B2AD3ED152A86ED204A7F
:10E33800E0EEC33A65EEC45A93ED143AC3ED053ADC
:10E34800E1EE274AF0EE477AA1EEC45AE2EE085A07
:10E35800E2EEC66AE3EE287AC3ED064A83ED0E5A6A
:10E36800C3ED0F5A86ED406AC3ED176AC3ED187AFC
:10E37800C4F80C11013505F01F05A4F81451A8F8CC
:10E388000400FEF782BCB0EE465AFFF706B800BF9D
:10E3980070910020E88A0020CC3F00201C790020E2
:10E3A8006C9100207C9100202C4900201C780020D2
:10E3B8009875002030490020B94B1B78192B07D8D5
:10E3C8000121B84A01FA03F31A40002A41F0748483
:10E3D800B54BB64EB64F01931B689D061CD5FB7A0C
:10E3E800FF2B04D0B34A12789A4201F2EF80B7F9B2
:10E3F8000880FB7DA6F80080FF2B04D0AD4A127878
:10E408009A4201F2DE80B7F914507580082005F0B1
:10E4180091FC002840F03186B7F90600B6F900C033
:10E42800B6F902E0B7F91210B7F91E20B6F9045090
:10E43800B7F90430B6F906806045A8BF6046714553
:10E44800A8BF7146AA42A8BF2A469C45A8BF034652
:10E458003380B7F91030B6F908009E45B8BF1946A1
:10E46800B7F92A307180B7F91C10B7F934E0434581
:10E47800A8BF43468D42B4BF0D461546B7F93620AE
:10E48800B580B7F92850B6F90A108242A8BF0246EB
:10E49800A845ACBF9846A846B7F94230B6F90C5023
:10E4A800A6F806808B42A8BF0B467045ACBF104645
:10E4B8007046B7F94E203081B7F94000B6F90EE042
:10E4C800AA42A8BF2A468842C8BF0346B7F95A00DD
:10E4D800B7F94C1073817045B7F95830764FA8BF1B
:10E4E80070469E45A8BF0346A942D8BF1146B181D0
:10E4F800F381BB892BB3DFF8D081DFF8D0A1DFF837
:10E50800B09108F11005B8F9023000EE103A504603
:10E51800B8EEC00AF2F77AF824F0AEFDB9F9043083
:10E52800B9F9062000B298420AF1240A09F10C0947
:10E5380003DB82421346A8BF034628F8023FA845DA
:10E54800E1D1574B1B78013B182B72D8DFE813F049
:10E558005F00710071001900710071007100780886
:10E5680071007100710071007100980871007100EC
:10E578007100710071001900860871007100980817
:10E588005F004E4BB6F908101A6802B111609B691A
:10E59800B6F90A2003B11A60019B1B689A0601F1BB
:10E5A800E98602220492D9027FF562AAFE7B112E27
:10E5B8003FF65EAA424B079333F91630DDF8108018
:10E5C80000EE103A4046B8EEC00A751C0CF08EFCFE
:10E5D80006F10E074346EDB29E1BFFB2DDF81C9014
:10E5E80000E0454605F10108A819122D5FFA88F8E0
:10E5F800C0B23FF43DAA39F9153000EE103AB8EE32
:10E60800C00A0CF073FCB845EBD1FFF731BABB7BFD
:10E61800002B42F079802B4B1B7813F0010342F05A
:10E628007380264A1268002A02F04D841360012381
:10E638000493019B1B68980603D4194A1278052A8B
:10E64800B1D1049A13460233551CDBB21046EDB221
:10E658000493B6F9003000EE103AB8EEC00A0CF098
:10E6680045FCB6F9023000EE103A2846B8EEC00A6A
:10E678000CF03CFC019B1B6895E724F0FDFC29F895
:10E688001600FEF70DBC95ED007A0BEB4602B8EECE
:10E69800C78A928F29F8162028EE278AFEF7DEBB54
:10E6A8004490002032413003987F00201C870020CE
:10E6B800F49100204C4800208479002094790020AF
:10E6C800D06E0020C04F00201A8700203C8E00200A
:10E6D800000000005FED026AFFF724BB59023FF516
:10E6E80067A8FFF769B8F9F791FAA94B059A1B785B
:10E6F800DFF8A082801A012BA8F8020000F07582CA
:10E70800072B7EF4DFADF9F781FA0290FEF7DCBD46
:10E71800F9F77CFA029A9F4B801AD880FFF7C3B9A1
:10E72800002F41F0618191ED006A9DED0A5A9A4BE4
:10E7380025EE866AA5EE076AB0EE675AA6EE265A57
:10E74800BDEEC56A16EE107A16EE106AAF42A8BF83
:10E758002E46B842C8BF064606EE106AB8EEC66A2C
:10E76800012A83ED006A3FF479A991ED046A9DEDD1
:10E778000B5A25EE866AA5EE076AB0EE675AA6EE32
:10E78800265ABDEEC56A16EE107A16EE106AAF422A
:10E79800A8BF2E46B842C8BF064606EE106AB8EEB5
:10E7A800C66A022A83ED016A3FF458A991ED086A06
:10E7B8009DED0C5A25EE866AA5EE076AB0EE675AFB
:10E7C800A6EE265ABDEEC56A16EE107A16EE106A47
:10E7D800AF42A8BF2E46B842C8BF064606EE106A2A
:10E7E800B8EEC66A032A83ED026A3FF437A991EDB1
:10E7F8000C6A9DED0D5A25EE866AA5EE076AB0EE05
:10E80800675AA6EE265ABDEEC56A16EE107A16EEBF
:10E81800106AAF42A8BF2E46B842C8BF064606EEE9
:10E82800106AB8EEC66A042A83ED036A3FF416A993
:10E8380091ED106A9DED0E5A25EE866AA5EE076ADF
:10E84800B0EE675AA6EE265ABDEEC56A16EE107AE5
:10E8580016EE106AAF42A8BF2E46B842C8BF064699
:10E8680006EE106AB8EEC66A052A83ED046A3FF41C
:10E87800F5A891ED146A9DED0F5A25EE866AA5EE6E
:10E88800076AB0EE675AA6EE265ABDEEC56A16EEBE
:10E89800107A16EE106AAF42A8BF2E46B842C8BF1B
:10E8A800064606EE106AB8EEC66A062A83ED056AC1
:10E8B8003FF4D4A891ED186A9DED105A25EE866AAA
:10E8C800A5EE076AB0EE675AA6EE265ABDEEC56AEF
:10E8D80016EE107A16EE106AAF42A8BF2E46B8425E
:10E8E800C8BF064606EE106AB8EEC66A072A83ED68
:10E8F800066A3FF4B3A891ED1C6A9DED115A65EEC6
:10E90800865AE7EE055AE6EEA57AFDEEE77A17EEA7
:10E91800901A8D42A8BF0D468842C8BF054607EE2B
:10E92800905AF8EEE77AC3ED077AFFF796B81B4AD4
:10E93800517900293EF4BDAD1949097800293EF402
:10E94800B8AD1278DFED174A07EE902A164AB8EEEE
:10E95800677A128807EE901A06EE902AF8EEE77AA0
:10E96800F8EE666A67EE277AB7EE007AC7EEA63A3F
:10E97800F4EEE43AF1EE10FA88BFF0EE643AF4EE01
:10E98800C73AF1EE10FAB8BFF0EE473AFEF793BD7A
:10E998002C490020304900202C870020948A002030
:10E9A800C93F0020713DAA3FC0490020002E00F059
:10E9B8005482002F41F0D286C049BEF1000F41F0C9
:10E9C8000F8591ED006ADDED0A4ABD4B25EE866A9A
:10E9D800BDEEC55AA4EE876A15EE100AB0EE675A66
:10E9E800A6EE265ABDEEC56A16EE107A16EE106A25
:10E9F800AF42A8BF2E46B842C8BF064606EE106A08
:10EA0800B8EEC66A012A83ED006A3FF427A891EDA3
:10EA1800046A9DED0B5A25EE866AA5EE076AB0EEEC
:10EA2800675AA6EE265ABDEEC56A16EE107A16EE9D
:10EA3800106AAF42A8BF2E468742B8BF064606EE08
:10EA4800106AB8EEC66A022A83ED016A3FF406A886
:10EA580091ED086A9DED0C5A25EE866AA5EE076AC7
:10EA6800B0EE675AA6EE265ABDEEC56A16EE107AC3
:10EA780016EE106AAF42A8BF2E468742B8BF0646B8
:10EA880006EE106AB8EEC66A032A83ED026A3EF4FF
:10EA9800E5AF91ED0C6A9DED0D5A25EE866AA5EE5F
:10EAA800076AB0EE675AA6EE265ABDEEC56A16EE9C
:10EAB800107A16EE106AAF42A8BF2E468742B8BF3A
:10EAC800064606EE106AB8EEC66A042A83ED036AA3
:10EAD8003EF4C4AF91ED106A9DED0E5A25EE866A9C
:10EAE800A5EE076AB0EE675AA6EE265ABDEEC56ACD
:10EAF80016EE107A16EE106AAF42A8BF2E4687426D
:10EB0800B8BF064606EE106AB8EEC66A052A83ED57
:10EB1800046A3EF4A3AF91ED146A9DED0F5A25EEF9
:10EB2800866AA5EE076AB0EE675AA6EE265ABDEECB
:10EB3800C56A16EE107A16EE106AAF42A8BF2E46C6
:10EB48008742B8BF064606EE106AB8EEC66A062ABD
:10EB580083ED056A3EF482AF91ED186A9DED105A77
:10EB680025EE866AA5EE076AB0EE675AA6EE265A23
:10EB7800BDEEC56A16EE107A16EE106AAF42A8BF4F
:10EB88002E468742B8BF064606EE106AB8EEC66A39
:10EB9800072A83ED066A3EF461AF91ED1C6A9DED8C
:10EBA800115A65EE865AE7EE055AE6EEA57AFDEEAD
:10EBB800E77A17EE901A8D42A8BF0D468842D8BF53
:10EBC800284607EE900AF8EEE77AC3ED077AFEF7D3
:10EBD80044BF3C4B93ED006AFFF786B8F9F716F887
:10EBE8000590FEF789B9DFF81081F9F70FF8364A72
:10EBF800D4F8783112680290C31A9A1AC4F87801C6
:10EC0800A8F80430A8F80620FEF75EBBB4F888011F
:10EC1800884240F245852D482D49D0ED007A91ED86
:10EC2800007A2C48C4ED637A77EE676AC4ED617A9E
:10EC38000121C4ED606A84ED647AD0ED006ADFEDED
:10EC4800267A84F89411FEF76FBB244B1B88002B9F
:10EC580040F04585224A234B11781868F3F7C6F926
:10EC6800D4F86821039B9A1AFEF733BA1E491F4845
:10EC7800D1ED006A1E4990ED006A0978C4ED636A17
:10EC880084ED646A002940F0B78476EEC65AF0EE47
:10EC9800466ABCEEC76A1748C4ED605A16EE101AE9
:10ECA800C4ED616AA4F88811FF21D0ED006A84F8E8
:10ECB800941177EEC77AFEF737BB00BFE431002026
:10ECC8002C87002044910020F08800206832002022
:10ECD800643200208432002000000000BC72002052
:10ECE800BE720020C0720020748700206C320020A1
:10ECF800687C00208032002030490020D1ED015A84
:10ED080065EEC65AB0EE674AA5EE874AB4EEE44A05
:10ED180074EE665AF1EE10FA48BFF0EE455A012A31
:10ED2800C3ED005A3EF49FAED1ED055A65EEC65AC2
:10ED3800B0EE674AA5EE874AB4EEE44A74EE665A26
:10ED4800F1EE10FA48BFF0EE455A022AC3ED015A17
:10ED58003EF489AED1ED095A65EEC65AB0EE674A5F
:10ED6800A5EE874AB4EEE44A74EE665AF1EE10FA5C
:10ED780048BFF0EE455A032AC3ED025A3EF473AE7B
:10ED8800D1ED0D5A65EEC65AB0EE674AA5EE874A30
:10ED9800B4EEE44A74EE665AF1EE10FA48BFF0EEAB
:10EDA800455A042AC3ED035A3EF45DAED1ED115A1B
:10EDB80065EEC65AB0EE674AA5EE874AB4EEE44A55
:10EDC80074EE665AF1EE10FA48BFF0EE455A052A7D
:10EDD800C3ED045A3EF447AED1ED155A65EEC65A56
:10EDE800B0EE674AA5EE874AB4EEE44A74EE666A66
:10EDF800F1EE10FA48BFF0EE456A062AC3ED056A3F
:10EE08003EF431AED1ED196A66EEC66AB0EE674AD5
:10EE1800A6EE874AF3EE045AB4EEE44A74EE656A45
:10EE2800F1EE10FA48BFF0EE456A072AC3ED066A0C
:10EE38003EF419AED1ED1D6A26EEC66AE6EE077AF3
:10EE4800F4EEE47A77EEE57AF1EE10FAB8BFF0EE78
:10EE5800457AC3ED077AFEF706BEC949BEF1000F31
:10EE680041F04A8191ED006ADDED0A4AC54B25EE75
:10EE7800866ABDEEC55AA4EE876A15EE100AB0EE92
:10EE8800675AA6EE265ABDEEC56A16EE10EA16EEC9
:10EE9800106AAE45A8BF2E467045C8BF064606EEA6
:10EEA800106AB8EEC66A012A83ED006A3EF4D4AD52
:10EEB80091ED046A9DED0B5A25EE866AA5EE076A68
:10EEC800B0EE675AA6EE265ABDEEC56A16EE10EAEF
:10EED80016EE106AAE45A8BF2E468645B8BF064650
:10EEE80006EE106AB8EEC66A022A83ED016A3EF49D
:10EEF800B3AD91ED086A9DED0C5A25EE866AA5EE34
:10EF0800076AB0EE675AA6EE265ABDEEC56A16EE37
:10EF180010EA16EE106AAE45A8BF2E468645B8BF61
:10EF2800064606EE106AB8EEC66A032A83ED026A40
:10EF38003EF492AD91ED0C6A9DED0D5A25EE866A70
:10EF4800A5EE076AB0EE675AA6EE265ABDEEC56A68
:10EF580016EE10EA16EE106AAE45A8BF2E46864594
:10EF6800B8BF064606EE106AB8EEC66A042A83EDF4
:10EF7800036A3EF471AD91ED106A9DED0E5A25EECF
:10EF8800866AA5EE076AB0EE675AA6EE265ABDEE67
:10EF9800C56A16EE10EA16EE106AAE45A8BF2E46F0
:10EFA8008645B8BF064606EE106AB8EEC66A052A58
:10EFB80083ED046A3EF450AD91ED146A9DED0F5A4D
:10EFC80025EE866AA5EE076AB0EE675AA6EE265ABF
:10EFD800BDEEC56A16EE10EA16EE106AAE45A8BF79
:10EFE8002E468645B8BF064606EE106AB8EEC66AD3
:10EFF800062A83ED056A3EF42FAD91ED186A9DED62
:10F00800105A25EE866AA5EE076AB0EE675AA6EE94
:10F01800265ABDEEC56A16EE10EA16EE106AAE451F
:10F02800A8BF2E468645B8BF064606EE106AB8EE5B
:10F03800C66A072A83ED066A3EF40EAD91ED1C6A96
:10F048009DED115A65EE865AE7EE055AE6EEA57A69
:10F05800FDEEE77A17EE901A8D42A8BF0D4688425A
:10F06800D8BF284607EE900AF8EEE77AC3ED077A8C
:10F07800002F7EF4F8ACFEF7F0BC94F8BC31012BFD
:10F0880001F0A184404B97F916005A8897F90AE0D5
:10F098001B883E4910FB03F31EFB02F281FB020CA6
:10F0A80081FB0301D217DB17C2EB2C12C3EB211330
:10F0B80042441D4432807580FFF7AEB9344FD4ED19
:10F0C800017A94ED006A38887B6977EEA77AF0EECA
:10F0D800006AB0EE677AA6EE267A013804EBC00221
:10F0E800D6EE267A083A1033F6EE003A27EE237A5F
:10F0F80067EEA37A84ED207AC4ED217A254C274661
:10F1080004F1800192ED027A92ED036AD7ED036A69
:10F11800D7ED027A53ED014A13ED025A37EE674AEA
:10F1280076EEC65A77EE277AE4EE845A0138A2F1D1
:10F138000802E5EE047A07F1080703F1080336EE42
:10F14800267A01F10801E4EE877AE5EE475A67EE80
:10F15800A37A25EEA37AC1ED007A81ED017AD1D1A7
:10F16800142E7DF446AEF8F751FD029BDFF8288097
:10F17800C01AA8F80200D4F81851FDF73ABE00BF2B
:10F18800E43100202C870020CC3F00201F85EB5164
:10F1980080750020E025002030490020DFF8949495
:10F1A80099F80020900801F08986DFF88CE400F1D6
:10F1B800010C4FEA4C1C0EEB0C070EF12003AEF1CC
:10F1C800700113ED076A53ED056A13ED037A53EDE9
:10F1D800017A53ED025A13ED084A53ED064A13ED2E
:10F1E800045A26EE066A66EEA66A27EE077A67EEE6
:10F1F800A77AA4EE046A20339F42E4EEA46A01F1E0
:10F208001001A5EE057AE5EEA57AF1EEC65AB1EE43
:10F21800E66AF1EEC76AB1EEE77A41ED085A01ED08
:10F22800076A41ED066A01ED057ACAD1ACF1200CF6
:10F23800E64404EB001012F0030318BF0EF1080EA9
:10F248000FD05EED017A1EED027A67EEA77A013BD8
:10F25800E7EE077A0EF1080EB1EEE77AA0EC017A34
:10F26800EFD1142E01F0FE850135C4F81851FDF7D1
:10F278002DBDE34FE348BA68B98922F0D5FCE24BCB
:10F288001E78142E01F07885D4F818510135C4F889
:10F29800185114E7DA4FB7F800E0D7F804C04FEA7E
:10F2A8005E084FEA880204EB8E055FEADE0E04EB87
:10F2B800020300F0A08010320EF1010ED34803EBD8
:10F2C8000E1E2A4410330CF1100605F1100151ED01
:10F2D800032A51ED043A10ED043A10ED032A51EDDA
:10F2E800026A11ED016A50ED020A10ED010A12EDF1
:10F2F800044A12ED035A53ED044A53ED035A13ED31
:10F30800027A53ED017A12ED021A52ED011A73EEE8
:10F31800238A32EE228A40ED048A00ED038A70EED9
:10F32800A68A30EE068A40ED028A00ED018A74EE64
:10F33800848A35EE858A43ED048A03ED038A77EEE5
:10F34800018A37EEA18A43ED028A03ED018A73EE42
:10F35800633A75EE655A16ED035A32EE623A74EE68
:10F36800644A25EE638A16ED044A23EE052A64EE04
:10F37800652AA3EE048A10339E4524EE843AA3EE50
:10F38800842A00F1100006F11006A5EE853A01F175
:10F39800100102F11002E4EE852A01ED078A01ED61
:10F3A800082A02ED073A42ED082A56ED055A16EDED
:10F3B800065A70EEE66A30EE466A31EE477A71EE2A
:10F3C800E77A26EE253A65EEE63A25EE674A67EED5
:10F3D800054AE6EE053AA6EE853AA7EE254AE7EE97
:10F3E800A54A01ED063A41ED053A02ED064A42ED1D
:10F3F800054A7FF46CAF1FFA88F862464146814897
:10F408001CF0D0FA41467A6828461CF0CBFA7E4BAD
:10F418001B78142B7FF4AFAEA5E6D4F81CC1B4F862
:10F4280014917B4BC9F120085FFA88F809EB4C1757
:10F4380003EB87075FEA980301F08484013318011E
:10F448007449724A07EB000E07F1100313ED024AE4
:10F4580013ED035A13ED016A13ED047A51ED024AD4
:10F4680051ED035A51ED016A51ED047A64EE244AD4
:10F4780065EE255A66EE266A67EE277A10339E45B2
:10F4880042ED024A42ED035A42ED016A42ED047A26
:10F4980001F1100102F11002D8D15F49A0F1100268
:10F4A800174401EB020E224418F0030309D0B7EC0D
:10F4B800017AFEEC017A67EE277A013BE2EC017AE9
:10F4C800F5D1B9F1000F41F0C980142E7DF491AC4B
:10F4D800F8F79CFB029BDFF86481D4F81851C01A36
:10F4E800A8F80200FDF785BCD4F81C714B4B4C4AB8
:10F4F800DFED4C7AD2ED008A4B4AF9000B44F8EE66
:10F50800688A9B8809EE103A643BC82BA8BFC823B9
:10F5180068EEA78AF8EE497A782BB8BF782368EEA8
:10F52800A78A07EE903A3944B0EE680A02EB8108E0
:10F53800B8EEE78A23F0ECFDB8EEC99AF0EE409AEF
:10F54800B0EE680A23F046FD38EE097A79EE487A7B
:10F5580028EE098A67EE877AB7EE006A88EE277A7E
:10F56800142EF8EE007A77EE076A60EE277A89EEB5
:10F57800A67A77EE065A36EE477AC6EE256A67EE21
:10F58800A67A27EE267AC8ED006A88ED047AC8EDD7
:10F59800026AC8ED017AC8ED037A01F07384234B3F
:10F5A800194A013783FB073CACEBE77C0CEB4C0CAE
:10F5B8000135A7EB0C0C1678C4F81851C4F81CC117
:10F5C8002DE71B4A32F91350FEF71FBF184A32F9CC
:10F5D8001380FEF70EBFF8F719FB0B4B02901E784D
:10F5E800142E05BFDFF85480D4F81851D4F81851F8
:10F5F800A8F80050FDF752BB76EE665AFFF749BBF4
:10F6080080750020E02500202C490020F0250020EE
:10F618009875002028770020187700209877002018
:10F62800887F002027D4D236407200205655555581
:10F63800D06E00207A750020602600203049002016
:10F64800D54BB6F906101A6802B111609B69B6F974
:10F658000820002B7EF49FAFFEF79EBFDFF8808363
:10F66800002538F9023B00EE103AE8B2B8EEC00ABD
:10F6780001350BF03BFC042DF3D10495FEF7D9BFFF
:10F68800DFF86083002538F9023F00EE103AE8B24F
:10F69800B8EEC00A01350BF029FC062DF3D1ECE7D2
:10F6A800BE49BF48D1ED007ABE4990ED007A09788D
:10F6B800C4ED637A84ED647A002901F0CB8277EE99
:10F6C800676AB948C4ED617AC4ED606AFF21D0ED7C
:10F6D800006ADFEDB67A84F89411FDF725BEB449C7
:10F6E8004B69002B3DF4F5ACB248B34B008893FB53
:10F6F800F0F00B684FF0010E186081F811E0FDF78B
:10F70800E8BCAE4EAE4F96ED004A96ED057AD6EDC2
:10F71800014A96ED066AD6ED046A96ED035AD6EDCF
:10F72800025A67EE897A07EB8503A4EE277AA4EEDE
:10F73800A76A66EEC76AA5EE476AE5EEA76A20EEF5
:10F74800070A86ED056AC6ED066A83ED007A29EE9A
:10F75800088A23F091FC69EE288AD6ED0E5AD6ED78
:10F76800176A96ED091AD6ED121A96ED0F5A96ED0C
:10F77800187A96ED0A2AD6ED132A96ED0D6AD6ED7B
:10F78800167A96ED0C3AD6ED0B3A96ED154AD6ED6B
:10F79800144AE1EE085A002207EB8503E8EEA16A55
:10F7A80000B2C4F80421A2EE085AC4F80821C4F82B
:10F7B8000C21A8EEA27A26EE656A67EEE67AA3EE39
:10F7C800655AA3EE886AA6EEC47AE8EEA47A86EDB6
:10F7D8000E5AC3ED205A86ED0F6AC3ED406A86EDD6
:10F7E800177AC6ED187AFEF7C5BD71494A69002A2D
:10F7F8003DF4A0AC0A6813604B74FDF79BBCBBF9E1
:10F808003C30CBF8242007EE903A0122F8EEE77A54
:10F81800CBF86C30CBF888200023012ECBED1F7A73
:10F82800CBED1E7ACBF8803001F07682AE427EF4C2
:10F8380093A9BBF93E30CBF8703007EE903A00221E
:10F848000123F8EEE77ACBF82820CBF89C30002388
:10F85800012ECBED247ACBED237ACBF8943001F04E
:10F868005F82AE427EF4AAA9BBF94030CBF874306F
:10F8780007EE903A00220123F8EEE77ACBF82C2025
:10F88800CBF8B0300023012ECBED297ACBED287AC6
:10F89800CBF8A8307EF4C4A99FED448A032F39D051
:10F8A800B9F1000F09D007EE909AF8EEE77AF4EE76
:10F8B800C87AF1EE10FA01F14E83424ADBF874304F
:10F8C800126894F82011A8F8060003EB550393FB7F
:10F8D800F5F50023CBF82C5093621363D36231B152
:10F8E800394B1B8823F40063002B7EF49BA9374B0C
:10F8F8001B6813F4003341F0078235491A46C85C87
:10F90800012803F10C0300F042850132152AF6D1D3
:10F91800FEF788B9B0EE480A23F0AEFB00B2BFE7A5
:10F928002C4B187800F00107002F7EF49CA8FEF7F6
:10F9380094B82949DFED297A0968C4ED4C7A11F0A9
:10F94800805840F03C8513F4800800F0DA824FF0CC
:10F958000008B6EE007A67EE877AF4EEE75AF1EE21
:10F9680010FA48BFF0EE675A40F12985C4ED665A8F
:10F97800FDF722BF74EE667AB7EE007AF4EEC77A26
:10F98800F1EE10FAC4ED4C7A41F36A8184EEA77A5D
:10F998008DED0A7AFDF706BF947900207487002060
:10F9A8006C320020687C00208032002000000000BB
:10F9B800C4720020DC72002020A107001C780020FF
:10F9C80098750020542A0020EC8A00208C300020F2
:10F9D800D46D0308C04F0020E08A0020000000809A
:10F9E800228700201E870020BCF1000F01F016803E
:10F9F80091ED006A9DED0A5AAE4B25EE866AA5EE9A
:10FA0800076AB0EE675AA6EE265ABDEEC56A16EE2C
:10FA1800107A16EE106AAF42A8BF2E46B842C8BF89
:10FA2800064606EE106AB8EEC66A012A83ED006A39
:10FA38003EF419A891ED046A9DED0B5A25EE866AED
:10FA4800A5EE076AB0EE675AA6EE265ABDEEC56A5D
:10FA580016EE107A16EE106AAF42A8BF2E46B842CC
:10FA6800C8BF064606EE106AB8EEC66A022A83EDDB
:10FA7800016A3DF4F8AF91ED086A9DED0C5A25EE48
:10FA8800866AA5EE076AB0EE675AA6EE265ABDEE5C
:10FA9800C56A16EE107A16EE106AAF42A8BF2E4657
:10FAA800B842C8BF064606EE106AB8EEC66A032A10
:10FAB80083ED026A3DF4D7AF91ED0C6A9DED0D5AC6
:10FAC80025EE866AA5EE076AB0EE675AA6EE265AB4
:10FAD800BDEEC56A16EE107A16EE106AAF42A8BFE0
:10FAE8002E46B842C8BF064606EE106AB8EEC66A89
:10FAF800042A83ED036A3DF4B6AF91ED106A9DEDDB
:10FB08000E5A25EE866AA5EE076AB0EE675AA6EE8B
:10FB1800265ABDEEC56A16EE107A16EE106AAF4286
:10FB2800A8BF2E46B842C8BF064606EE106AB8EE11
:10FB3800C66A052A83ED046A3DF495AF91ED146A0F
:10FB48009DED0F5A25EE866AA5EE076AB0EE675A54
:10FB5800A6EE265ABDEEC56A16EE107A16EE106AA3
:10FB6800AF42A8BF2E46B842C8BF064606EE106A86
:10FB7800B8EEC66A062A83ED056A3DF474AF91EDC6
:10FB8800186A9DED105A25EE866AA5EE076AB0EE52
:10FB9800675AA6EE265ABDEEC56A16EE107A16EE1C
:10FBA800106AAF42A8BF2E46B842C8BF064606EE46
:10FBB800106AB8EEC66A072A83ED066A3DF453AFA9
:10FBC80091ED1C6A9DED115A65EE865AE7EE055ACD
:10FBD800E5EEA67AFDEEE77A17EE902A9542A8BFE1
:10FBE80015469042D8BF284607EE900AF8EEE77A05
:10FBF800C3ED077AFDF737BF012A41F38D8007EE81
:10FC0800101AB8EEC77AC7EE876AB1EEE68A032FF4
:10FC180015D0B9F1000F09D007EE909AF8EEE77AFF
:10FC2800F4EEC87AF1EE10FA01F19581DBF86C3048
:10FC380003EB550393FBF5F3CBF82430F6E5B0EE70
:10FC4800480A23F019FA00B2E3E7012A41F3688071
:10FC580007EE101AB8EEC77AC7EE876AB1EEE68AE1
:10FC6800032F15D0B9F1000F09D007EE909AF8EEDE
:10FC7800E77AF4EEC87AF1EE10FA01F16C81DBF85C
:10FC8800703003EB550393FBF5F3CBF82830E8E528
:10FC9800B0EE480A23F0F0F900B2E3E7012A7FF753
:10FCA800FBAD07EE101AB8EEC77AC7EE876AB1EE59
:10FCB800E68AF3E52C870020974B1B88DF0540F187
:10FCC800D787964B964A93ED017AD3ED006AD3ED28
:10FCD800027A944B0793BDEEC77AB3F906E0924BCC
:10FCE8000193FDEEE66A17EE103AFDEEE77A118B06
:10FCF800ADF82A3016EE902A17EE903AADF8282083
:10FD0800ADF82C30894A8A48B2F90230B2F900209D
:10FD1800884DD0ED007A9FED887A88484FF47A763E
:10FD280003F5E16306FB03F302F5E16206FB02F269
:10FD380085FB03761E44DB1785FB0275C3EBE623C0
:10FD480077EEC77A079E0078378806901544D21751
:10FD58003046C2EBE522FDEEE77A35467688AD8877
:10FD68008446A3F5FA73761A0089ADF8403017EE89
:10FD7800903AA2F5FA72ADF83260BCF80E60ADF8B0
:10FD880042206D1A401ABCF80A20ADF82E30BCF893
:10FD98000C30ADF83450ADF83800751A0698684E36
:10FDA800ADF83E50AEEB010E7F1A521A5B1A0021D5
:10FDB800ADF836E0ADF83070ADF83A20ADF83C302B
:10FDC80031607160B160F160002801F0CD805D4B59
:10FDD800DFF87C815C4FCDF820B08A4699460994BB
:10FDE8003CE012AB03EB440030F9200CA9F800000A
:10FDF80098F902E001230D4403FA04F4534B57F831
:10FE080025501EFB00F083FB003EC017039B2C42CD
:10FE1800C0EB6E100CBF01244FF0FF3498420EDB8C
:10FE2800059B02FB03F2494B83FB0253D217C2EB3B
:10FE38006313A3EB0C031BB28342A8BF034636F837
:10FE4800112003FB042326F81130069B0AF1010A4E
:10FE58009A4508F1070809F102097BDA98F80600C3
:10FE6800002837D198F8001098F9052005924D0020
:10FE7800681807EB800098F90430C288808898F8E1
:10FE880003E098F80140121A92B2304802FB03F3DB
:10FE980080FB03C0DB17C3EB60134FEA520CA3EBE4
:10FEA8000C031BB20393BEF1000F9AD012AB03EB05
:10FEB800440BB9F900003BF920BC584513DA8644D5
:10FEC800704503DCF3455846A8BF704600B2A9F850
:10FED80000008DE71630C0B203F02CFF0028C1D116
:10FEE800A9F80000B1E783DDA0EB0E0EDE4503DBC9
:10FEF8007045A8BF704683460FFA8BF0A9F800003A
:10FF080076E7B6EE007AF4EEC75AF1EE10FA3FF74C
:10FF180020ADFDF751BC00BFBC3F0020803F002052
:10FF280054500020D06E0020987F0020CC3F002045
:10FF38002C870020C5B3A2910080BB44CC8F002041
:10FF48001C8700207C270020F49100201F85EB519E
:10FF5800D08F0020DDF820B0099C97F90A0033887B
:10FF6800634A644910FB03F3F87A097882FB035269
:10FF7800FF284FEAE373C3EB621200F0E683814285
:10FF880040F2E383079B33F9100097F91650738802
:10FF980010443080564AF87D15FB03F382FB035268
:10FFA800FF284FEAE373C3EB621200F0CB83814270
:10FFB80040F2C883079B33F9100097F92250B388A1
:10FFC800104470804A4A97F8230015FB03F382FB1C
:10FFD8000352FF284FEAE373C3EB621200F0AF83CA
:10FFE800814240F2AC83079B33F9100097F92E50F9
:08FFF800F3881044B0803E4A7A
:020000040801F1
:1000000097F82F0015FB03F382FB0352FF284FEAFA
:10001000E373C3EB621200F09383814240F290835A
:10002000079B33F9100097F93A5033891044F08058
:10003000314A97F83B0015FB03F382FB0352FF287C
:100040004FEAE373C3EB621200F07783814240F220
:100050007483079B33F9100097F946507389104455
:100060003081254A97F8470015FB03F382FB0352C2
:10007000FF284FEAE373C3EB621200F05B83814217
:1000800040F25883079B33F9100097F95250B38917
:1000900010447081184A97F8530015FB03F382FB54
:1000A0000352FF284FEAE373C3EB621200F03F8371
:1000B000814240F23C83079B33F9100097F95E5070
:1000C000F3891044B0810C4A97F85F0015FB03F3E5
:1000D00082FB0352FF284FEAE373C3EB621300F085
:1000E0002383884280F02083079A32F9102013443A
:1000F000F381019BFEF774B91F85EB514C4800203A
:10010000D1ED004A9DED0A4AB54B65EEA44AFDEEDD
:10011000C53AE4EE074AB0EE674AA4EEA64A13EEEB
:10012000900AB4EEC46AF1EE10FAF0EE444A88BFC9
:10013000F0EE454AFDEEE44A14EE90EA14EE906AC1
:10014000AE45A8BF2E467045C8BF064604EE906A6D
:10015000F8EEE44A012AC3ED004A3DF481ACD1ED4A
:10016000044A9DED0B4A65EEA44AE4EE074AB0EE60
:10017000674AA4EEA64AB4EEC46AF1EE10FAF0EEB5
:10018000444A88BFF0EE454AFDEEE44A14EE90EA98
:1001900014EE906AAE45A8BF2E468645B8BF064607
:1001A00004EE906AF8EEE44A022AC3ED014A3DF4F7
:1001B00057ACD1ED084A9DED0C4A65EEA44AE4EE39
:1001C000074AB0EE674AA4EEA64AB4EEC46AF1EE5E
:1001D00010FAF0EE444A88BFF0EE454AFDEEE44ADC
:1001E00014EE90EA14EE906AAE45A8BF2E468645FE
:1001F000B8BF064604EE906AF8EEE44A032AC3ED5F
:10020000024A3DF42DACD1ED0C4A9DED0D4A65EE50
:10021000A44AE4EE074AB0EE674AA4EEA64AB4EE5A
:10022000C46AF1EE10FAF0EE444A88BFF0EE454A97
:10023000FDEEE44A14EE90EA14EE906AAE45A8BFD3
:100240002E468645B8BF064604EE906AF8EEE44AAC
:10025000042AC3ED034A3DF403ACD1ED104A9DEDF1
:100260000E4A65EEA44AE4EE074AB0EE674AA4EEF1
:10027000A64AB4EEC46AF1EE10FAF0EE444A88BF22
:10028000F0EE454AFDEEE44A14EE90EA14EE906A70
:10029000AE45A8BF2E468645B8BF064604EE906A16
:1002A000F8EEE44A052AC3ED044A3DF4D9ABD1ED9A
:1002B000144A9DED0F4A65EEA44AE4EE074AB0EEFB
:1002C000674AA4EEA64AB4EEC46AF1EE10FAF0EE64
:1002D000444A88BFF0EE454AFDEEE44A14EE90EA47
:1002E00014EE906AAE45A8BF2E468645B8BF0646B6
:1002F00004EE906AF8EEE44A062AC3ED054A3DF49E
:10030000AFABD1ED184A9DED104A65EEA44AE4EE7C
:10031000074AB0EE674AA4EEA64AB4EEC46AF1EE0C
:1003200010FAF0EE444A88BFF0EE454AFDEEE44A8A
:1003300014EE90EA14EE906AAE45A8BF2E468645AC
:10034000B8BF064604EE906AF8EEE44A072AC3ED09
:10035000064A3DF485ABD1ED1C4A9DED114A65EE90
:10036000A45AE7EE045AE6EEA57AB4EEE76AF1EE97
:1003700010FAC8BFF0EE457AFEF76EBE04230325DF
:1003800004930220FEF769B98223FCF724BDDFED58
:10039000157AFCF7ECBCD4F8245153003DB1981801
:1003A00001EB80006D784078A842BDF43FAC134467
:1003B00001EB83010023C4F82411A4F8BE31C4F872
:1003C000C031FDF733BCB7EE007A77EE677AF4EE12
:1003D000E75AF1EE10FA88BFF0EE675AFFF7CABA93
:1003E0002C87002000000243D1ED004A9DED0A4A0F
:1003F000D94B65EEA44AFDEEC53AE4EE074AB0EEED
:10040000674AA4EEA64A13EE900AB4EEC46AF1EE6F
:1004100010FAF0EE444A88BFF0EE454AFDEEE44A99
:1004200014EE907A14EE906AAF42A8BF2E46B842FE
:10043000C8BF064604EE906AF8EEE44A012AC3ED0E
:10044000004A3DF40FABD1ED044A9DED0B4A65EE39
:10045000A44AE4EE074AB0EE674AA4EEA64AB4EE18
:10046000C46AF1EE10FAF0EE444A88BFF0EE454A55
:10047000FDEEE44A14EE907A14EE906AAF42A8BF03
:100480002E468742B8BF064604EE906AF8EEE44A6C
:10049000022AC3ED014A3DF4E5AAD1ED084A9DEDDB
:1004A0000C4A65EEA44AE4EE074AB0EE674AA4EEB1
:1004B000A64AB4EEC46AF1EE10FAF0EE444A88BFE0
:1004C000F0EE454AFDEEE44A14EE907A14EE906A9E
:1004D000AF42A8BF2E468742B8BF064604EE906AD8
:1004E000F8EEE44A032AC3ED024A3DF4BBAAD1ED7B
:1004F0000C4A9DED0D4A65EEA44AE4EE074AB0EEC3
:10050000674AA4EEA64AB4EEC46AF1EE10FAF0EE21
:10051000444A88BFF0EE454AFDEEE44A14EE907A74
:1005200014EE906AAF42A8BF2E468742B8BF064677
:1005300004EE906AF8EEE44A042AC3ED034A3DF45F
:1005400091AAD1ED104A9DED0E4A65EEA44AE4EE63
:10055000074AB0EE674AA4EEA64AB4EEC46AF1EECA
:1005600010FAF0EE444A88BFF0EE454AFDEEE44A48
:1005700014EE907A14EE906AAF42A8BF2E468742DE
:10058000B8BF064604EE906AF8EEE44A052AC3EDC9
:10059000044A3DF467AAD1ED144A9DED0F4A65EE79
:1005A000A44AE4EE074AB0EE674AA4EEA64AB4EEC7
:1005B000C46AF1EE10FAF0EE444A88BFF0EE454A04
:1005C000FDEEE44A14EE907A14EE906AAF42A8BFB2
:1005D0002E468742B8BF064604EE906AF8EEE44A1B
:1005E000062AC3ED054A3DF43DAAD1ED184A9DED1A
:1005F000104A65EEA44AE4EE074AB0EE674AA4EE5C
:10060000A64AB4EEC46AF1EE10FAF0EE444A88BF8E
:10061000F0EE454AFDEEE44A14EE907A14EE906A4C
:10062000AF42A8BF2E468742B8BF064604EE906A86
:10063000F8EEE44A072AC3ED064A3DF413AAD1EDC9
:100640001C4A9DED114A65EEA45AE7EE045AE6EE07
:10065000A57AB4EEE76AF1EE10FAC8BFF0EE457A7B
:10066000FEF7A9BA3D4B4FEA88075FEA990801EB0C
:10067000070E03EBCC1C274400F0818408F101082D
:100680004FEA08180CEB08000CF110030EF11001F2
:1006900007F1100213ED024A13ED035A13ED016A3C
:1006A00013ED047A51ED024A51ED035A51ED016AFE
:1006B00051ED047A64EE244A65EE255A66EE266A08
:1006C00067EE277A1033984242ED024A42ED035A10
:1006D00042ED016A42ED047A01F1100102F11002CB
:1006E000D8D1A8F11008C4440EEB0801474419F012
:1006F00003093EF4EEAEBCEC017AF1EC017A67EE50
:10070000277AB9F10109E7EC017AF4D1FEF7E1BEED
:10071000134BB6F90A201B68002B00F0D8831A602F
:1007200001230493FDF789BFB7F95C20DFE4B7F933
:100730005000C3E4B7F94400A7E4B7F938008BE4EC
:10074000B7F92C006FE4B7F9200053E4B7F91400AF
:1007500037E4B7F908001CE42C87002098750020C6
:1007600094790020BCF1000F00F01683A9499DED9B
:100770000A4AD1ED004A65EEA44AE4EE074AB0EE1B
:10078000674AA4EEA64AF0EE444ABEF1000F06D036
:10079000B4EE446AF1EE10FAC8BFF0EE454ABDEE81
:1007A000C55A15EE106ABDEEE45A04EE906A15EED5
:1007B000103A9E4200F3D983AB42A8BF2B4605EE08
:1007C000103AB8EEC55A944B012A83ED005A3DF415
:1007D0004EA991ED045A9DED0B4A25EE855AA4EEE3
:1007E000075AB0EE674AA5EE264AB0EE445ABEF16B
:1007F000000F00F0AA83B4EEC46AF1EE10FA40F3E1
:10080000A4833046A842A8BF284605EE100AB8EED9
:10081000C55A022A83ED015A3DF429A991ED085ADF
:100820009DED0C4A25EE855AA4EE075AB0EE674AB4
:10083000A5EE264AB0EE445ABEF1000F00F07B83CD
:10084000B4EEC46AF1EE10FA40F375833046A84264
:10085000A8BF284605EE100AB8EEC55A032A83ED54
:10086000025A3DF404A991ED0C5A9DED0D4A25EE76
:10087000855AA4EE075AB0EE674AA5EE264AB0EEB6
:10088000445ABEF1000F00F04C83B4EEC46AF1EE9E
:1008900010FA40F346833046A842A8BF284605EE2A
:1008A000100AB8EEC55A042A83ED035A3DF4DFA8B6
:1008B00091ED105A9DED0E4A25EE855AA4EE075A89
:1008C000B0EE674AA5EE264AB0EE445ABEF1000FDC
:1008D00000F01D83B4EEC46AF1EE10FA40F3178302
:1008E0003046A842A8BF284605EE100AB8EEC55A01
:1008F000052A83ED045A3DF4BAA891ED145A9DEDF2
:100900000F4A25EE855AA4EE075AB0EE674AA5EEC7
:10091000264AB0EE445ABEF1000F00F0EE82B4EE6B
:10092000C46AF1EE10FA40F3E8823046A842A8BF4C
:10093000284605EE100AB8EEC55A062A83ED055A78
:100940003DF495A891ED185A9DED104A25EE855A73
:10095000A4EE075AB0EE674AA5EE264AB0EE445A16
:10096000BEF1000F00F0BF82B4EEC46AF1EE10FADF
:1009700040F3B9823046A842A8BF284605EE100AC7
:10098000B8EEC55A072A83ED065A3DF470A891EDDA
:100990001C5A9DED114A65EE855AE4EE075AE5EEC4
:1009A000A67ABEF1000F00F09682F4EEC67AF1EE60
:1009B00010FA40F190823246AA42A8BF2A4604EEBD
:1009C000902AF8EEE44AC3ED074AFDF750B8134900
:1009D00097F916E00B8897F90A20B1F9020010493F
:1009E0001EFB03F3524200FB02F081FB03E21211F3
:1009F00081FB00E1DB17C017C0EB2110991AD31A55
:100A000001440344A8EB01011D4431807580FDF7CA
:100A100007BD00BFE43100202C870020CC3F002020
:100A20001F85EB5191ED006ADDED0A4A25EE866ADD
:100A3000A4EE876AF0EE674AE6EE264ABDEEE46A67
:100A400016EE103A984200F39881AB42A8BF2B46AD
:100A500006EE103AB8EEC66AB8F1000F00F01D833A
:100A6000D54B012A83ED006A3DF401A891ED046A9B
:100A7000DDED0B4A25EE866AA4EE876AF0EE674A42
:100A8000E6EE264ABDEEE46A16EE106AB04200F3C6
:100A90007181AE42A8BF2E4606EE106AB8EEC66A55
:100AA000B8F1000F00F01483022A83ED016A3CF4D0
:100AB000DEAF91ED086ADDED0C4A25EE866AA4EE04
:100AC000876AF0EE674AE6EE264ABDEEE46A16EE65
:100AD000106AB04200F34B81AE42A8BF2E4606EE2C
:100AE000106AB8EEC66AB8F1000F00F0E882032A77
:100AF00083ED026A3CF4BBAF91ED0C6ADDED0D4A6B
:100B000025EE866AA4EE876AF0EE674AE6EE264A8C
:100B1000BDEEE46A16EE106AB04200F32581AE42E3
:100B2000A8BF2E4606EE106AB8EEC66AB8F1000FEE
:100B300000F0E082042A83ED036A3CF498AF91ED63
:100B4000106ADDED0E4A25EE866AA4EE876AF0EEA5
:100B5000674AE6EE264ABDEEE46A16EE106AB04237
:100B600000F3FF80AE42A8BF2E4606EE106AB8EE34
:100B7000C66AB8F1000F00F0B482052A83ED046A5A
:100B80003CF475AF91ED146ADDED0F4A25EE866AEF
:100B9000A4EE876AF0EE674AE6EE264ABDEEE46A06
:100BA00016EE106AB04200F3D980AE42A8BF2E46BE
:100BB00006EE106AB8EEC66AB8F1000F00F0768251
:100BC000062A83ED056A3CF452AF91ED186ADDED1B
:100BD000104A25EE866AA4EE876AF0EE674AE6EED2
:100BE000264ABDEEE46A16EE106AB04200F3B38006
:100BF000AE42A8BF2E4606EE106AB8EEC66AB8F13D
:100C0000000F00F04182072A83ED066A3CF42FAF03
:100C100091ED1C6ADDED114A65EE865AE7EE245A25
:100C2000E5EEA67AFDEEE77A17EE902A904203DC15
:100C3000AA42A8BF2A46104607EE900AF8EEE77AC5
:100C4000B8F1000F7EF4D8AF019A002A7EF4D4AF39
:100C5000D145B8BFF0EE457AFEF7CEBF77EEC76A52
:100C6000F0EE477AFEF731BD5449096811F080581B
:100C70007EF473AEFEF76BBE514B9FED526A93ED5F
:100C8000007A514BD3ED003A4D4BD3ED017A4E4BE8
:100C900093ED014A4A4BD3ED026A4B4BD3ED024A26
:100CA0004A4B37EE237A93ED005AD3ED015A484B65
:100CB000019377EE847A37EE057A76EEA46A77EEC2
:100CC000A57A27EE067A66EE866A67EE867A194678
:100CD000BDEEC77AFDEEE66AFDEEE77A17EE102A62
:100CE0000968CDED036A17EE903AADF82820CE04DE
:100CF000BDF90C20ADF82A30ADF82C2000F1D480DD
:100D0000344A354B0792198BB2F906E0FEF7FEBF65
:100D1000324B1B78032B00F02E810023FEF7F1BD30
:100D20009FED2F8AFEF777BF9FED2D8AFEF79CBFC0
:100D30009FED2C0ADFF8C08025EE800A22F0A0F992
:100D4000D4F81851A8F80600FCF757B82649274AE6
:100D50008E46FEF7ADBB06EE100A4EE706EE100A11
:100D600028E706EE100A02E706EE100ADCE606EEB9
:100D7000100AB6E606EE100A90E606EE100A69E6DC
:100D8000F6F748FF1A4BDFF870801E78029BC01AF6
:100D9000A8F80200FEF77CBA0AAB03EB8202FDEE74
:100DA000C54A9446474672461249034814EE906A73
:100DB000A046E64628E000BF2C870020E08A0020FD
:100DC000CC8600203333333FD8860020E4860020D1
:100DD000987F0020D06E002054500020DC8A002034
:100DE000000000000000C84218770020E025002025
:100DF0002C490020E4310020304900209E45E0ECE1
:100E0000014A01F110012ED0D1ED004AB3EC014AA4
:100E100065EEA44AE7EE044AB0EE674AA6EEA44A9D
:100E2000F0EE444A32B1B4EE446AF1EE10FAC8BFB3
:100E3000F0EE454AFDEEE44A14EE90CA664504EE33
:100E4000906A04DCAC45A8BFAC4604EE90CAF8EE4C
:100E5000E44A002FD2D1019C002CCFD1D145B8BF9C
:100E6000F0EE454ACAE74446FCF701BEF6F7D2FE6B
:100E7000A54BDFF8D4821E78029B99F80020D4F8A5
:100E80001851C01AA8F80400FEF7F2B9F6F7C2FE2E
:100E9000029BDFF8B482D4F81C71D4F81851C01A40
:100EA000A8F80200FEF77FBB984B07931946984BB2
:100EB000B1F906E0198B8E45BCBF5242ADF82C202B
:100EC000FEF724BF934800F1800EFEF7B8B9012366
:100ED0000493FDF7B2BBFDEEE77A17EE902AB2421B
:100EE000FFF66FAD68E5BDEEC55A15EE100AB042CB
:100EF000BFF641AD05EE106A42E5BDEEC55A15EEEE
:100F0000100AB042BFF612AD05EE106A13E5BDEE51
:100F1000C55A15EE100AB042BFF6E3AC05EE106AF2
:100F2000E4E4BDEEC55A15EE100AB042BFF6B4AC0B
:100F300005EE106AB5E4BDEEC55A15EE100AB042D2
:100F4000BFF685AC05EE106A86E4BDEEC55A15EE17
:100F5000100AB042BFF656AC05EE106A57E4A8F886
:100F60000600ABF8B450FCF768BE05EE106A28E442
:100F7000694FFEF7F6BF20F027FCFCF757BE71461D
:100F8000FFF7B5BB94F87431002B7CF497A9FCF7FC
:100F900082B9624BD3ED007AB1EE677AB4EEC7DA6C
:100FA000F1EE10FA48D4B4EEE7DAF1EE10FA88BFA9
:100FB000B0EE67DA5A4BC7ED00BA1B689342BCF635
:100FC000B5A8FDF725B9574A574B10681B689847D5
:100FD000564B9BED007AD3ED007A554BD7ED006A66
:100FE00083ED020A534B67EE277A2B4427EE8C7A67
:100FF000D3ED007A504B67EE277AF0EE665AEDEEAD
:10100000275A93ED006AB1EE467AF4EEC75AF1EE34
:1010100010FA14D5494B1B78012B02D0192B7CF404
:10102000C4A8DFED477AB4EEE7DAF1EE10FACCBFF0
:1010300001230023FCF7C4B8B0EE47DABAE7F4EEB8
:10104000C65AF1EE10FA8CBFB0EE467AB0EE657A71
:10105000E0E7132B05D1B0EE480A22F011F8A9F809
:101060000000B0EE480ADBF8143236489847264BA9
:101070001B78132BB0EE408A7BF404AF22F000F80B
:10108000A9F80200FBF7FEBE019E002E7FF4BBAD67
:10109000D145B8BFB0EE456AB5E5019B002B7FF4A2
:1010A000DFACD145B8BFB0EE456AD9E4019E002E51
:1010B0007FF486ADD145B8BFB0EE456A80E5019EAC
:1010C000002E7FF414ADD145B8BFB0EE456A0EE5F1
:1010D000019E002E7FF4E8ACD145B8BFB0EE456A62
:1010E000E2E4019E002E7FF448ADD145B8BFB0EEDA
:1010F000456A42E5019E002E7FF41CADD145B8BF84
:10110000B0EE456A16E500BF2C490020D06E0020E5
:1011100054500020E0250020F49100208091002010
:1011200064910020F49000200891002040000020ED
:10113000CC8600201C910020849100204490002047
:101140000000964240720020304900202DE9F04F07
:10115000874B2DED028B1C6891B081468CB12046E7
:101160001CF074FF0546002800F0C380814B824AC2
:101170001968914205D08149096811B180481A6007
:101180000160804B804D18781CF06AFF2B788342F9
:1011900004460AD0002840F085807C4E306805F077
:1011A000D7FA7B4B34602C701C707A4B1C68ACB146
:1011B00020461CF04BFF88B1774E337833B96F4B24
:1011C0001B681BB1754901220B603270744B1B7890
:1011D000D3B111B0BDEC028BBDE8F08F714B6E4EF8
:1011E00018781CF03DFF337883420746EED0002884
:1011F00040F09D80694C206805F0AAFA684B276092
:101200001B783770002BE4D1DFF8BCB1DBF800208D
:101210005405DED5DFF85C81634FD8F80020002A42
:1012200000F07081614C38682168411A7C2940F2D5
:10123000698194F804E020604FF0240A0EF1010166
:10124000217105949FED5A8A03935446DFF87CA1DF
:1012500004965E209047D8F8002020469047554BD2
:10126000FAEC016A9B8A07EE103AF8EEE66AB8EEED
:10127000C77AC6EE877A67EE887AFDEEE77ACDED1B
:10128000027ABDF90860F0B211F012FFC6F3072030
:1012900011F00EFF631CDCB2272C00F09980D8F807
:1012A0000020D6E7444B1B68002B3FF47EAF434A37
:1012B00093F9020093795279002B0CBF0023082385
:1012C000002A08BF43F0010303228DE80C0020210F
:1012D0004FF46143002205F07FFA2C4B1860002880
:1012E0003FF463AF2A4A304F012313702B703B68E1
:1012F0005BE7334B1F4F1878DFF87C801CF0B0FEA3
:101300003B68A3EB0803B3FA83F35B098342064609
:101310003FF437AF002840F01B82194C20680028AA
:101320003FF42FAF05F014FA26603E6029E7002C49
:101330003FF44CAFA379002B00F04C81214A52F8C6
:1013400023301E4A94F902005279003218BF01225C
:1013500002218DE806000022102105F03DFA0F4B16
:10136000186000283FF432AF012333702EE700BF2E
:10137000748B0020C44B002069220208788B002067
:10138000B04900207D8B00207E8B0020AC490020DE
:10139000848B0020888B00208C8B00201C6B00200D
:1013A0003A4300208D8B0020E4720020A827002003
:1013B00000007A44B0470020808B0020B44B00200E
:1013C0007C8B0020C87D0308987F0020E847002020
:1013D000039BD8F8002002935E20059C049E904752
:1013E000D8F8002030209047BD4AD2F800A05FFA1C
:1013F0008AF011F05DFECAF3072011F059FED8F80B
:1014000000205E2090472279029B12F0030A36D119
:10141000226841F288318A4200F29A84D8F800208A
:1014200002935E209047D8F8002014209047AD4AE0
:10143000AD49B2F9042081FB02314FEAE27ACAEBEE
:10144000A10A0FFA8AFA5FFA8AF011F031FECAF3A4
:10145000072011F02DFED8F800205E209047D8F824
:1014600000201C209047002011F022FE002011F0E7
:101470001FFED8F800205E2090472279029B12F0D0
:10148000070A00F08583282A3CD14FF0000AD8F8DB
:10149000003084F804A05E203C689847D8F80030FB
:1014A00017209847504611F003FE904BA3FB0423EE
:1014B0008F4A9B0BA2FB03125209C2EB0212A3EB51
:1014C0008203D8B211F0F4FDD8F800305E209847BE
:1014D000D8F8003018209847864BA3FB0423844A91
:1014E0009B09A2FB03125209C2EB0212A3EB820377
:1014F000D8B211F0DDFD504611F0DAFDD8F8003019
:101500005E2098472B78D7F800A043B17A4D286821
:1015100028B17A4B1B78013B012B40F231813378A3
:101520004BB1774D2B6833B1764C3E68236AF31A82
:10153000632B00F29680744B1B78002B4DD1734BBC
:101540001B78002B3FF445AE6E4C236B03F5C33381
:10155000A0339945FFF43DAE94F834306C4AC4F89A
:10156000309002EB8302526A42B310AD04F13B03A8
:10157000684E45F8203D002104F14D033180099368
:1015800080211523A52784F83A30284684F839109D
:1015900084F83870904728463188F1F754FA089D4E
:1015A0005D4804F138016D1A152DA8BF15252A468E
:1015B00021F05CFB594A94F834301570584A0133D5
:1015C00082FB0312A2EBE37202EB42029B1A84F845
:1015D0003430FEE54FF49643B3E6524C2278A2B184
:1015E000514B9B7A53B1F6F715FB504B1B68C31A4E
:1015F000A3F57A73B3F5FA6F07D822784C4B4D49AF
:101600001868EFF7FCFB002323703E4CA36A03F538
:10161000C333A033994592D3474DC4F828902B7813
:10162000002B40F05C84454D2B78002B40F07683F6
:1016300094F82C2042498D5CEA0700F10D86AB0737
:1016400000F1CD856F0700F1BB843E4A94F82C3041
:101650001178013393FBF1F201FB123384F82C3043
:101660006DE7DFF880A0DFF88080374F412011F070
:1016700093FCBAF9023088FB0320DB17C3EBA00010
:1016800080B211F06FFCBAF9003088FB0320DB1741
:10169000C3EBA00080B211F065FCBAF9043088FBFE
:1016A0000320DB17C3EBA00080B211F05BFC39789C
:1016B0002868EFF7CDFB94F8243013F0010200F016
:1016C0008083224A26620133DBB2A2FB0312D208D6
:1016D00002EB8202A3EB420384F824302BE700BF25
:1016E000FC3F0020CC3F00206766666673B2E7458A
:1016F00089888888D34D6210AC490020848B0020F3
:101700001C6B0020A82700208E8B00209D8B0020C2
:1017100008580308EE8A0020BC730020D173002013
:1017200056555555708B00205450002028750020C8
:10173000908B0020308B0020948B0020958B002014
:10174000988B00209C8B0020A86F0020CDCCCCCCA7
:10175000B44B94F902005B79B3FA83F35B0902217D
:101760008DE80A002A464FF41653042105F034F898
:10177000AD4B186000283FF404ADC7F8008000E5C9
:10178000AA4CDFF8D8820AE01B2B00F0B5820D2BA3
:1017900000F0E3814FF0010388F800302868EFF78C
:1017A00054FB90B32868EFF74AFB83B27E2B3A686C
:1017B00024D098F800100029F0D1227A002AE3D032
:1017C0007D2B00F0DA8194F818E0BEF1000F03D011
:1017D00080F02003DBB22176511CC9B222440929D2
:1017E0002172137300F0BF810829D7D8E28A13440D
:1017F00003EB132303F0FF03E382CFE74FF0000373
:101800002372637288F80030C8E7637E23B1637B7C
:101810006076302B00F08485627A854BDFF840C219
:10182000DFF840824FF0010E002A3FF478AE3968AD
:10183000A1EB0A01012900F28D81A57E002D40F067
:101840006582E17E33F8110010B984F81BE0EBE704
:101850000131B0F5826FE17600F006811CD9B0F558
:10186000E26F00F0908030D9B0F5046F00F09880FE
:10187000B0F5116F00F09E80B0F5E46FD4D16D4AE1
:10188000156C918A642303FB05F393FBF1F111F0CE
:10189000B9FB0023637242E6B0F5007F00F0A2803E
:1018A00029D8B0F5807F00F02D81B0F5887FBBD1BD
:1018B000DCF800104907B7D55F4B4FF48870196802
:1018C00011F0A0FB0023637229E6B0F5C06F00F0B1
:1018D0009A80B0F5E06FA7D1564A906B918A642345
:1018E00003FB00F34FF4E06093FBF1F111F08AFB8E
:1018F0000023637213E6B0F5047F00F01181B0F5A8
:10190000806F91D1217F0131CBB2032B00F23B815B
:1019100042F21071237701FB03F1484B1B88002B27
:1019200040F02F810131464B1B78DB07454B1B886C
:1019300048BF0431DD0748BF0A31980748BF14315A
:101940001A0648BF2831DD0548BF2831580748BF6F
:1019500064311A0748BFC8319D0548BF01F5C871F9
:10196000980648BF01F57A71DA0648BF01F5FA61B9
:101970005D0648BF01F57A614FF4806011F042FBCB
:1019800000236372CBE52B4AD2F83CE0918A6423B2
:1019900003FB0EF393FBF1F111F034FB6572BEE52E
:1019A000294BB3F9041001EB8101490011F02AFB26
:1019B0006572B4E598F8051000293FF435AF234966
:1019C000097800293FF430AF214B1B8803EB8303D8
:1019D0005B004FF4116093FBF1F111F013FB002356
:1019E00063729CE598F8061000293FF41DAF194B6F
:1019F00019491B6881FB0321DB17C3EBA10111F01F
:101A000001FB65728BE598F8061000293FF40CAFD6
:101A1000104B4FF4C060996811F0F4FA0023637220
:101A20007DE500BFB44B0020B0490020A82700206E
:101A300008580308B0470020FC3F0020EC8A002033
:101A4000C04F0020BC3F0020CC3F0020C93F0020F9
:101A5000C0490020B4490020676666664400002043
:101A6000E88A0020948A0020DCF8001011F02001A0
:101A70007FF4DAAEDBF80000000600F13784AA49F3
:101A8000097B00293FF4D0AE617F032900F267840F
:101A9000DFE801F02E241602A44B1B6859799A79CD
:101AA000DB7901F1407101EB022101EB03410023DD
:101AB00063774FF4826011F0A5FA002363722EE57C
:101AC0009B4B1A68137A507992781B0403EB00231E
:101AD00013444A1C627703EB0161EAE7944B1A68EE
:101AE000D379107952781B0403EB00231344F0E7F9
:101AF0008F4B1A689379D07812781B0403EB00237C
:101B00001344E6E7DCF8001048077FF58DAE894BFB
:101B10004FF48070196811F075FA00236372FEE4C7
:101B200098F8051000293FF47FAE83490978002911
:101B30003FF47AAE7C4B5B7B002B00F0F8837F4B4D
:101B40001B8893FBF1F101EB810149004FF4047014
:101B500011F058FA00236372E1E44FF001012172A1
:101B60002373E2821AE6E28AC2F1FF0293427FF413
:101B700011AE4FF0010363760CE64FF001032376BC
:101B80000CE60231CFE60123237742F21071C4E65E
:101B9000D8F8002002935E209047D8F80020022059
:101BA0009047FF2010F0C0FF0278029BFF2A00F050
:101BB000B38390F901004FEAE07A5FFA8AFAC0B283
:101BC000029311F075FA504611F072FAD8F800201D
:101BD0005E209047D8F8002003209047FF2010F0A7
:101BE000A3FF0278029BFF2A1CBFB0F908A05FFA8E
:101BF0008AF3184614BFCAF3072A4FF0000A11F0FF
